:020000040800F2
:1000000000000120590C0408A50C040825EC000888
:10001000A50C0408A50C0408A50C040800000000A9
:10002000000000000000000000000000A50C040813
:10003000A50C040800000000A50C040845E7000812
:10004000A50C0408A50C0408A50C0408A50C0408BC
:10005000A50C0408A50C0408A9EC0008D5ED0008BF
:1000600099ED00085DED000821ED0008EDBD0008E8
:10007000DDBD0008CDBD0008BDBD0008ADBD000858
:1000800099BD000885BD0008A50C0408A50C04084E
:10009000A50C0408A50C0408A50C0408E5EC000850
:1000A000A50C040869A90008A50C040859A90008B2
:1000B000A50C040849A9000839A900080DC40008C6
:1000C00019C40008F5C3000801C40008A50C040801
:1000D000A50C0408759F0008699F0008A50C04087A
:1000E0006DEC0008A50C0408A50C0408A50C040878
:1000F00025A90008A50C040815A9000871BD000871
:10010000A50C0408A50C040829A90008A50C0408DE
:100110005D9F0008A50C0408A50C0408155E0208E4
:100120005DBD000849BD000835BD000821BD0008BF
:100130000DBD0008000000000000000000000000ED
:10014000000000000000000000000000655F0208E1
:10015000F9BC0008E5BC0008D1BC0008A50C0408E7
:10016000DDC30008E9C30008A50C0408A50C0408B9
:10017000A50C0408A50C0408000000000000000005
:10018000A50C0408A50C0408A50C0408A50C04087B
:10019000A50C0408A50C040800000000A50C040828
:1001A000000000000000000000000000A50C040892
:1001B000A50C0408A50C04080000000000000000C5
:1001C000000000000000000000000000000000002F
:1001D000000000000000000000000000A50C040862
:0801E000980704000100000073
:1001E80002020300202001201C2001200000000042
:1001F80000000000160008002C20012034200120F7
:10020800000000008406000803000100D026012039
:10021800D826012000000000000000001D00010099
:10022800E826012078270120000000008C0600083D
:1002380027000400082701207C2701200000000077
:100248008E06000803123300FF290120CC29012063
:10025800000000009406000825005A001829012013
:10026800722901200000000000000000F6110C00B7
:100278000C2901200029012000000000C806000800
:1002880001200800102B01205C2B01200000000039
:10029800D40600081A000800F42A0120642B012063
:1002A80000000000DC06000809020100DC2B012028
:1002B8009C39012000000000E406000812100B0021
:1002C800EE380120A039012000000000E6060008F1
:1002D8000C00240000390120AC3901200000000086
:1002E800D1B8020829005000C43F0120A0400120D5
:1002F800000000000000000014000200C03F0120C0
:10030800F040012000000000F20600080500060089
:100318003C460120A847012000000000F406000820
:100328000E20EA0020450120B0470120000000000F
:1003380049E4010813000400684601209C48012094
:1003480000000000FC060008020103000B45012024
:10035800A048012000000000F9B8020800020500CA
:10036800A44801201C4C01200000000000000000EF
:100378001E000400E4490120244C01200000000074
:100388000007000822000C0064490120284C0120C5
:1003980000000000040700080B201000604F012037
:1003A800984F012000000000100700081F000E00F1
:1003B800CC4C0120A84F01200000000020070008B5
:1003C80005020100204D0120B84F01200000000067
:1003D8002E07000801010400FC4F012034620120AF
:1003E800000000000000000008020C00D26101209B
:1003F80038620120000000008DC8000806021000C5
:10040800DE6101204462012000000000B9C8000834
:10041800070202001C620120546201200000000053
:1004280030070008FF0101003062012058620120F6
:10043800000000003207000802000C00F0610120F3
:100448005C6201200000000000000000F7010600C7
:10045800CC61012068620120000000003407000818
:10046800FE01080090640120A06401200000000043
:10047800E5C7000803010600086A0120446A012054
:10048800000000003A07000818102C000C77012023
:10049800847F01200000000049810308FD01240039
:1004A800E8760120B07F0120000000000BC800089A
:1004B800FB010100F0750120D47F0120000000003D
:1004C800DDC70008FC010900BC740120D87F0120A9
:1004D80000000000A9C700080A101200A46C01203F
:1004E800E47F012000000000400700080600160015
:1004F80054770120F87F01200000000069E401081A
:10050800340010004C6A0120108001200000000017
:10051800ADDB03080A020A00308101204081012076
:100528000000000052070008040080006CB10120A0
:10053800ECB301200000000000000000F9010400F5
:10054800F09301206CB40120000000007DC8000871
:100558001B00F40078B4012018B701200000000047
:10056800F585020826000E001CB801200CB80120F1
:1005780000000000C16403082C00100044BA0120E8
:1005880034BA012000000000257C03082B00240059
:1005980078BA012054BA012000000000F57B030856
:1005A80010000300A0BC0120A4BC01200000000032
:1005B8005C07000828000C0094BC0120A8BC01209E
:1005C80000000000600700082300100084BC012020
:1005D800B4BC012000000000C12302081900050076
:1005E8007CBC0120C4BC0120000000006C0700088E
:1005F800F811010078BC0120CCBC012000000000EB
:10060800720700080001040074BC0120D0BC01205E
:1006180000000000740700082F00110060BC0120D2
:10062800D4BC012000000000780700082A00600000
:10063800C0C4012060C401200000000085DB03085D
:100648001500700098BE012020C5012000000000A0
:10065800000000000D003400CCCA012000CB0120AE
:1006680000000000ADE30208FA01020060C70120A3
:0C06780034CB01200000000001C8000885
:10068400C40900001901282800002003000000000C
:100694000000000000000000000000000000000056
:1006A4000000000000000000000000000000000046
:1006B4000000000000000000000000000000000036
:1006C4000000010000000000000000000000000025
:1006D400E8036400040A00017E05EA05B40532005B
:1006E40018000000000100414646370000000300E6
:1006F40020000200010000001800000000000100BA
:10070400C800141E010064002C0128002B21231EA4
:1007140064000200000001000A012900000000003A
:10072400000001000000000500000000013C000082
:100734003D01000000000401010000000030010040
:10074400005A0000000090012C01C8006400000061
:100754004A01B400D60100000001050000000001B8
:100764000000000000000000000028010000040058
:1007740065FDC40900000000000000000000000046
:05078400000000000070
:100789000000803F0000803F0000803F0000803F64
:100799000000803F0000803F0101000058700408FC
:1007A90000A40408000000000000000068700408AC
:1007B9007070040800000000012000007470040833
:1007C9007C700408000000000140000080700408EB
:1007D9003C83040800000000012000008C7004081C
:1007E9009870040800000000040000009C700408D0
:1007F900A87004080000000004000000AC700408A0
:1008090048990408000000000100000002010000EE
:10081900685E0C00FF0000000000803F0000803F80
:10082900FFFFFFFF0000803F01010100349C040825
:100839000E000000E50902080000000000000000A9
:100849002C020120F89B04080000000000000000B1
:10085900000000000000000000A4040800000000DF
:1008690000000000C806012004000000849B040861
:100879000C00000079720208A406012000000000A3
:100889009C9A04080C00000049720208980601208D
:1008990000000000189C0408080000000000000087
:1008A9008C06012004000000089C04080C000000CC
:1008B900057202088006012000000000849A0408DD
:1008C90003000000AD740208680601200000000062
:1008D900109C040803000000AD74020850060120B2
:1008E90000000000889A04080100000000000000D0
:1008F9000000000000000000000000000D000000E2
:10090900000000000000000000000000F89B04083F
:1009190000000000000000000000000000000000CE
:1009290000A404080000000000000000C80601201F
:10093900040000001C9B040803000000610A02086F
:100949003806012008000000089C04080C0000007B
:10095900057202088006012000000000849A04083C
:1009690003000000AD7402086806012000000000C1
:10097900109C040803000000AD7402085006012011
:1009890000000000889A040801000000000000002F
:100999000000000000000000000000000D00000041
:1009A900000000000000000000000000209C040876
:1009B900000000000000000000000000000000002E
:1009C90000A404080000000000000000C80601207F
:1009D90004000000249B040803000000AD74020811
:1009E900B006012000000000889A040801000000F8
:1009F90000000000000000000000000000000000EE
:100A09000D000000000000000000000000000000D0
:100A19002D202D2D202D2D2D2D202D2D2D2D00007E
:100A290000000000000000000000000000000000BD
:100A3900762B012088130C1701000000782B012068
:100A490088130C17000000005C9A040800000000DD
:100A59000000000000000000000000006C9A04087B
:100A69000800000000000000BC0201200400000092
:100A7900789A04080800000000000000B002012074
:100A890000000000849A04080400000035100208E0
:100A99000000000000000000889A0408010000001E
:100AA900000000000000000000000000000000003D
:100AB9000D00000000000000000000000000000020
:100AC900742B012088130C1701000000722B0120E0
:100AD90088130C1700000000CC9A04080E000000CF
:100AE9003D0A02080000000000000000C8020120C1
:100AF900D42B012001000000EC5B0408702B0120BD
:100B090001000000F85B04083A6A012002000000B5
:100B1900005C040832B2012000000000000000005F
:100B290030B2012000000000000000002EB20120B8
:100B390000000000000000002CB2012000000000AD
:100B4900000000002AB2012000000000000000009F
:100B590028B2012000000000000000003019012027
:100B690000000000000000006F2B012002000000BF
:100B79000C5C0408D49A040800000000000000007E
:100B890000000000000000006C9A04080800000042
:100B9900000000004C03012004000000789A0408BA
:100BA90008000000000000004003012000000000D0
:100BB900849A0408040000001D0A020800000000CD
:100BC90000000000889A04080100000000000000ED
:100BD9000000000000000000000000000D000000FF
:100BE900000000000000000000000000E49A040872
:100BF90000000000000000000000000000000000EC
:100C0900F49A04080C000000A1710208880301206D
:100C190004000000009B04080C0000007D6D020820
:100C29007C030120040000000C9B04080C00000058
:100C3900697102087003012000000000189B040874
:100C490003000000810A020858030120080000007F
:100C5900249B040803000000AD740208B0060120BB
:100C690000000000889A040801000000000000004C
:100C79000000000000000000000000000D0000005E
:100C89000000000000000000000000002C9B040888
:100C9900000000000000000000000000000000004B
:100CA900349B0408040000005110020800000000F1
:100CB90000000000889A04080100000000000000FC
:100CC9000000000000000000000000000D0000000E
:100CD9000000000000000000000000008C9B0408D8
:100CE90000000000000000000000000000000000FB
:100CF900989204080C00000000000000E80301209D
:100D0900040000009C9B040808000000000000008B
:100D1900DC03012004000000A89B0408080000006F
:100D290000000000D003012004000000B09B04086B
:100D39000800000000000000C403012004000000B6
:100D4900B89B04080800000000000000B803012057
:100D590004000000C09B0408080000000000000017
:100D6900AC03012004000000C89B0408080000002F
:100D790000000000A003012004000000D09B04082B
:100D89000800000000000000940301200400000096
:100D9900889A04080100000000000000000000001B
:100DA90000000000000000000D000000000000002D
:100DB9000000000000000000D89B04080E0000009D
:100DC9002D0A02080000000000000000F4030120C1
:100DD900E09B04080E000000000000000000000075
:100DE900000000006C040120E89B04080E000000CC
:100DF9000000000000000000000000000C050120B8
:100E0900D52B012004000000185C040836390120A4
:100E1900E0150C1700000000D22B0120080000008B
:100E2900C85B0408D32B0120050000002C5C0408D2
:100E3900F09B04080E000000000000000000000004
:100E4900000000005C0501202D202D2D202D2D2DC9
:100E59002D202D2D2D0000000000000000000000B5
:100E690000000000000000000001010165290208DE
:100E79000000000000000000010000000A06000256
:100E8900000000400100000009074300020104C0FE
:100E990032090400000102020100052400100105C5
:100EA9002401000104240202052406000107058229
:100EB900030800FF09040100020A000000070501F8
:100EC90002400000070581024000000009024300BA
:100ED900020100C0320904000001020201000524D8
:100EE9000010010524010001042402020524060062
:100EF900010705820308001009040100020A000025
:100F09000007050102000200070581020002000036
:100F190009024300020100C0320904000001020273
:100F29000100052400100105240100010424020226
:100F390005240600010705820308001009040100C1
:100F4900020A0000000705010240000007058102AE
:100F5900400000001A03000000000000000000002B
:100F69000000000000000000000000000000000078
:100F790020700020702D720050A204080E0000009D
:100F8900000000000000000000000000E81501203A
:100F9900FFFFFFFFFA000000010000000100000050
:100FA9002C9B040800000000000000000000000065
:100FB90000000000C19C040804000000C50F0208DD
:100FC9000000000000000000889A040801000000E9
:100FD9000000000000000000000000000000000008
:100FE9000D000000000000000000000000000000EB
:100FF900D6B201200100C40900000000D4B20120CA
:101009000100C40900000000D2B201200100C40996
:1010190000000000D0B201200100C4090000000056
:10102900CCB201200100C40900000000CEB20120A9
:101039000100C40900000000CAB201200100C4096E
:1010490000000000C8B201200100C409000000002E
:10105900F49C04080E0000000000000000000000DD
:101069000000000020080120046A01209CFF2C01D7
:1010790000000000AA0001200A0000008C5D04089D
:101089006C2B0120E0150C1700000000A9000120BD
:1010990008000000C85B0408A80001200500000042
:1010A9002C5C04086E2B012002000000A45D0408DA
:1010B900424601200100FF7F010000003A4601205D
:1010C90002000000B05D040814450120030000007F
:1010D900C05D04081345012003000000C05D040839
:1010E900124601200000F401010000001046012011
:1010F9000000F401010000000E4601200000F40187
:10110900010000000C4601200000F401010000006C
:101119000A46012000FF010026460120E803D00706
:101129000A00000024460120006401000A000000B2
:1011390025460120006401000A0000001E46012026
:10114900006401000A000000234601200064010038
:101159000A00000022460120006401000A00000084
:1011690021460120006401000A0000001D460120FB
:1011790000FF01000A0000001C46012000FF0100D9
:101189000A0000001C4501200000F40101000000D4
:101199001A4501200000F401010000001845012052
:1011A9000000F40101000000164501200000F401CF
:1011B900010000001946012000C80100184601205D
:1011C90000C801001746012000C801001646012089
:1011D900006401000A0000001546012000FF01001B
:1011E9000A0000003146012000C8010030460120F4
:1011F90000C801002F46012000C801002E46012029
:1012090000C801002D46012000C801002C4601201C
:1012190000C801002B46012000C801002A46012010
:1012290000C801002946012000C80100FC9C0408EF
:1012390000000000000000000000000000000000A5
:101249000C9D04080900000000000000C4080120EA
:1012590004000000149D04080900000000000000BB
:10126900B808012004000000E4A0040809000000F7
:1012790000000000AC08012004000000589C04088C
:101289000900000000000000A0080120040000007F
:101299001C9D0408090000000000000094080120BA
:1012A90004000000249D040809000000000000005B
:1012B90088080120040000002C9D04080900000092
:1012C900000000007C08012004000000349D04088F
:1012D900090000000000000070080120040000005F
:1012E900889A0408010000000000000000000000C6
:1012F90000000000000000000D00000000000000D8
:101309000000000000000000209E0408000000000A
:10131900000000000000000000000000309E0408EA
:101329000500000000000000124501200000000037
:10133900889A040801000000000000000000000075
:1013490000000000000000000D0000000000000087
:101359000000000000000000389E040800000000A2
:1013690000000000000000000000000000A40408C4
:1013790000000000000000009002012004000000AD
:10138900549C04080C0000000D10020824090120D7
:1013990000000000849B04080C000000B109020849
:1013A90018090120000000009C9A04080C000000A4
:1013B9007D0902080C09012000000000189C04089E
:1013C90008000000000000000009012004000000DE
:1013D900089C04080C00000069090208F4080120AF
:1013E90000000000449E04080900000000000000FD
:1013F900E808012004000000849A040803000000A2
:10140900AD740208D008012000000000889A040881
:1014190001000000000000000000000000000000C2
:10142900000000000D0000000000000000000000A6
:10143900000000004C9E04080000000000000000AD
:1014490000000000000000005C9E04080C00000081
:10145900000000003C09012000000000649E04080F
:101469000A00000000000000C4460120000000003E
:10147900709E04080A00000000000000CC4601200C
:1014890000000000789E04080A0000000000000027
:10149900D446012000000000809E040808000000D6
:1014A900000000003009012000000000889E0408A7
:1014B900040000008176020800000000000000001E
:1014C900889A0408010000000000000000000000E4
:1014D90000000000000000000D00000000000000F6
:1014E9000000000000000000949E040800000000B5
:1014F900000000000000000000000000A89E040891
:101509000C00000000000000540901200000000048
:10151900B89E040804000000F572020800000000EB
:1015290000000000C09E04080C000000000000003C
:101539004809012000000000D49E040804000000AE
:10154900D57202080000000000000000889A040813
:101559000100000000000000000000000000000081
:10156900000000000D000000000000000000000065
:1015790000000000DC9E04080000000000000000DC
:101589000000000000000000F09E040807000000B1
:10159900000000009009012000000000FC9E0408E2
:1015A900080000000000000084090120000000007C
:1015B900089F0408080000000000000078090120C5
:1015C90000000000149F040808000000000000004B
:1015D9006C09012000000000209F04080800000099
:1015E900000000006009012000000000889A04083A
:1015F90001000000000000000000000000000000E1
:10160900000000000D0000000000000000000000C4
:10161900000000002C9F04080000000000000000EA
:10162900F307012000000000389F04080B000000A8
:1016390000000000F809012000000000409F040894
:101649000B00000000000000EC0901200000000070
:101659004C9F04080B00000000000000E009012075
:1016690000000000589F04080B0000000000000063
:10167900D409012000000000649F04080B00000049
:1016890000000000C809012000000000709F040844
:101699000B00000000000000BC0901200000000050
:1016A900789F04080B00000000000000B009012029
:1016B90000000000849F04080B00000000000000E7
:1016C900A409012000000000909F04080800000000
:1016D900000000009809012000000000889A040811
:1016E90001000000000000000000000000000000F0
:1016F900000000000D0000000000000000000000D4
:10170900000000009C9F0408000000000000000089
:101719000000000000000000B09F0408080000005D
:1017290000000000280A012000000000BC9F0408F6
:1017390008000000000000001C0A01200000000051
:10174900C89F04080800000000000000100A0120DA
:1017590000000000D49F04080800000000000000F9
:10176900040A012000000000889A04080100000012
:101779000000000000000000000000000000000060
:101789000D00000000000000000000000000000043
:10179900DC9F04080000000000000000F0070120A1
:1017A90000000000EC9F04080B000000000000008E
:1017B900580A012000000000F89F04080B000000EF
:1017C900000000004C0A01200000000004A00408E9
:1017D9000700000000000000440A0120000000008A
:1017E90010A0040807000000000000003C0A0120C6
:1017F900000000001CA00408070000000000000011
:10180900340A012000000000889A04080100000041
:1018190000000000000000000000000000000000BF
:101829000D000000000000000000000000000000A2
:1018390028A004080000000000000000F0070120B3
:101849000000000034A004080700000000000000A8
:10185900A40A0120000000003CA0040807000000C1
:10186900000000009C0A01200000000044A00408B8
:101879000700000000000000940A01200000000099
:101889004CA0040807000000000000008C0A012099
:101899000000000054A00408070000000000000038
:1018A900840A0120000000005CA004080700000071
:1018B900000000007C0A01200000000064A0040868
:1018C9000700000000000000740A01200000000069
:1018D9006CA0040807000000000000006C0A012049
:1018E9000000000074A004080700000000000000C8
:1018F900640A012000000000889A04080100000021
:1019090000000000000000000000000000000000CE
:101919000D000000000000000000000000000000B1
:101929007CA004080E00000000000000496E0208B7
:1019390000000000AC0A012010450120170000003A
:10194900D05D04080F4501200A3201000E4501202F
:1019590001FA01000A45012000C8010008450120DB
:10196900E803D00701000000414C49454E464C4967
:101979004748544E4746370084A004080E0000002B
:101989005F6E020800000000A9720208880B01209E
:101999008CA004080E000000CB080208000000001B
:1019A90000000000D80B012094A004080E000000DC
:1019B90061760208917002088D700208B40C01204A
:1019C9009CA004080E000000816E020800000000BF
:1019D90000000000680D0120A4A004080E0000000A
:1019E900096F0208D96E020800000000F40D0120F9
:1019F900ACA004080E000000816F0208C56F020840
:101A090000000000940E01201A4601200103010084
:101A1900B8A004080E000000B56E0208916E020815
:101A290000000000840F0120C0A004080E0000007F
:101A3900396F020815730208000000001010012018
:101A4900CCA004080E000000F56F02085D730208BF
:101A590000000000B010012014460120010301001C
:101A6900D4A00408000000000000000000000000ED
:101A790000000000E0A004080800000000000000C9
:101A8900DC11012000000000E8A0040807000000A4
:101A990000000000D411012000000000F8A0040893
:101AA9000700000000000000CC1101200000000028
:101AB90004A104080700000000000000C41101206F
:101AC9000000000010A104080C0000000000000044
:101AD900B8110120000000001CA104080300000047
:101AE900AD740208A011012000000000889A0408C2
:101AF90001000000000000000000000000000000DC
:101B0900000000000D0000000000000000000000BF
:101B19000000000024A104080000000000000000EB
:101B2900000000000000000034A104080A000000C1
:101B390000000000B8700408000000003CA104087F
:101B49000A000000000000003870040800000000CE
:101B590044A104080A0000000000000032460120E8
:101B6900000000004CA104080A0000000000000069
:101B7900E811012000000000889A04080100000013
:101B8900000000000000000000000000000000004C
:101B99000D0000000000000000000000000000002F
:101BA90054A104080000000000000000000000002B
:101BB9000000000068A1040803000000AD740208D9
:101BC900281201200000000074A10408030000008D
:101BD900AD740208AC000120000000007CA10408DB
:101BE90003000000AD74020810120120000000007B
:101BF90084A1040803000000AD740208F811012053
:101C090000000000889A040801000000000000009C
:101C19000000000000000000000000000D000000AE
:101C290000000000000000000000000090A104086E
:101C3900000000000000000000000000000000009B
:101C49009CA1040807000000A9730208D81201200A
:101C59000000000074A7040803000000AD74020826
:101C6900C012012000000000A8A104080300000020
:101C7900AD740208A812012000000000B0A10408F8
:101C890003000000AD74020890120120000000005A
:101C9900B8A10408070000008D730208881201200A
:101CA90000000000A09B040803000000AD740208B6
:101CB9007012012000000000C4A104080300000004
:101CC900AD7402085812012000000000D0A10408D8
:101CD90003000000AD74020840120120000000005A
:101CE900889A0408010000000000000000000000BC
:101CF90000000000000000000D00000000000000CE
:101D09000000000000000000DCA104080E00000033
:101D1900116E0208D96D020800000000E0120120CE
:101D2900E4A104080E000000617002080000000030
:101D39000000000094130120F0A104080E00000027
:101D49000000000000000000000000002014012035
:101D590000A204080E00000039700208C5730208C9
:101D690000000000AC14012008A2040800000000D3
:101D790000000000000000000000000014A2040898
:101D890003000000AD740208D01501200000000016
:101D9900F4A1040803000000AD740208B81501207D
:101DA900000000001CA2040803000000AD74020832
:101DB900A01501200000000028A20408030000006B
:101DC900AD740208881501200000000030A2040843
:101DD90002000000CD7602080000000000000000AB
:101DE90038A2040802000000CD76020801000000B4
:101DF9000000000044A2040802000000CD76020899
:101E09000200000000000000000000000D000000BA
:101E19000000000000000000000000000000803FFA
:101E29000100000000620408050804000000000029
:101E39002C5C0408C85B0408EC610408000000007D
:101E49002C62040805080A00000000002C5C040844
:101E5900C85B04088C5D04080000000000E6DF0C84
:101E6900006002401060024000000000000B00000A
:101E79000000200000000000000000000060024097
:101E89002860024000000000060C0000000020004D
:101E990000000000000000000060024040600240B5
:101EA90000000000100D00000000200000000000EC
:101EB900000000000060024058600240000000007D
:101EC900160E0000000020000000000000000000C5
:101ED900006002407060024000000000200F000016
:101EE9000000200000000000000000000060024027
:101EF9008860024000000000261000000000200059
:101F0900000000000000000000600240A0600240E4
:101F19000000000030110000000020000000000057
:101F29000000000000600240B860024000000000AC
:101F3900362F000000002000000000000000000013
:101F490000640240106402400000000000380000F4
:101F59000000400000000000000000000064024092
:101F6900286402400000000006390000000040001B
:101F790000000000000000000064024040640240CC
:101F890000000000103A00000000400000000000BE
:101F99000000000000640240586402400000000094
:101FA900163B000000004000000000000000000097
:101FB900006402407064024000000000203C000000
:101FC9000000400000000000000000000064024022
:101FD9008864024000000000264400000000400020
:101FE900000000000000000000640240A0640240FC
:101FF9000000000030450000000040000000000023
:102009000000000000640240B864024000000000C3
:1020190036460000000040000000000000000000FB
:1020290001BB0308F5BA0308015E020899BB03085E
:10203900015D0208ED5D0208D95D020891490208B7
:10204900D1480208E153020800000000594602087D
:10205900B5460208814602080000000000000000A1
:1020690000000000414602084D46020835460208B4
:1020790029460208155503088D53030841530308DF
:102089003153030800FFFF0000000000AA550501B5
:102099000000AA5507010000AA5503009FAA550B85
:1020A900010000AA5509020000000000010000001B
:1020B900C012010100C20100000008000000010176
:1020C900FFFF000024900408000000000000000049
:1020D9000DB90208A08601000400000000000000FC
:1020E90000000000000000000000000000000000E7
:1020F900000000000000000074A70408788F04089D
:1021090000000000ED5C01087D00000006000000F1
:1021190000000000000000000000000000000000B6
:1021290000000000000000000000000088A504086D
:10213900000000000000000059D50308E803000072
:102149000300000000000000000000000000000083
:102159000000000000000000000000000000000076
:1021690090A504080000000000000000A5E5010892
:10217900102700000300000000000000000000001C
:102189000000000000000000000000000000000046
:1021990000000000109E040800000000AD7A03084A
:1021A900D93D0108204E0000050000000000000094
:1021B9000000000000000000000000000000000016
:1021C90000000000000000009891040800000000D1
:1021D90000000000F1CF03081027000001000000F3
:1021E90000000000000000000000000000000000E6
:1021F9000000000000000000000000009CA5040889
:10220900000000000000000075C70008E803000096
:1022190005000000000000000000000000000000B0
:1022290000000000000000000000000000000000A5
:10223900A8A50408000000000000000031BB020846
:10224900204E000003000000000000000000000014
:102259000000000000000000000000000000000075
:1022690000000000B8A504080000000000000000FC
:102279003DB90208204E00000300000000000000E4
:102289000000000000000000000000000000000045
:102299000000000000000000C8A5040800000000BC
:1022A9000000000079CD0308400D03000300000081
:1022B9000000000000000000000000000000000015
:1022C900000000000000000000000000D890040891
:1022D900000000000000000081F50208102700003E
:1022E90001000000000000000000000000000000E4
:1022F90000000000000000000000000000000000D5
:10230900948F040800000000000000002D960208C8
:10231900102700000300000000000000000000007A
:1023290000000000000000000000000000000000A4
:1023390000000000D8A5040800000000000000000B
:102349005D3C0108A08601000100000000000000BA
:102359000000000000000000000000000000000074
:102369000000000000000000848F04080000000045
:1023790000000000813B010850C30000010000007B
:102389000000000000000000000000000000000044
:10239900000000000000000000000000E09D0408AB
:1023A9000000000000000000F1360108A8610000EB
:1023B9000100000000000000000000000000000013
:1023C9000000000000000000000000000000000004
:1023D900E0A504080000000000000000E1A00208D8
:1023E900A0860100010000000000000000000000BC
:1023F90000000000000000000000000000000000D4
:1024090000000000A0910408000000000000000086
:102419006DEF0008A00F000001000000000000009F
:1024290000000000000000000000000000000000A3
:102439000000000000000000ECA5040800000000F6
:1024490000000000C968030810270000010000000F
:102459000000000000000000000000000000000073
:1024690000000000000000000000000004920408C1
:102479000000000000000000DDA202081027000093
:102489000100000000000000000000000000000042
:102499000000000000000000000000000000000033
:1024A9006C8F040800000000000000001D7802087D
:1024B9001A410000010000000000000000000000B7
:1024C9000000000000000000000000000000000003
:1024D90000000000F8A5040800000000000000004A
:1024E90089E30208400D030000000000000000001D
:1024F90000000000000000000000000000000000D3
:10250900000000000000000000A604080000000010
:102519000000000045E30208400D03000000000030
:1025290000000000000000000000000000000000A2
:1025390000000000000000000000000008A60408D8
:10254900000000000000000039BD0208A08601005B
:10255900030000000000000000000000000000006F
:102569000000000000000000000000000000000062
:1025790001010000303030302D30312D30315430F0
:10258900303A30303A3030000403090412010002B5
:1025990002000040830440570002010203010000C9
:1025A9000000000100000000000000000000000021
:1025B90043000000000000000000000000000000CF
:1025C9000000000000000000000000000000000002
:1025D90043000000000000000000000000000000AF
:1025E90000000000000000000000000000000000E2
:1025F900430000000000000000000000000000008F
:1026090000000000000000000000000000000000C1
:10261900430000000000000000000000000000006E
:1026290000000000000000000000000000000000A1
:10263900430000000000000000000000000000004E
:102649000000000000000000000000000000000081
:10265900430000000000000000000000000000002E
:102669000000000000000000000000000000000061
:10267900430000000000000000000000000000000E
:102689000000000000000000000000000000000041
:102699004D1404088D1204080000000007AB04085B
:1026A900BC9C040823A5040823A5040823A5040841
:1026B90023A5040823A5040823A5040823A50408C1
:1026C90023A5040823A50408FFFFFFFFFFFFFFFF61
:1026D900FFFFFFFFFFFF000001004153434949008D
:1026E90000000000000000000000000000000000E1
:1026F9000000000000000000000041534349490068
:1027090000000000000000000000000000000000C0
:10271900000000000000000000000000A01F0120D0
:1027290000000000000000000000000000000000A0
:102739000000000000000000000000000000000090
:102749000000000000000000000000000000000080
:102759000000000000000000000000000000000070
:102769000000000000000000000000000000000060
:102779000000000000000000000000000000000050
:04278900010000004B
:10800000002830B41FDB0928044622DD012303EBDE
:1080100083035B00B0FBF3F2092AF8D87BB10F4D64
:10802000A5FB0320B4FBF3F2092A03FB1244CCBFE7
:1080300057233023134401F8013BC308F0D1002338
:1080400030BC0B7070472D234042013101F8013CD8
:10805000D9E7303001F8010BF1E700BFCDCCCCCC33
:10806000884230B44FF001042ED301FB04F4B0FB7E
:10807000F4F58D42F9D284B1AAB901E0B0FBF4F570
:10808000092D04FB1500CCBF57223022B4FBF1F4BC
:10809000154403F8015B002CF0D1002230BC1A70AB
:1080A0007047B0FBF4F5092D04FB1500CCBF372257
:1080B0003022B4FBF1F4154403F8015B002CF0D13D
:1080C000002230BC1A7070470546002AEBD1D7E772
:1080D00003685A1C02601970704700BF2DE9F04711
:1080E000089C002B8846074621780CBF4FF02009DA
:1080F0004FF03009651C39B3002A2ADD2B4601E018
:108100000246A8B113F8016B501E002EF8D1961E3E
:1081100070B1B2460AF1FF3A49463846C0470AF103
:108120000103002BF6DC26EAE6702178013049B124
:10813000041B3846C047281915F8011B0029F8D13F
:10814000BDE8F087BDE8F087002A04DC0846BDE8FA
:10815000F0870020ECE7561EDBE700BF8368D0ED18
:10816000037A416800EB8302013370EE277A82EDD7
:10817000040A8B428360C0ED037A1ED000EB8303B8
:10818000026893ED047A914277EEC77AC0ED037AE4
:108190000CDA0132B7EE007A06EE902A0260F8EEB1
:1081A000E66A87EEA60A30EE070A704707EE101A55
:1081B000B8EEC77A87EE870A7047002213468260BE
:1081C000DCE700BFD0ED007AB0EE406AD0ED056A82
:1081D000D0ED015AE7EE806A90ED067AD0ED047A90
:1081E000A0EE257A90ED035AD0ED025A67EEE67ABA
:1081F000B0EE660AA6EEC57AE6EE257A80ED057A3F
:10820000C0ED067A704700BF90ED057AF0EE406A47
:10821000D0ED017A90ED006A27EE270AD0ED064AEC
:1082200090ED024AD0ED077AA6EE260A90ED035AA9
:1082300090ED086AD0ED045AC0ED056A80ED067A2B
:10824000C0ED087AA4EE240AA5EE670AA5EEC60AD8
:1082500080ED070A704700BFD0ED007A90ED017AFB
:1082600030EE670AE7EE007AB0EE670AC0ED007AFA
:10827000704700BF704700BF0A4491421AD00139CD
:1082800030B4551E41F2210411F8012F082380EA71
:10829000022002E0013B90B209D010F4004F4FEAF7
:1082A0004002F7D084EA4000013B80B2F5D18D4214
:1082B000EAD130BC704700BF2DE9F04F824F8FB03C
:1082C000824C0025B7F80AC04FF0000826684FF02E
:1082D00000093C894FEA0C224FEA1C630B908C4644
:1082E000B7F80CA04FF0000ECDE90445FC8800253E
:1082F000CDE9064535460026069CA81ACDE9008939
:10830000CDE9028966EB03018046AAFB002389467A
:10831000A4FB0845D60D0AFB0133CB460499009611
:10832000A1FB0001049ECDE908452C46069D06FBF5
:10833000091105FB0B440994009C44EA4324DB1516
:108340000094C40901930294B888029BDDE900AB54
:1083500043EA41631AF5FA6A4FEAE11102934BF1DD
:10836000000B03910104CDE904ABDDE908ABCDE9D5
:108370000C8956468846320A060C788842EA0B6217
:10838000B1465E46C4033312450CDDE9026716EBC5
:10839000080647EB090712EB040ADDE9048943EB01
:1083A000050BB8F5FA6F79F100023CDA0199009DEE
:1083B0008C00AA0044EA9573DDE90045A4185D41EC
:1083C0002246019C2B46009D02FB04F405FB03445E
:1083D000A2FB0523234490085D104FEA320440EAD3
:1083E000837099104FF0FF32361B67EB0507BAEB2D
:1083F000000A6BEB010B3649884579EB020332DB4F
:10840000DDE90C8908FB09F4A8FB082303EB44030E
:10841000D00FD91740EA4300DDE904341B1A64EB9E
:108420000104CDE90434294B5968A1FB0A2301FB5F
:108430000B334FEA52580B9A48EAC3284FEA635964
:10844000B8EB060869EB07094FEAD83343EA49431A
:1084500002B11360BCF1000F02D0049BCCF80030D5
:108460000FB0BDE8F08F40F6AC540025DDE90023E5
:1084700012196B41A2FB024502FB03F3221905EB23
:1084800043054FEAC50145EB0503121941EA547152
:108490006B418946E10098008846910040EA92705D
:1084A000B4EB080865EB090916EB080647EB09076A
:1084B0000A1B60EB05035B104FEA3202BAEB020ABB
:1084C0006BEB030B9CE700BF6C40012004200120F4
:1084D00024FAFFFF2DE9F04F8B4B89B08B4DD3F879
:1084E00008E02A880691C2EB2E11B5F9043052003B
:1084F000059001FB01F1B5F90200C2EBEE02B5F9FE
:108500000A60091300FB02F2F71703FB01F18B135A
:1085100003EBE222B2F5FA304FEAE27102EB820C91
:10852000AA6141F1FF31A0FB00AB0CF1800CB5F961
:10853000082000FB01FE4FEA2C230BEB4E0B02FB45
:1085400001FE0793D31706FB0BFC00FB03EE0AFBAF
:1085500007CCA6FB0A67A2FB00236744340A7344D6
:108560004FEA023844EA07644FEA0339EB88009483
:108570003C1249EA125901940024DDE90067CDE973
:10858000023416EB0806029C47EB0907003647F554
:108590000047A6FB048904FB07994FEA69024FEAEA
:1085A000E97352EA030400F0A380B5F90E60564C5B
:1085B000F71706FB01F1A6FB0089B5F9106000FB77
:1085C0000710E46806FB0BFEF7178144C4F580141E
:1085D0000AFB07EE4FEA4941A6FB0A67B5F90CA072
:1085E0004FEAE47941EAD8317744E00701914FEA54
:1085F000484100914FEACA01DDE900AB03914FEA1F
:10860000C9711AEB060A4FF0000641EA54010296BE
:108610004BEB070BDDE9026716EB0A0647EB0B078E
:10862000801B61EB070110EB000A41EB010B1AEB19
:10863000000A4BEB010B4FEA8A184FEA8B1918EB33
:108640000A0849EA9A694FEA880649EB0B094FEA9A
:10865000890444EA987416EB000844EB01094FEAD8
:1086600088064FEA8904801944EA9874614138F019
:108670001FF9B5F91680B5F912404F13460BB5F93D
:10868000142008FB07FC4FEAE87946EAC14602FBE2
:1086900001FEE517D31706FB09CCCDE90045A8FB81
:1086A000064500FB03EE04FB07F76544A2FB00232D
:1086B000734406FB057EA4FB0645D60CDF14754407
:1086C0004FEA546A46EA43364AEAC51A4FEA656BEE
:1086D00010EB0A0041EB0B018019DDE900AB794199
:1086E0004FEA1028544648EA0168220112EB0802BA
:1086F000059909B1120A0A60069B0BB1079A1A6024
:1087000009B0BDE8F08F00BF0420012080400120A7
:10871000704700BF704700BF4FF40063038370478A
:108720004FF4006303837047012250F8043CA0F12A
:10873000100180F849200BB108461847704700BF68
:10874000D0F8F020034630B46AB1C168D0F80821EF
:108750004469881A013A205C08BF0A46C0B2C3F8CF
:10876000082130BC7047006A5D69411CDC68285CE8
:10877000A14228BF1146C0B2196230BC704700BF89
:10878000D0F8F43013B190F888017047836A406ADA
:10879000181AB0FA80F04009704700BF416A836A36
:1087A00099420ED3CB1AD0F8F410026981B1D0F8F7
:1087B0007411501E0A685268134483420BD2C01AC7
:1087C000704702691144CB1AD0F8F4100029EED199
:1087D000501EC01A70470020704700BFD0F8F0301C
:1087E0006BB1D0F87831D0F808211B685B689342F0
:1087F00001D3981A7047C068801A18447047C2693C
:10880000036A9A4203D2C0681044C01A7047D01A53
:10881000704700BFBFF34F8F0549064BCA6802F48B
:10882000E0621343CB60BFF34F8F00BFFDE700BF93
:1088300000ED00E00400FA05704700BF70B582B09B
:108840000446056E06236A4643211430A847C0B18A
:108850009DF8003001209DF801109DF8026041EA6A
:1088600003219DF803209DF804509DF8053042EA4D
:108870000622A4F8401043EA0523A4F84220A4F8F5
:10888000443002B070BD00BF70B582B00446856A46
:1088900006236A463B210830A847A8B19DF800305E
:1088A00001209DF801109DF8026041EA03219DF826
:1088B00003209DF804509DF8053042EA06226183AA
:1088C00043EA0523A283E38302B070BD2DE9F041A2
:1088D0000F46016886B00646C1F30D04002C48D14E
:1088E0001022214602A83AF02CFF384B38480122CA
:1088F00002218342049205911ED900F580408342F3
:1089000025D9344A934218D902F58042934220D99E
:1089100002F5803293421ED902F5003293421CD9EF
:1089200002F5003293421AD902F50032934218D967
:10893000052005F0A9F9FBE72146274B03911B7D94
:10894000012B10D14FF0FF3006B0BDE8F081114689
:10895000F3E70321F1E70421EFE70521EDE7062125
:10896000EBE70721E9E701A902A832F067FB00283D
:10897000E8D1194D2B7D012B02D16FF00100E3E707
:108980000123D6F800802B7528F0E0FFB0B9134C16
:10899000236923F440732361236943F40073236143
:1089A000236943F001032361C8F80070BFF34F8FC0
:1089B00028F0CCFF236923F00103236100232B75EA
:1089C0000028DAD1336804333360BDE70040000883
:1089D000FF3F0008FFBF000838770120003C02403D
:1089E000F8B504460D468E180027B54201D120691E
:1089F000F8BDE368591C2344E160042915F8012BF4
:108A00001A72F2D1206918B9A1682046FFF75EFFFB
:108A10002061E760E9E700BF014B186805F0F6BE8A
:108A2000E8BC012008B505F047FD044B5B68C01A9F
:108A3000C0F5FA5020EAE07008BD00BF44C701202D
:108A400000B5002183B00A2036F09AFD0F210A20DC
:108A500036F096FD01AA0321102036F0BDFD9DF9E8
:108A60000430F7EE007A9FED265A06EE103A9DF993
:108A70000530DFED245A002106EE903A9DF90630CC
:108A8000B8EEC66A0A2007EE103AF8EEE66A1E4B08
:108A9000B8EEC77A76EEC56A36EE456A37EE457AA5
:108AA000B0EE675AA6EE255AB0EE456AB0EE675AA8
:108AB000E7EE257AA6EEA55AF3EE0E5A26EE256AC3
:108AC00067EEA57A25EE257A83ED006AC3ED027A7A
:108AD00083ED017A36F054FD0DF1030201210220ED
:108AE00036F07AFD0DF103020121092036F074FD04
:108AF00001210A2036F044FD012003B05DF804FB9B
:108B0000000000430000803B0000012000B583B05E
:108B1000002002AB03F8012D0A46682124F05AFB1D
:108B200003B05DF804FB00BF38B5044690F85D0063
:108B300000285AD104F11405636E80226B21284667
:108B40009847642005F060FD636E0722682128467F
:108B50009847642005F058FD636E00226B2128467B
:108B60009847642005F050FD636E01226B21284672
:108B700098470F2005F048FD94F85720636E1B219D
:108B8000032A28468CBF1A22182298470F2005F086
:108B90003BFD636E18221C21284698470F2005F0E4
:108BA00033FD636E94F856201A21284698470F200B
:108BB00005F02AFD636E94F858201921284698473D
:108BC000642005F021FD636E102237212846984766
:108BD0000F2005F019FD2846636E012238219847C1
:108BE0000F20BDE8384005F00FBD05F0EBFE05464F
:108BF00006F032F800289DD115B12023E871AB7141
:108C0000034B2146284641F8103F25F03FF891E7F5
:108C100029870008F8B590F87D3190F87E2113433C
:108C200003F02103212B0FD0436A846AA3420CD89E
:108C300002690023121B92B290F87D110025836215
:108C4000202980F8885103D0F8BD1A1B92B2F3E7AF
:108C50008369E34203EB0401F6D0B2FA82F46409BB
:108C6000002CF1D190F87C31012BEDD00546012785
:108C7000A0F866211346A0F864214FF0210ED0F829
:108C80007461C0F86011C0F88041304685F87C718D
:108C90000C4A0D4F85F87DE1F76332640B4FD5F830
:108CA000142134652832F76432F0A8F8D5F814316D
:108CB00040221A6285F87C419A6842F080029A60EC
:108CC000C2E700BF414702087D470208D9460208B3
:108CD000426A10B48469A154426A04690132D0F82E
:108CE000F410A24228BF0022426241B10B68DB07A8
:108CF00002D55DF8044B70475DF8044B8AE7D0F865
:108D000014215DF8044B136843F08003136070472F
:108D1000406990301CF006BFF8B5D0F81431044615
:108D2000DA69910614D5586AE36AC0B2002B00F0E4
:108D3000A1809847D4F814311A6822F480721A601E
:108D40009A6822F001029A609A6942F008029A61D8
:108D5000DA69D20701D501221A62DA69970701D5CB
:108D600002221A62DA69560701D504221A62DA6908
:108D7000150701D508221A62D4F8F420002A00F061
:108D80008580D969490600D4F8BDD96904F58A708F
:108D90001E680F079D6818D18F0602D5B50600F131
:108DA000F0800F0602D5350600F1CD80480602D5C9
:108DB000710600F1A780002AE6D0626AA36A9A428F
:108DC0007DD1012384F88831F8BD15F001057AD1F1
:108DD00016F4907FE5D011F0010700F0D08016F472
:108DE000807774D13D4605EA91073FB104271F62A1
:108DF000D4F8807147F00207C4F880710F070AD5D4
:108E0000B70640F18E8008251D62D4F8805145F0E8
:108E10000805C4F88051D4F88051002DCBD08F06BE
:108E200005D5B50603D51CF01FFDD4F81431D4F8D0
:108E3000802111076ED51A68202122F490721A60E1
:108E40009A6822F001029A6084F87E119A685206AC
:108E50000DD59A68D4F8781122F040029A6031B1A9
:108E6000564B08460B6531F005FE00285DD1D4F85D
:108E7000F420A0E7E3696269D054E369E168013353
:108E8000B3FBF1F201FB1233E36153E7D969080642
:108E90007FF577AF94F87D1121293FF472AFA16A75
:108EA000606A814248D0A069405C0131C0B29862DA
:108EB0002569B1FBF5F005FB1011A16261E72046C1
:108EC000BDE8F840A6E6CF0709D5F70507D5012785
:108ED0001F62D4F8807147F00107C4F88071EDB2C9
:108EE00015EA51073FF47FAF4FF0020E3D46C1F344
:108EF0008007C3F820E0D4F880E14EF0040EC4F8F7
:108F000080E172E71968202021F04001196084F89F
:108F10007D0150E79A6812F040028CD1C4F880219C
:108F2000A5E7002D3FF477AF6DE7D4F87801036D26
:108F30009847D4F8F4203EE7A4F86621196821F098
:108F4000800119601DE794F87D1121297FF433AF6A
:108F5000B4F8661189B2C9B1D4F81C11B1F5805FBB
:108F60001DD0D4F86011481CC4F8600109789962DA
:108F7000B4F86631013B9BB2A4F866311BE73D466D
:108F80003CE71CF071FCD4F8F42014E7196821F0D8
:108F900080011960196841F0400119600BE7D4F8AD
:108FA00024110029DDD1D4F8601131F8020BC0F38F
:108FB00008009862C4F86011DAE700BFC9460208E9
:108FC0002DE9F0470569C3681D4028D00F460646C5
:108FD0004FF000484FF00009B5FA85F328FA03F284
:108FE0001B3BD24332611540042B16D8DFE803F057
:108FF0003129211903007B6A002B32D003F1FF3A9B
:10900000C7F824901FFA8AFA3C6A34B123682046D4
:10901000514698476468002CF8D1002DDCD1BDE89A
:10902000F0873868716B036889B29847002DD3D1F7
:10903000F5E77868B16B036889B29847002DCBD10A
:10904000EDE7B868F16B036889B29847002DC3D18A
:10905000E5E7F868316C036889B29847002DBBD109
:10906000DDE7F36A1FFA83FACEE700BF4269C2EB7D
:10907000421270B5D4000D4D2E19738903EB4203D3
:109080001E3355F823001CF04DFD736804F15800A1
:10909000DA7959792844530703D4BDE8704032F097
:1090A000EDBBBDE8704032F00BB900BF7C7701200A
:1090B000436910B508330D4C54F823001CF032FD01
:1090C0000B4B1B7843B90B4B2046198832F0D6FB6B
:1090D000094B00221A7010BD064B2046198832F049
:1090E000EFF8054B00221A7010BD00BFAC3801200C
:1090F000A9380120EC3801207BB5012070B54488E7
:109100000D4606460021C4F30B04284622463AF0D9
:1091100018FB3369094A934209D3094A934206D29C
:10912000224628461946BDE8704038F0C1B823B140
:1091300021462846BDE87040184770BD84060008E7
:1091400089070008064B07498B4202D300231846C3
:1091500070471A88C2F30B029042F8D01433F3E739
:10916000E801000884060008024A136823EA0000A8
:109170001060704768460120F8B5174D2B78A32B77
:1091800028D16B78BE2B25D1AC1C144F0222294666
:109190004FF6FF70FFF770F822884AB1A618BE425A
:1091A00018D2052A16D921463446FFF765F8F3E7A9
:1091B00021460222FFF760F80222A1180634FFF7C9
:1091C0005BF8074B641B1C8041F60F53C31A5842CF
:1091D0005841F8BD0020F8BD00400008008000089C
:1091E000442A01202DE9F04FDFF850918BB04E4F0B
:1091F0000326A7EB09071822002104A83AF0A1FAD8
:109200004A4BCDF8109005971A69002A04DA484AAB
:109210005A6002F188325A6001230222694604A88A
:109220008DF824304FF0000B424B434C1B88DFF885
:1092300010A1ADF80030FFF7D3FB022269464FF6CC
:10924000FF70FFF719F88046544539D30AAC002562
:10925000022204A824F8245D2146FFF7C1FB022264
:1092600021464046FFF708F840BA022202A9C0434F
:10927000ADF8080004A8FFF7B3FB079878B106AB78
:10928000C0F10402294618443AF05BFA089818B96C
:10929000069904A8FFF71AFB0023089007939DF88E
:1092A0002430089A23B121490B6943F000430B6134
:1092B000013E30D0002A9ED1FFF75EFF68B32FE059
:1092C000658802A904A88DF80DB0C5F30B05143408
:1092D000AB1DADF8083034F8143CC3F30B021B0B84
:1092E000ADF80A2006228DF80C30FFF779FB062234
:1092F00002A94046FEF7C0FF804654F8101C2A46DB
:1093000004A8FFF76DFB54F8101C40462A46FEF7F0
:10931000B3FF804698E7002ACED0052004F0B4FCC5
:109320000BB0BDE8F08F00BF00800008003C024099
:1093300023016745443A0408E8010008004000089A
:10934000840600080378092B01D0202B05D110F8E2
:10935000013F202BFBD0092BF9D02D2B00F0898069
:109360002B2B00F08B80B7EE000AA3F13002D1B2B4
:10937000092900F29080F2EE046ADFED4A7A07EEE6
:10938000102A10F8013FB8EEC77AA3F13002D1B22B
:10939000A7EEA67A0929F0EE477AF0D92E2B4BD00A
:1093A00003F0DF03452B39D110B442782D2A6AD05F
:1093B0002B2A6CD0411C0024A2F13003092B6DD85C
:1093C000002303EB830302EB430311F8012FA2F107
:1093D0003000303B0928F4D9B3F59A7FB7EE007A14
:1093E00028BF4FF49A73072B09D91A46DFED2E6A6E
:1093F000083A27EE267A072AFAD803F007032BB19A
:10940000F2EE046A013B27EE267AFBD16CB1C7EE7F
:10941000876A5DF8044B20EE260A7047B7EE007AA3
:1094200067EE876A20EE260A704767EE876A5DF866
:10943000044B20EE260A704743780130A3F1300236
:10944000D1B20929ACD8B2EE047AF0EE475A06EE52
:10945000902A10F8013FB8EEE66AA3F13002D1B2CB
:10946000C6EE076A092927EE257A77EEA67AEED9A5
:1094700096E74378BFEE000A013076E74378B7EE0F
:10948000000A013071E7811C8278012494E7811C75
:109490008278002490E7DFED037A7FE7B7EE007A69
:1094A000B4E700BF0000000020BCBE4CB5EEC00A0F
:1094B000DFED357A0023F1EE10FA30B5C8BF30EE9B
:1094C000270A87B0D8BF30EE670ADFED307A05464D
:1094D00003A9019320EE270A00930293FDEEC07AC0
:1094E00017EE904A84EAE470A0EBE4702CF06CFA7A
:1094F000002C03A8ACBF20232D238DF8003036F0BC
:109500002DFD012829D0022833D003281DD003A91E
:1095100068463AF0F9F9684636F020FDC41E6946FF
:109520002846E4B222463AF04DFA002328462B554D
:1095300036F014FD2E22431C0DEB04012A54E818CA
:109540003AF0FFF9284607B030BD302303A968463A
:109550008DF801303AF0D8F9DDE7302303A96846E9
:109560008DF801308DF802308DF803303AF0CCF9E7
:10957000D1E7302303A968468DF801308DF8023019
:109580003AF0C2F9C7E700BF6F12033A00007A440D
:109590002DE9F041064615460846B6FBF2F43CB903
:1095A00005FB1464124B1B5D00F8013BBDE8F08124
:1095B000B4FBF2F767B90E4B05FB174705FB1464C4
:1095C000DA5D1B5D00F8012B00F8013BBDE8F0817E
:1095D000B7FBF2F8B8F1000F02D04046FFF7D8FF12
:1095E00005FB1878024B13F8082000F8012BE3E77D
:1095F000F46F0408026830B41146541CD31C151DC6
:10960000046011F8024B01605178036093780560A3
:109610001B04D07843EA0123234330BC43EA0060B3
:10962000704700BF0368591C1A46016012F8021BFC
:109630000260587841EA0020704700BF03685A1C56
:1096400002601878704700BF38B5044600681546B8
:1096500037F02EFE22682A44226038BD03680A0AC9
:1096600070B45E1C0D0E0C0C06601D7003685D1C52
:1096700005601C7003685C1C04601A7003685A1C47
:109680000260197070BC704703680A0A10B45C1C51
:1096900004601A7003685A1C026019705DF8044B6C
:1096A000704700BF03680A0E70B45E1C0D0A0C0CF4
:1096B000066019700368591C01601D700368591C0D
:1096C00001601C700368591C01601A7070BC7047FF
:1096D00003680A0A10B45C1C046019700368591C02
:1096E00001601A705DF8044B704700BF2DE9F04728
:1096F000002488B080460F461E46A14605AD531C87
:109700000393117841B3252935D1931CCDF81090DE
:1097100003935378302B52D04FF0000AA3F130025C
:10972000D2B2092A44D96C2B1AD0642B00F09C8049
:1097300026D8252B1ED06BD9582B7ED0632B1DD15C
:10974000331D3178404601341E46B847039A531CF6
:10975000039311780029D6D1204608B0BDE8F087E0
:10976000039B5A1C03921B78642B00F084802CD836
:10977000252B5AD1252140460134B847039ABEE72C
:10978000732B37D04AD9752B55D106F1040E3068AA
:109790002B4600220A217646FEF762FC049A5346C5
:1097A000009539464046FEF799FC039A0444A6E723
:1097B000184604AA03A92CF0E3F80346B3E7D31C28
:1097C0004FF0010A03939378A8E7732B12D060D966
:1097D000752B3FD0782B92D1A3F1580206F1040EDD
:1097E00030682B46B2FA82F2102176465209FEF713
:1097F00037FCD3E7306806F1040E049A002300908A
:10980000394640467646FEF769FC039A044476E7FB
:10981000002BB3D1204608B0BDE8F0876E2BADD148
:10982000039A336804361C6069E72BD9582BD3D0D0
:10983000632B85D063E7782BA0D1A3F15802311DAB
:1098400030682B46B2FA82F20E4610215209FEF71A
:1098500007FCA3E706F1040E30682B4600220A211C
:109860007646FEF7FDFB99E7331D306829461E4614
:10987000FEF7C6FB92E7331D306829461E46FEF709
:10988000BFFB8BE7002B7FF43AAF204608B0BDE862
:10989000F0876E2BC5D032E70EB410B585B00949FC
:1098A00007AC019001A854F8042B23460394FFF75A
:1098B0001DFF019B00221A7005B0BDE8104003B0E7
:1098C000704700BFD18000080FB430B583B00C4B97
:1098D0000C4806AC1968006854F8042B2346019420
:1098E000FFF704FF084C0546206804F07BFF0028C2
:1098F000FAD0284603B0BDE8304004B0704700BF3E
:10990000A0610120A4610120E8BC0120DFED2A7ADA
:10991000B4EEE70AF1EE10FA4BDDDFED286A9FEDB9
:10992000287AB4EEC70A70EE667AF1EE10FAB0EE5D
:10993000670AF6DC9FED237AF4EEC77AF1EE10FAAF
:1099400034D5DFED1E6A9FED207AF4EEC77A37EE4C
:10995000A60AF1EE10FAF0EE407AF6D4DFED1B7AAB
:10996000B4EEE70AF1EE10FA14DDDFED137A37EE0C
:10997000C00A60EE006A9FED166A9FED167ADFED71
:10998000167AA6EE867A20EE266AE6EE877AA6EEAC
:10999000270A7047DFED117AB4EEE70AF1EE10FA0C
:1099A000E7D5DFED087A37EEC00AE2E7B0EE670AE6
:1099B000D4E7F0EE407ABDE7DB0F4940DB0FC9404A
:1099C000E4CB1641DB0F49C0E4CB16C1DB0FC93F26
:1099D00092E741B99730083C15A82ABEDB0FC9BFF2
:1099E00080EAE073A3EBE0738B4205DB002801DD26
:1099F000401A704702D170470020704708447047F2
:109A000009B909E0194690FBF1F301FB130308467D
:109A1000002BF7D1084670470146FBE7B0EEC07A4D
:109A2000F0EEE06A86FE876AB5EE406AF1EE10FA63
:109A300039D0C6FEC75AC5EE867ADFED1F2ADFEDA4
:109A40001F3ADFED1F4A9FED1F5A9FED1F3AB7EEF9
:109A5000006A9FED1E4ADFED1E5AE7EEE23AA7EEDE
:109A6000834AE7EEA34AA7EE846AA7EEA45AE7EE7C
:109A7000855AC5EE867AF4EEC76AF1EE10FA03D580
:109A80009FED147A77EE677AF5EEC00AF1EE10FAE0
:109A90000CD4B5EEC00AF1EE10FA48BFF1EE677AC9
:109AA000B0EE670A7047DFED0A7AE4E79FED0A7AC5
:109AB00077EE677AEDE700BF39094E3DE3B59E3E8C
:109AC00088FA163E45FE7F3F99FB243F69A2163E69
:109AD000A7DFA834DB0FC93FDB0F4940DFED307A49
:109AE00030EE277AFDEEC76A16EE903A2033402B0F
:109AF00002D99FED2C0A7047B4EEE70AF1EE10FA96
:109B00004BDD9FED296ADFED296AB4EEE67A77EE48
:109B1000467AF1EE10FAB0EE677AF6DC9FED247A21
:109B2000F4EEC77AF1EE10FA34D5DFED1F6A9FED3F
:109B3000217AF4EEC77A37EEA60AF1EE10FAF0EECB
:109B4000407AF6D4DFED167AB4EEE70AF1EE10FAB9
:109B50001BDCDFED197AB4EEE70AF1EE10FA03D55B
:109B6000DFED137A37EEC00A60EE006A9FED136AEC
:109B70009FED137ADFED137AA6EE867A20EE266A41
:109B8000E6EE877AA6EE270A7047DFED0F7A37EE0A
:109B9000C00AE9E7B0EE670AD4E7F0EE477ABDE71E
:109BA000DB0FC93F00000000DB0FC940E4CB1641CA
:109BB000DB0F49C0E4CB16C1DB0FC9BF92E741B947
:109BC0009730083C15A82ABEDB0F4940FDEEC07A4D
:109BD00017EE903A2033402B4FD8DFED2C7AB4EEBD
:109BE000E70AF1EE10FA4BDDDFED296A9FED297AE5
:109BF000B4EEC70A70EE667AF1EE10FAB0EE670ABC
:109C0000F6DC9FED257AF4EEC77AF1EE10FA3AD53C
:109C1000DFED1F6A9FED217AF4EEC77A37EEA60AD0
:109C2000F1EE10FAF0EE407AF6D4DFED1D7AB4EEE4
:109C3000E70AF1EE10FA14DDDFED147A37EEC00A10
:109C400060EE006A9FED176A9FED177ADFED177AD5
:109C5000A6EE867A20EE266AE6EE877AA6EE270A38
:109C60007047DFED137AB4EEE70AF1EE10FAE7D5AC
:109C7000DFED097A37EEC00AE2E79FED0E0A704782
:109C8000F0EE407ABDE7B0EE670ACEE7DB0F494061
:109C9000DB0FC940E4CB1641DB0F49C0E4CB16C152
:109CA000DB0FC93F92E741B99730083C15A82ABE9F
:109CB000DB0FC9BF0000000007EE901A10B52DEDB4
:109CC000028BB8EE678ADFED217A044628EE008A1F
:109CD00028EE278AB0EE480A37F064FCF0EE408A9E
:109CE000B0EE480A37F0C0FBB7EE006A9FED187A75
:109CF000F8EE006AF6EE007A0023B0EE465AF0EE77
:109D0000465AA3616361A8EE875A2362E8EEC75AF8
:109D1000E36136EE407A20EE260A67EE277AC6EE39
:109D2000056ABDEC028B67EEA67A25EEA66A27EEE1
:109D3000267A20EE260AC4ED007A84ED046A84EDCA
:109D4000017AC4ED027A84ED030A10BD27D4D2361D
:109D5000F304353F10B401224C0901F01F0150F803
:109D6000243002FA01F10B4340F824305DF8044B33
:109D7000704700BF01234A0901F01F0150F822205B
:109D800003FA01F1114214BF18460020704700BFCA
:109D90003F4BF0B51B78012B73D03E4B1B78012B4A
:109DA00069D03D4C02253D4800212368012244260C
:109DB0003B4F43F4806305723A4D23603A4B417246
:109DC00079712E825A719A71384B35202D213422A7
:109DD00003F1EA064025122418704E3303F84D1C97
:109DE00003F84C2C03F84B0C03F84A1C03F8492CDD
:109DF00003F8485C03F8464CB342EDD12C4D2D4C92
:109E000005F1100E05F1200704F1100695E80F008A
:109E100084E80F009EE80F0005F1300E86E80F0081
:109E200097E80F0004F1200605F1400786E80F00CF
:109E300004F130069EE80F0005F1500E86E80F0091
:109E400097E80F0004F1400605F16007703586E8D9
:109E50000F0004F150069EE80F0086E80F0004F1A1
:109E60006006703497E80F0086E80F0095E80F0051
:109E700084E80F00F0BD094A052113721375D174EF
:109E8000A2E70D494FF4FA400C4A0880137084E7AA
:109E90008828012000230120684601200C7701203A
:109EA000CC4C0120CCCA0120604F0120204501206C
:109EB000483A04086CB101205477012078BC012095
:109EC00010B50D4C3D2004F07DFD206118B111222C
:109ED00000238271C371202104F042FE0A2004F0A5
:109EE00039FB206904F0B8FE0028044B14BF01229E
:109EF00002221A7010BD00BF04200120002301209F
:109F0000094B0A4A1B781078834206D9084AC3F1E4
:109F100080030344106818447047C31A044A0020A1
:109F2000034410681844704720470120A4470120CB
:109F30001C470120074A084B10781B78834205D93B
:109F4000C3F180031844C0F17F007047C01AC0F10C
:109F50007F007047A447012020470120014BD868AB
:109F6000FEF7DABEAC610120014B5868FEF7D4BEA3
:109F7000AC610120014B1868FEF7CEBEAC61012038
:109F8000F8B510F58A75044614D0D0F814212421B0
:109F9000002380F87D11116821F001011160136028
:109FA00053609360C0F8803180F87C3180F87D3157
:109FB00080F87E31A279A36812F00401C4F8183148
:109FC00000F0F8804FF48053C4F81C3112F0020303
:109FD00000F029814FF400534FF48061C4F8203120
:109FE00063790020C4F8241113F00101C4F82C0196
:109FF000C4F83401C4F8280102D00420C4F82801B0
:10A0000013F0020605D0D4F8280140F00800C4F887
:10A010002801D0070DD549B1D4F838014FF4803765
:10A0200040F00200C4F84071C4F83801002E40F03E
:10A03000E88012072AD5002D58D094F87D3103F01E
:10A04000FF02002B00F0E880D4F8142124232846D6
:10A0500084F87D31136823F0010313601BF092FA3A
:10A06000012840D0D4F83831002B40F0D880D4F803
:10A07000143128465A6822F490425A609A6822F0B5
:10A0800022029A609A6842F0080225E075B394F8BB
:10A090007D3103F0FF020BB984F87C21D4F8142140
:10A0A0002423284684F87D31136823F001031360CC
:10A0B0001BF068FA012816D0D4F8383113B12846BD
:10A0C0001BF008FAD4F8143128465A6822F490425A
:10A0D0005A609A6822F02A029A601A6842F00102D5
:10A0E0001A601BF0C1F9637903F0010100292ED039
:10A0F000D4F8F020002A75D00023D4F8F8004FF4EB
:10A10000806E4FF4803104F130074FF48076A36302
:10A11000E3636364A3646365A3652366E365226305
:10A1200060633846C4F840E02165E66430F0AAFE7A
:10A13000384630F0E3FE94F87E31C4F87871202B75
:10A14000A5667AD0226B63795268C4F808219B0710
:10A150002FD5D4F8F420002A3DD0002340204FF41E
:10A160008031C4F8902004F19006D4F8FC204FF41C
:10A170008067C4F89800C4F894203046C4F89C3036
:10A18000C4F8A430C4F8A830C4F8AC30C4F8B43073
:10A19000C4F8B830C4F8C030C4F8BC30C4F8A070FB
:10A1A000C4F8B01030F06EFE304630F0A7FE50B16B
:10A1B000FEE7F8BD12F00203C4F81C1138D1C4F850
:10A1C000203119460CE7D4F89030C4F87461C4F813
:10A1D000C8505860F8BDD4F88421136843F0800358
:10A1E0001360F8BDD4F88421116841F480711160C6
:10A1F000916841F001019160116841F02001116006
:10A20000A5E7D4F838014FF4003640F00100C4F857
:10A210003C61C4F838010CE784F87C2114E7284637
:10A220001BF058F923E7C4F820314FF48061D7E6DA
:10A230004FF40053C4F82031D2E6E368626999B262
:10A24000002A3FF47FAFB1FA81F67609002E7FF441
:10A2500079AF94F87C0101283FF474AF0B46A4F861
:10A260006C1138461449154F4FF0010C4FF0220E77
:10A270002167E766D4F81411114FC4F880612431C6
:10A28000C4F86821C4F8806084F87CC184F87EE159
:10A29000E76730F0B3FDD4F8143184F87C611A68B4
:10A2A00042F480721A609A6842F001029A609A68D9
:10A2B00042F040029A6045E74547020849470208D4
:10A2C000D946020841715BE6816059E6B0B5BB4BE7
:10A2D000B8B0BB491A6C00AFBA4842F08052BA4CD1
:10A2E0001A641A6C02F08052C7F8D820D7F8D82028
:10A2F0001A6B42F480221A631A6B02F48022C7F8A8
:10A30000D420D7F8D4200A6842F480720A60026828
:10A31000A24200F04882AD4C4FF6FF05AC4AE1681E
:10A32000AC4829400A43E2605A6F02601A6B42F45B
:10A3300080221A631A6B02F48022C7F8DC20D7F857
:10A34000DC201A6B42F480121A631A6B02F480123A
:10A35000C7F8D020D7F8D0201A6B42F480021A63D5
:10A360001A6B02F48002C7F8CC20D7F8CC201A6B05
:10A3700042F000521A631A6B02F00052C7F8C8206C
:10A38000D7F8C8201A6B42F080421A631A6B02F0A9
:10A390008042C7F8C420D7F8C4201A6B42F00102EB
:10A3A0001A631A6B02F00102C7F8C020D7F8C02068
:10A3B0001A6B42F002021A631A6B02F00202C7F82B
:10A3C000BC20D7F8BC201A6B42F004021A631A6B47
:10A3D00002F00402C7F8B820D7F8B8201A6B42F090
:10A3E00008021A631A6B02F00802C7F8B420D7F803
:10A3F000B4201A6B42F010021A631A6B02F01002BA
:10A40000C7F8B020D7F8B0201A6B42F020021A63C8
:10A410001A6B02F02002C7F8AC20D7F8AC201A6BF8
:10A4200042F040021A631A6B02F04002C7F8A820FB
:10A43000D7F8A8201A6B42F080021A631A6B02F058
:10A440008002C7F8A420D7F8A4201A6B42F48072C7
:10A450001A631A6B02F48072C7F8A020D7F8A02004
:10A460001A6C42F001021A641A6C02F00102C7F879
:10A470009C20D7F89C201A6C42F002021A641A6CD5
:10A4800002F00202C7F89820D7F898201A6C42F020
:10A4900004021A641A6C02F00402C7F89420D7F878
:10A4A00094201A6C42F008021A641A6C02F0080236
:10A4B000C7F89020D7F890201A6C42F010021A6466
:10A4C0001A6C02F01002C7F88C20D7F88C201A6C96
:10A4D00042F020021A641A6C02F02002C7F88820A9
:10A4E000D7F888201A6C42F040021A641A6C02F005
:10A4F0004002C7F88420D7F884201A6C42F080020A
:10A500001A641A6C02F08002C7F88020D7F8802005
:10A510001A6C42F480721A641A6C02F48072FA6740
:10A52000FA6F1A6C42F400721A641A6C02F4007228
:10A53000BA67BA6F1A6C42F480421A641A6C02F459
:10A5400080427A677A6F1A6C42F400421A641A6C7D
:10A5500002F400423A673A6F1A6C42F400321A640D
:10A560001A6C02F40032FA66FA6E1A6C42F4802217
:10A570001A641A6C02F48022BA66BA6E1A6C42F43B
:10A5800000221A641A6C02F400227A667A6E1A6C3F
:10A5900042F480121A641A6C02F480123A663A6E1F
:10A5A0001A6C42F400121A641A6C02F40012FA6572
:10A5B000FA6D1A6C42F480020EE000BF00380240CF
:10A5C0000070004004400240EFBEADDE00ED00E050
:10A5D0000005FA05EC9301201A641A6C02F480025B
:10A5E000BA65BA6D1A6C42F400021A641A6C02F46D
:10A5F00000027A657A6D1A6C42F000721A641A6C65
:10A6000002F000723A653A6D1A6C42F000521A6418
:10A610001A6C02F00052FA64FA6C1A6C42F0804232
:10A620001A641A6C02F08042BA64BA6C1A6C42F076
:10A6300000421A641A6C02F000427A647A6C5A6C16
:10A6400042F001025A645A6C02F001023A643A6C18
:10A650005A6C42F002025A645A6C02F00202FA6327
:10A66000FA6B5A6C42F010025A645A6C02F01002F3
:10A67000BA63BA6B5A6C42F020025A645A6C02F008
:10A6800020027A637A6B5A6C42F480725A645A6C74
:10A6900002F480723A633A6B5A6C42F400725A6464
:10A6A0005A6C02F40072FA62FA6A5A6C42F48062DE
:10A6B0005A645A6C02F48062BA62BA6A5A6C42F402
:10A6C00000625A645A6C02F400627A627A6A5A6CC6
:10A6D00042F480525A645A6C02F480523A623A6AE6
:10A6E0005A6C42F400525A645A6C02F40052FA61F5
:10A6F000FA695A6C42F480325A645A6C02F480321D
:10A70000BA61BA695A6C42F400325A645A6C02F463
:10A7100000327A617A695A6C42F480225A645A6C27
:10A7200002F480223A613A695A6C42F480125A6407
:10A730005A6C02F48012FA60FA685A6C42F4800291
:10A740005A645A6C02F48002BA60BA685A6C42F4D5
:10A7500000025A645B6C03F400037B607B6830F09A
:10A7600031FE1D4B02461D491B681D48A1FB03130A
:10A770001C49A0FB02029B09920C013B0A60B3F149
:10A78000807F08D2184AF02500200721536084F802
:10A79000235090601160144AE037136843F00403BB
:10A7A0001360BD46B0BD114A01F5484102605A6CC4
:10A7B0000F4842F480425A645B6C03F48043C7F84C
:10A7C000DC30D7F8DC300A6803680A6083F3088855
:10A7D000084B1B689847FEE7DC160120D34D62103A
:10A7E00083DE1B433064012010E000E0EDFEFECA72
:10A7F0000000F01F0400F01F08B5054B1B6803B1F3
:10A800009847044B044A1A6072B6FEF703F800BF7B
:10A81000FC3B012004400240EFBEADDE08B5034B17
:10A820001B6803B1984772B6FDF7F4FFFC3B0120AB
:10A8300030B40D4D182400222B4604E001321833A9
:10A840000D2A0DD01C79A042F8D19C79214201D16A
:10A850000029F3D102EB420205EBC20030BC704785
:10A86000002030BC704700BF7063040830B5F02290
:10A8700087B00021244838F064FF244A244C112377
:10A88000516C04F59C7541F001015164516C01F06B
:10A89000010101910199116C41F002011164116CE7
:10A8A00001F0020102910299116C41F0040111645E
:10A8B000116C01F0040103910399116C41F008013E
:10A8C0001164116C01F0080104910499516C41F07C
:10A8D00002015164526C02F002020592059A2BB9F2
:10A8E0001834AC420DD0A379002BF9D0207918345C
:10A8F00004F068F814F8102C022104F02DF9AC4291
:10A90000F1D107B030BD00BF2480012000380240E3
:10A910007063040801490248FEF752BBC48001205D
:10A9200000040140FFF7F6BF01490248FEF748BBAB
:10A930009C800120000C004001490248FEF740BB0A
:10A94000748001200008004001490248FEF738BB2E
:10A950004C8001200004004001490248FEF730BB52
:10A960002480012000000140FFF7F6BF0368134A6E
:10A970009B0A93421FD010D8023A934219D0013259
:10A98000934213D102214279022389010C48DA4013
:10A9900041589340DB430B6170470A4A934206D00B
:10A9A0000132934201D10421EDE770477047002145
:10A9B000E9E70121E7E70321E5E700BF0300100015
:10A9C00090C501204000100003681B4A9B0A934277
:10A9D0002FD013D8023A934229D00132934222D188
:10A9E0000223A1B99B01417902221448D140C058E9
:10A9F0008A40C36823EA0203C3607047104A934247
:10AA000013D0013293420FD104230029EAD002224D
:10AA10009B0141790948D140C05802FA01F3C2684C
:10AA20001343C3607047704770470023D9E7012381
:10AA3000D7E70323D5E700BF0300100090C501202E
:10AA40004000100003682DE9F0439B0A554CA342D7
:10AA500000F0918028D8023CA34200F0908001349D
:10AA6000A3427CD1407902244F4F860841BBA50107
:10AA70004FF0020E4FEA840C57F8058020FA0EF0D2
:10AA80000CEB04050EFA00FED8F80C0006EB4505A9
:10AA900020EA0E00DFF818E12E1DC8F80C004EF871
:10AAA00025104EF8262025E0404CA34265D0013405
:10AAB000A34256D1042440793B4F86080029D6D0C2
:10AAC0004FEA841E02254FEA840C57F80E8005FADF
:10AAD00006F00CEB040ED8F80C9006EB4E05DFF8F0
:10AAE000D0E040EA09002E1D4EF825104EF8262031
:10AAF000C8F80C002B4A934247D034D8023A93420C
:10AB000041D00132934248D102260CEB0403DB0012
:10AB100003F120007044EFF31185502282F3128874
:10AB20001033002273441968013211B101601868B2
:10AB30000430042A03F10403F5D10023EDB20360CD
:10AB400085F311886444B6010EEBC404BA59236A34
:10AB5000EBB1D36843F00103D360BDE8F083BDE8F7
:10AB6000F083BDE8F083114A93420AD00132934248
:10AB700015D10426C9E703249DE700249BE701249F
:10AB800099E70026C1E70126BFE70326BDE7D368A2
:10AB900023F00103D360BDE8F083BDE8F083BDE896
:10ABA000F08300BF0300100090C50120400010009A
:10ABB00024800120F0B5830A544C85B0A34200F0F4
:10ABC000A08040D8023CA34200F099800134A34207
:10ABD00037D10225AD014E4E73597719984230D0C6
:10ABE0004C4B01394FF0000E04461B6889B270517E
:10ABF0003846F960C7F810E0C7F808E0C7F814E075
:10AC0000B3FBF2F2013A7A6030F094FE4249B4F1BB
:10AC1000804F18BF8C420CBF012100211BD03F4B3D
:10AC20009C4218D003F580639C4214D03C4A03F543
:10AC30007C439C4218BF94420DD003F570539C4254
:10AC400009D005B0F0BD374CA34256D00134A34221
:10AC5000F7D10425BEE7721900234FF4805792F80C
:10AC60003C0001930128029303930097E9D07059A7
:10AC70000227DFF8B8E04FF0010C82F83D708768DA
:10AC800007EA0E0E284FC0F808E0D0F808E00EEAF8
:10AC90000707876082F83C3082F83DC0B9B91F4B86
:10ACA0009C4214D003F580639C4210D003F580636E
:10ACB0009C4203D003F578439C42C2D17219002311
:10ACC00092F83C200093012A01930293B9D0735962
:10ACD00011485A688342996815D000F58060834214
:10ACE00011D022F0700221F08001354400205A601A
:10ACF000996085F83C0005B0F0BD00256AE70125A4
:10AD000068E7032566E722F47002EAE70300100013
:10AD100090C50120DC160120000001400004004025
:10AD2000000C004040001000F8FFFEFF8800FEFF0E
:10AD3000F8B50668324CB30AA34239D007D8023CB2
:10AD4000A34237D00134A3422ED1022506E02D4C78
:10AD5000A3422BD00134A34227D104250446304618
:10AD6000FFF728FF284AAB01022021680127D518E8
:10AD7000D658264A002385F83D00346824483C43D1
:10AD8000346085F83D7001E050F83320914213D0D3
:10AD900001330E2BF8D10020012122F00FF9002001
:10ADA000BDE8F8401AF0B2BEF8BDF8BD0025D5E701
:10ADB0000325D3E70125D1E7154A012102EBC3039F
:10ADC0005C7965B2284622F0F9F828461AF09EFE12
:10ADD0001B2C0AD02E2C11D101212C2022F0EEF8B0
:10ADE0000C4B4FF480525A60F8BD0121192022F01B
:10ADF000E5F8084B4FF000721A60F8BDF8BD00BFCF
:10AE0000030010004000100090C501200000014028
:10AE1000DC64040800E100E0800A0E4B984216D082
:10AE200007D8023B984210D00133984209D10A4812
:10AE300070470A4B984206D00133984201D1084826
:10AE40007047002070470748704707487047074819
:10AE5000704700BF0300100010C601204000100022
:10AE600090C6012090C50120D0C5012050C6012008
:10AE70002DE9F041284EC0EB401506EBC5056B6887
:10AE800083B3DB6873B32B7BC0EB40100027234AEE
:10AE900043EA41011268C4008BB22F73284619128D
:10AEA00081EA1311594001F00F0141EA031189B2FF
:10AEB00090476A6895F89530D179490710D4022BEC
:10AEC00010D095F895305179012B1CD004F1100267
:10AED000583483B232443019BDE8F04130F07ABBC7
:10AEE000022B01D1BDE8F08195F895305179012B05
:10AEF0000DD004F11002583483B232443019BDE849
:10AF0000F04130F06BB9022385F89530DEE702237B
:10AF100085F89530EDE700BF7C7701207077012040
:10AF2000114B98421ED003F5806398421AD00368F3
:10AF300023F04003036059B141F48071002991FA74
:10AF4000A1F3B3FA83F108BF4FF0FF310139C90013
:10AF5000036823F0380319430160036843F040039A
:10AF6000036070474908E2E70038004030B44468A5
:10AF7000012B24F4805444601CDD40F2E93401E0EC
:10AF8000013C35D08568AD07FAD500293DD031F8B0
:10AF9000024B848140F2E93401E0013C28D085680D
:10AFA000ED07FAD5C468A4B20AB122F8024B023BFD
:10AFB000012BE2DC446844F48054446013B340F253
:10AFC000E93301E0013B37D08468A407FAD50029B2
:10AFD00036D00B78037340F2E93301E0013B2BD00C
:10AFE0008168C907FAD5C368DBB25AB1137009E0AA
:10AFF000144B98420CD0144B984219D003F580633F
:10B00000984217D0012030BC70474FF6FF74C0E75C
:10B0100023460E4AD82101FB03239A89013292B2BA
:10B020009A81988980B2003030BC18BF01207047E7
:10B030000123EEE70223ECE7024A9042DBD1E8E786
:10B04000FF23C7E7003001400038004064C70120FB
:10B0500030B5144C83B023781BB90120237003B0A2
:10B0600030BD052200238DF800208DF8013000BF8F
:10B070000D4D2B68D86803F077FD2B6801AA69464F
:10B0800058680223FFF772FF2B68D86803F072FD3F
:10B0900000BF9DF8053003F0010383F00100237029
:10B0A00003B030BDC4CA01204CC7012070B5064CA6
:10B0B0000646256803E023685B1BB34203D8FFF70D
:10B0C000C7FF0028F7D070BD2C64012070B503467F
:10B0D00082B003240E468DF80730190C1B0A062097
:10B0E00015468DF805108DF806308DF80440FFF7F1
:10B0F000DDFFC8B100BF0D4C2368D86803F034FDF4
:10B10000226801A9042350680022FFF72FFF21685D
:10B1100032462B4648680021FFF728FF2368D8688D
:10B1200003F028FD00BF284602B070BD4CC70120C7
:10B13000F0B589B00E4E0D4660F03F0308AC3068A4
:10B14000174604F8203D03F00FFD224621466B1CF4
:10B150000848FFF70BFF306803F00CFD2A4638461D
:10B160000DF1010136F0A4F8012009B0F0BD00BFD7
:10B1700064400120003C004070B582B004460621C6
:10B1800003206A46FFF7D4FF00283CD09DF800302A
:10B190009DF801109DF8026041EA03219DF803200B
:10B1A0009DF804509DF8053042EA062209B243EAB0
:10B1B000052312B206EE901A1BB2144907EE102AAC
:10B1C000F8EEE66A07EE903A91ED035AB8EEC77AC8
:10B1D000D1ED055AF8EEE77A91ED046A66EE856ADC
:10B1E00027EE257A67EE867AFDEEE66ABDEEC77A2F
:10B1F000FDEEE77A16EE901A17EE102A17EE903A47
:10B200002180A280638002B070BD00BF00000120D9
:10B2100010B50B4C88B000F07F0320688DF801104A
:10B220008DF8003003F0A0FC022300226946054897
:10B23000FFF79CFE206803F09DFC012008B010BDC4
:10B2400064400120003C00402DE9F043002483B01D
:10B2500032200A2703F0D8F9112120462546FFF7AE
:10B26000D7FF602101202646FFF7D2FF642003F0BC
:10B27000CBF96846DFF83081FFF77EFF012102201D
:10B28000FFF7C6FF322003F0BFF96846FFF774FFEF
:10B29000BDF90230BDF904100120BDF900201D44A4
:10B2A0008B420C441644A8BF0B469342A8BF1346DA
:10B2B00043456CDB03F0BEFA013FDFD14FF00109DB
:10B2C000122100200A27DFF8E080FFF7A1FF01210B
:10B2D0000220FFF79DFF322003F096F96846FFF742
:10B2E0004BFFBDF90230BDF904100120BDF900206B
:10B2F000ED1A8B42A4EB0104A6EB0206A8BF0B4695
:10B300009342A8BF1346434544DB03F093FA013F41
:10B31000DDD107EE906ADFED215A9FED215A7021B1
:10B32000F8EEE76A07EE905A0020B8EEE77A07EEEB
:10B33000904A85EEA66A1B4CC5EE876AF8EEE77A5E
:10B3400085EE277AF0EEC67AC4ED037AF0EEE67A5F
:10B35000C4ED047AF0EEC77AC4ED057AFFF758FF22
:10B3600020210120FFF754FF00210220FFF750FFAA
:10B37000642003F049F9B9F1000F04D14FF07E5376
:10B38000E36023616361012003B0BDE8F0834FF007
:10B39000000995E74FF00009BBE700BF00406F468A
:10B3A00001C05E460000012001F0FFFF70B50446B9
:10B3B00082B0006A03F0D8FB6A4607231049A069EF
:10B3C000FFF7D4FD206A03F0D5FB9DF801309DF80E
:10B3D000021001209DF8036041EA03219DF804203A
:10B3E0009DF805509DF8063042EA0622A4F8401068
:10B3F00043EA0523A4F84220A4F8443002B070BD0B
:10B40000C83A040840F2E93300E09BB18268013B8E
:10B4100012F0020F9BB2F8D0017340F2E93300E062
:10B4200043B18268013B12F0010F9BB2F8D0C068B3
:10B43000C0B270470C4A904209D00C4B984211D0D0
:10B4400003F58063984201D0FF2070470223084A29
:10B45000D82101FB03239A89013292B29A819889FB
:10B46000C0B270470123F2E70030014000380040CD
:10B4700064C7012038B5054600BF084C2368D8686A
:10B4800003F072FB236829465868FFF7BBFF236867
:10B49000D86803F06FFB00BF38BD00BF4CC7012068
:10B4A0002DE9F04FB2F1000A89B0029004910393A4
:10B4B00040F3AD800B46002201EB8A0153F8040BE8
:10B4C0008B420244FAD1039B0592002B00F0978037
:10B4D000059B002B6BD0059BDFF858910093504BD8
:10B4E0001B68DAB200995118B1F5807F8CBFC2F5A4
:10B4F0008072009A01924B4A92689A426BD9190C59
:10B500004FF002041A0A06208DF81F308DF81E2015
:10B510008DF81D108DF81C40FFF7C8FD0620FFF7C1
:10B52000A9FF0123404A137000BFD9F8003000245E
:10B53000049DD868A34603F017FBD9F8002007A99B
:10B54000042350682246FFF711FD029E019F2968DF
:10B550004FEA8408002201340B4671B1B942D9F890
:10B56000000028D231684068FFF700FD2A68336880
:10B57000BF1A13443360C5F800B0A24505F10405B5
:10B5800006F10406E3D1D9F80030D86803F0F2FAE6
:10B5900000BF234B9DE806001B68891A1344204A0C
:10B5A00000911360039A1AB3009A002A99D1059862
:10B5B00009B0BDE8F08F029C3B46406854F8081083
:10B5C000FFF7D4FC54F808202B683A44DF1B44F8FA
:10B5D00008202F60D7E705980023009C1349001B23
:10B5E000134A0B7005900598137009B0BDE8F08FF1
:10B5F000059B5B1A0593059809B0BDE8F08FFFF72E
:10B6000027FD00287FF464AF039B0593CFE7039BDE
:10B610001BB90593FFF71CFDC9E700230593C6E797
:10B620001C470120201E0120C4CA0120A44701207C
:10B63000204701204CC70120F0B5104E85B0104FB7
:10B6400033783A78934214D00E4903EB010003910A
:10B65000029010D9C3F18004154604A901230222E7
:10B6600002A841F8104D0195FFF71AFF00233B7027
:10B67000337005B0F0BDD41A0025EEE72047012055
:10B68000A447012024470120124BF0B59D6885B0E6
:10B690000DB905B0F0BDED0A14D0002704AE7C1939
:10B6A000102269466410E002FFF710FD0F2809DD43
:10B6B0006B4653F8042B01320AD1B342F9D1254627
:10B6C000AF42ECDBFFF7B8FF034BED021D60E0E794
:10B6D000671CF5E7201E01201C470120F0B5194D1D
:10B6E00085B0194E2B7832789A4228D0174903EB4F
:10B6F00001000391029019D2C3F18004174604A9F6
:10B700000023022202A841F8104D0197FFF7C8FE5E
:10B710002B781844C0B20306337848BF80F080000D
:10B720008342287005D0002005B0F0BDD41A002750
:10B73000E5E70023012033702B7005B0F0BD012038
:10B7400005B0F0BD20470120A44701202447012077
:10B7500008B545F20820FFF7A9FC0620FFF78AFE8E
:10B76000064B0122C7201A70FFF784FE002304480D
:10B770000449054A03700B70136008BDC4CA012058
:10B78000A4470120204701201C47012030B5044672
:10B790000D4683B0C06803F0E7F945F080016068AA
:10B7A000FFF730FE01230DF1070200216068FFF76B
:10B7B000DDFBE06803F0DEF99DF8070003B030BD63
:10B7C00008B5034B02211868FFF7E0FF002008BD11
:10B7D00068400120F8B504460F4615461E46C0686D
:10B7E00003F0C2F947F080016068FFF70BFE3346B3
:10B7F0002A4600216068FFF7B9FBE06803F0BAF958
:10B800000120F8BD70B50B4C0646237853B90A49A0
:10B81000002532466378086849212570FFF7DAFF72
:10B82000012070BDFDF7FEF80028F0D002F092FE76
:10B83000EDE700BF44C7012040C70120F0B54A4CE6
:10B8400083B0257D012D13D028D3022D0DD1474B78
:10B8500006461B78002B77D16846FFF7D3FF20B14F
:10B860009DF8063013F0030722D0002003B0F0BD8E
:10B870003E4E3378002B62D16846FFF7C3FF9DF838
:10B88000003008B1DB0764D40023237533784BB153
:10B89000002301330020237503B0F0BD334E33780D
:10B8A000002BF5D10121022033F0C6FE237DF0E705
:10B8B0009DF8012001219DF800500A209DF80330D9
:10B8C00045EA02259DF802209DF805E042EA0322A0
:10B8D0009DF804302DB2277543EA0E23244C12B292
:10B8E0006D421BB294ED005A524206EE905A5B42F2
:10B8F000D4ED015A07EE102AF8EEE66A07EE903A08
:10B9000094ED026AB8EEC77AF8EEE77A66EE856AD9
:10B9100027EE257A67EE867AFDEEE66ABDEEC77AF7
:10B92000FDEEE77A16EE904A17EE102A17EE903ADF
:10B9300034807280B38033F023FE03B0F0BDFDF796
:10B9400071F8002898D090E7FDF76CF800288CD1AA
:10B9500082E7337823B90721032033F06DFE257D7C
:10B9600001350020257581E70420012044C701200E
:10B970000000012070B504460E461546C06803F06D
:10B98000F3F831466068FFF73DFD29466068FFF730
:10B9900039FDE06803F0EEF8012070BD10B51D4CD4
:10B9A00082B01D220F212068FFF7E4FF0A2002F079
:10B9B0002BFE00220A212068FFF7DCFF142002F092
:10B9C00023FE0F220A212068FFF7D4FF0A2002F08D
:10B9D0001BFE032301AA10212068FFF7FBFE0A20AB
:10B9E00002F012FE00220A212068FFF7C3FF0A209E
:10B9F00002F00AFE20680221FFF7C8FE2068092134
:10BA0000FFF7C4FE206801220A21FFF7B3FF0120DF
:10BA100002B010BD6840012030B5037883B0012B1F
:10BA20000AD0022B02D0002003B030BD01F07F010C
:10BA3000FFF7A0FF03B030BD0446154602AB0A462F
:10BA4000647903F8015D214690F9040021F0C2FBFE
:10BA500003B030BD01224821DEE700BF012258219A
:10BA6000DAE700BF3122F421D6E700BF10B54FF46A
:10BA7000807104468069FFF753FA012002F06AFDE5
:10BA80002046FDF751F810226A2104F11400FFF757
:10BA900071FF642002F0B8FDA0690421FFF740FAAD
:10BAA0000120BDE8104002F055BD00BFF8B5D82315
:10BAB000604D614A044603FB00F3E9582B44914270
:10BAC00000F09580D823661C03FB0453F6B2187966
:10BAD00002F078FF074610B11223C6718371D82394
:10BAE00003FB0453587902F06DFF10B11323C671A4
:10BAF0008371D82303FB0453987902F063FF10B1DC
:10BB00001423C6718371D82303FB04539A7B002A44
:10BB10005CD0DA7938464E2103F01EF8D82606FBB1
:10BB200004F6AF19787902F04DFF3A7A2E2103F02E
:10BB300013F8B87902F046FF7A7A0E2103F00CF878
:10BB4000AB593E491A688B4222F040021A6051D02C
:10BB5000394A934258D03A4A934260D0394A934284
:10BB60003AD0394A934209D102F56842516A41F408
:10BB700080115162516A21F480115162D8225968B2
:10BB800002FB045441F48051A27B5960002A1968D9
:10BB900014BF0024022449060FD41D6882F001025C
:10BBA0002A482B492840024342F4457222431A6036
:10BBB0005A68114041F4E0615960DA6922F4006288
:10BBC000DA611A6842F040021A60F8BDDA79384644
:10BBD0002E2102F0C1FFA1E702F58232516A41F441
:10BBE00000515162516A21F400515162C6E70122AD
:10BBF0009A7367E7174A516A41F480515162516A5A
:10BC000021F480515162B9E702F50032116A41F422
:10BC100080411162116A21F480411162AEE702F5A0
:10BC2000FE32116A41F400411162116A21F40041AF
:10BC30001162A3E764C701200038004000300140D2
:10BC4000003C004000340140005001404000FFFF34
:10BC5000FBF0FFFF0038024070B5C0EBC0000D4C98
:10BC60000D4E82B004EB8004306B256928433063AD
:10BC7000366B94F90D003540A1606361910901951F
:10BC8000019B21F09BF994F90D0019F03FFF02B0E0
:10BC900070BD00BFE0160120003802400A4BC0EB27
:10BCA000C00030B403EB8000084C82B0256B036900
:10BCB0001D432563246B0176234042760193019B4B
:10BCC00002B030BC704700BFE016012000380240CF
:10BCD0000348D0F8AC3113B100F5D2701847704763
:10BCE000E01601200348D0F8903113B100F5C4707C
:10BCF00018477047E01601200348D0F8743113B19B
:10BD000000F5B67018477047E01601200348D0F8D8
:10BD1000583113B100F5A87018477047E01601209C
:10BD20000348D0F83C3113B100F59A7018477047BA
:10BD3000E01601200348D0F8203113B100F58C70D3
:10BD400018477047E01601200348D0F804310BB1C2
:10BD5000FC301847704700BFE01601200348D0F8B8
:10BD6000E8300BB1E0301847704700BFE016012003
:10BD70000348D0F8CC300BB1C4301847704700BF2F
:10BD8000E01601200348D0F8B0300BB1A8301847B6
:10BD9000704700BFE01601200348D0F894300BB183
:10BDA0008C301847704700BFE01601200248836FAF
:10BDB0000BB1703018477047E01601200248C36D80
:10BDC0000BB1543018477047E01601200248036C4D
:10BDD0000BB1383018477047E01601200248436A1B
:10BDE0000BB11C3018477047E016012002488368E9
:10BDF00003B11847704700BFE016012004282DE961
:10BE0000F04FD4BF0024012483B0B0F1FF3F08BF3E
:10BE100044F0010404BB4FEA400ADFF83C930AEB0C
:10BE20000006760109EB060C1436DCF814E04E44EB
:10BE3000BEF1000F0CD0174605469CF85520FF2F89
:10BE40000FD0202A7BD0BF4A138801339BB21380C6
:10BE5000204603B0BDE8F08F0024204603B0BDE8C3
:10BE6000F08F202AEFD19CF85420012AEBD0012238
:10BE7000DFF8E8828CF85420D8F8007005E0D8F894
:10BE80000020D21B192A00F20A81DEF8182012F4D1
:10BE90000042F4D110460AEB05029BB24FF0220B90
:10BEA00009EB42124FF0100C490082F855B082F8AD
:10BEB00056C09065D387D38F00919BB20C99906444
:10BEC000FF2B916340F21F81FF20DEF80410DFF8A2
:10BED00090C290879C4B01EA0C01009A13430B43DC
:10BEE000CEF804300AEB050B984B009A09EB4B1B7C
:10BEF00013430193BBF83E309BB2002B00F0168138
:10BF0000DBF814100BE08B6913F0200340F0AF80D6
:10BF1000D8F80020D21BB2F5805F00F2CC808B698C
:10BF20005B0769D48B69DA06EDD53946304621F0D6
:10BF30009DF8002840F0AD80DBF81410E3E79AB2DA
:10BF40000C9B002B3FF47FAF002A3FF47CAF9CF8A2
:10BF50005430012B3FF477AF0123DFF800828CF8D7
:10BF60005430D8F800B006E0D8F80030A3EB0B034B
:10BF7000192B00F29480DEF8183013F40043F3D14B
:10BF800018460AEB05034FF0220C4FEA410809EB73
:10BF900043134FF0400183F855C048F4903C83F8B8
:10BFA000561059469865DA87DEF8042098643046C2
:10BFB00000920C9A9A63009A009322F07F7222F406
:10BFC000593222F47F7222F003024CEA0202CEF8C8
:10BFD000042021F08BF8009B002800F0C3809B6DAB
:10BFE0000AEB0503002209EB43139B6D602303FB5F
:10BFF000059585F8542026E7DBF838304A6A591C45
:10C00000CBF838101A70BBF83C30BBF83E20013B2F
:10C01000013A9BB292B2ABF83C30ABF83E20002B19
:10C020007FF468AFBBF83E309BB2002B3FF462AFA9
:10C030003A468021304621F083F800287FF403AF90
:10C04000BBF83E309BB2FF2B43D9DBF81420FF2115
:10C050005368ABF83C1023F07F73019923F45933F4
:10C0600023F47F7323F003030B43536042E720263E
:10C07000374A0AEB0503CE61486809EB43131040C9
:10C08000002248609A6583F8542083F8556083F84D
:10C090005620554409EB4519D9F85830D3E6554494
:10C0A0000023202209EB451989F8552089F85430DE
:10C0B00089F85630C7E61A460AEB0503202009EB3B
:10C0C0004313996D83F854200143996583F8550013
:10C0D000DFE7DBF81410009BBBF83E2043F0007054
:10C0E0004B6892B223F07F735FFA82FEABF83C207C
:10C0F00023F4593323F47F7323F00303034343EA08
:10C100000E434B60F6E6D18FDFF854C089B2DEF8FB
:10C110000400104B918700EA0C00009AC9B2134347
:10C12000034343EA0143CEF80430DBE639463046A8
:10C1300021F026F86023002800F0A98003FB059574
:10C14000AB6D80E6F46301200024FF010000FF01D5
:10C1500000E800FE002400027462012070620120E9
:10C16000009800FC586940215A4600938762304687
:10C1700020F0E6FF009B00287FF432AFDB8F9BB2FC
:10C18000FF2B40F295806022FF20564B02FB059268
:10C1900048EA0303516990874A6822F07F7222F4CB
:10C1A000593222F47F7222F0030213434B600AEBF0
:10C1B00005034D4F09EB431A48EA070704E0BAF8B4
:10C1C0003E309BB2002B5AD05A460421304620F014
:10C1D000B7FF00287FF437AEDAF83830DAF81420E9
:10C1E000591C526ACAF838101A70BAF83C30BAF8BA
:10C1F0003E20013B013A9BB292B2AAF83C30AAF829
:10C200003E20002BDBD1BAF83E309BB2002BD6D0BB
:10C210005A468021304620F093FF48F00072FF21FB
:10C2200000287FF410AEBAF83E309BB28B420FD993
:10C23000DAF81420AAF83C10536823F07F7323F433
:10C24000593323F47F7323F003033B435360B6E772
:10C25000DAF81410BAF83E004B6880B223F07F730E
:10C260005FFA80FEAAF83C0023F4593323F47F736D
:10C2700023F00303134343EA0E434B609FE7594601
:10C28000304620F07DFF602300287FF457AF03FB8A
:10C2900005952021154E01246B69D9615A683240F9
:10C2A0005A6085F8551085F8540085F85600CFE59A
:10C2B00060270F4807FB059748EA00007969FA8F65
:10C2C0004B6892B223F07F73BA87D2B223F459330A
:10C2D00023F47F7323F00303034343EA02434B60D9
:10C2E00065E700BF0024FF010000FF0100E800FE39
:10C2F0000024000270B5057882B01E46012D0DD0D5
:10C30000022D02D0002002B070BD134641F0800122
:10C31000324602B0BDE87040FFF75CBA13460A46E9
:10C32000417990F904000096FFF768FD02B070BDF6
:10C3300000B583B00322002101ABFFF7DBFF9DF8BE
:10C3400005309DF804201B029DF8060043EA0243D5
:10C35000184303B05DF804FB08B5FFF7E9FF014B94
:10C36000586008BD0420012008B5FFF7E1FF014B2C
:10C37000186008BD0420012000B583B00622F72113
:10C380006B46FFF7B7FF9DF801209DF804309DF83C
:10C39000001012019DF803001B0142EA01329DF8D2
:10C3A000021043EA00339DF8050042EA11120449E5
:10C3B00043EA1013CA608B6003B05DF804FB00BF52
:10C3C0000420012000B583B0002000920A466821B5
:10C3D000FFF714FD03B05DF804FB00BF01482EF029
:10C3E000EFBE00BF4863012001482EF0ABBE00BF86
:10C3F0004863012001482EF0E3BE00BFE86201203F
:10C4000001482EF09FBE00BFE862012001482EF0D7
:10C41000D7BE00BF8862012001482EF093BE00BF46
:10C4200088620120A54A0021A54BA64870B5D2F824
:10C4300088404FF00065A44EA4B044F47004C2F8E4
:10C4400088401C6844F001041C6099601C6820400E
:10C4500018605E60186820F480201860D9609560CC
:10C46000BFF34F8FBFF36F8FC2F85012516941F481
:10C4700000315161BFF34F8FBFF36F8F196C934A37
:10C4800041F080511964196C01F0805102910299B8
:10C49000116841F440411160126802F44042019277
:10C4A000019A9A6802F00C02042A52D09A6802F0AB
:10C4B0000C02082A4AD0824B854C1A68194642F46D
:10C4C00080321A60226803E023689B1A642B3CD8F0
:10C4D0000B689803F8D57A4B9A6802F00C02082A88
:10C4E00033D01A68184622F080721A60226803E07E
:10C4F00023689B1A022B28D803689B01F8D447F6BF
:10C50000C07393FAA3F34FF44031B3FA83F291FA74
:10C51000A1F14FF0706191FAA1F10926B1FA81F110
:10C520004FF4D8736B4D8E406549934033431D43A0
:10C530004560036843F08073036022680B689E01C6
:10C540000BD423689B1A022BF8D9FEE75B685C02C8
:10C55000B1D55B4B5E4C1B68BDE7086C5B4A40F095
:10C56000805013460864096C01F0805103910399CF
:10C57000116841F48031116021685A68D50305D4EF
:10C580002268521AB2F57A7FF7D9FEE71A684F4946
:10C5900042F400321A60226804E023689B1AB3F563
:10C5A0007A7FF2D84B689803F7D54FF400164FF016
:10C5B00000654FF4C0710722032304A80496219557
:10C5C000089109920A9334F075FB00B1FEE7424AE4
:10C5D000136803F00F03062B1BD9394B9A6822F01E
:10C5E000F0029A601A68920167D59A68184641F27B
:10C5F000883122F0030242F002029A6022688368C6
:10C6000003F00C03082B10D023689B1A8B42F6D939
:10C610000AE0136823F00F0343F007031360136865
:10C6200003F00F03072BD8D0FEE72B4A136803F063
:10C630000F03072B35D8224CA36823F4E05343F4AF
:10C64000A053A360A36823F4604343F40043A360B2
:10C650002EF0B8FEA368F02292FAA2F2B2FA82F2A9
:10C6600003F0F0031D4ED3401D4D334493F88C303E
:10C6700020FA03F32B6020F0D5FC0023194A04A80C
:10C680000492139314931593169317931893199375
:10C690001A931B931C931D931E9334F00BFB18B33A
:10C6A000FEE7136823F00F0343F0070313601368DA
:10C6B00003F00F03072BB7D1BDE7B5E700ED00E0AE
:10C6C00000380240FFFFF6FE1030002400700040EA
:10C6D0007062012008004020003C0240443A0408F7
:10C6E000DC160120C0FF0300D4F88C3023F08073E7
:10C6F000C4F88C30D4F88C3043F08073C4F88C309C
:10C70000A36803F00C03042B27D0082B0DD0154B86
:10C71000154A16499268C2F30312164496F88C2003
:10C72000D3408B422B601AD0FEE7616862684B02EF
:10C73000616802F03F024CBF0D4B0A4BB3FBF2F3B2
:10C74000C1F3881203FB02F3074A5268C2F30142A5
:10C7500001325200B3FBF2F3DAE7054BD8E724B01D
:10C7600070BD00BF0024F4000038024000E6DF0C7A
:10C7700000127A0038B50B4C23688BB15A68054615
:10C78000821A002A04DA0CE05A68AA1A002A07DB87
:10C790009A6818461B68226098472368002BF3D1DB
:10C7A00038BD38BD2C3F012000210B4B10B40A4688
:10C7B0001124017202E007290BDC9C79A40702F125
:10C7C000010202D51C79445401310C2A03F11803EB
:10C7D000F1DD5DF8044B70477063040818230370A3
:10C7E000704700BF0123312134224171C2700370B0
:10C7F0000371837010B4302444705DF8044B7047AB
:10C800002C2202230270437070470B4B30B503F1AA
:10C81000140493F90020043313F8035C072AC8BFFB
:10C82000143A81180D7313F8025C855413F8012C27
:10C83000A3420A76EDD130BDE03A040803682DE941
:10C84000F041DF691FB13B46BDE8F0411847002ABF
:10C85000164611DD04460D460E4400E023689B6831
:10C86000204698470028F9D02368204615F8011B78
:10C870001B689847AE42F1D1BDE8F08100233C210E
:10C880004222017042708370C3707047094B03F1FC
:10C890000C0110B593F90020043313F8034C8454B1
:10C8A000024413F8024C147113F8014C8B421472B9
:10C8B000F0D110BDF43A040810B51022002104464E
:10C8C00036F03FFF26232370272323710123237291
:10C8D000237310BD08B513F0C5FAFDF79FFF00BF25
:10C8E000024A034B1278197814F096BD01230120F7
:10C8F00002230120A0F10A032DE9F04F0C462DED93
:10C90000028B89B0E72B00F27887DFE813F01C0177
:10C91000760776077607760776077607760776072F
:10C92000760776077607760776077607760776071F
:10C93000760776077607760776077607760780010B
:10C940007607760776077101760776077607640122
:10C950007607810276073E027607330276072B02BE
:10C960007607FF017607EC01760776077607E60182
:10C97000DF0176071606760776070E0676071F068E
:10C9800076077607760781037607760776077607B8
:10C9900017037607FC0076075903360376077607F8
:10C9A000760776077607760776071F077607D2069B
:10C9B00076079D06760748067607610776077607AD
:10C9C00076077607EA05AF057B05C502E8003E0558
:10C9D0002A0563051D057607E504C7047607760773
:10C9E00076077607BC04760776079B0476077607FA
:10C9F00076078C04750461041D04760776077607B4
:10CA0000E303CC03BD039D0376077607760776071D
:10CA1000760776077607760776077607760776072E
:10CA2000760776077607EA057607760776077607AC
:10CA3000760776077607760776077607760776070E
:10CA400076072D017607760776077607760776074D
:10CA500076077607760776077607760776077607EE
:10CA600076077607760776077607760776077607DE
:10CA700076077607760776077607760776077607CE
:10CA800076077607760776077607760776077607BE
:10CA900076077607760776077607760776077607AE
:10CAA000760776077607760776077607760776079E
:10CAB000760776077607760776077607760776078E
:10CAC000760776077607760776077607760776077E
:10CAD00076077607760776077607A201AD01B74E8F
:10CAE000337853B1B64F002537F8021F2046FCF7C4
:10CAF000EFFD01353378AB42F6DC012009B0BDEC27
:10CB0000028BBDE8F08FAD4E3378002BF5D0AD4FE2
:10CB10000025B8462368204617F815200135591C12
:10CB200008F1020821601A7018F8011C01EB81015C
:10CB300001EB810101F2EE2189B2FCF7C9FD3378E6
:10CB4000AB42E7DCD9E7A04D284633F007FA0028CE
:10CB5000D3DD2B460544226813F8011B501C9D426F
:10CB600020601170F7D1C8E70B68DFF8A0C2591C2C
:10CB70009CF8002021601A709CF80030002BBCD07B
:10CB8000924E0023924D934893492268013316F840
:10CB9000017F02F1010EC4F800E01770226815F859
:10CBA000017F02F1010EC4F800E01770226810F84E
:10CBB000017F02F1010EC4F800E01770226811F83D
:10CBC000017F02F1010EC4F800E017709CF800200C
:10CBD0009A42DADC91E70B680120804A1D1811782F
:10CBE0002560197023685278191821601A7085E73A
:10CBF0007B4D08462988FCF76BFDA9882046FCF789
:10CC000067FD20462989FCF763FD012076E7754D15
:10CC100005F150062878043530F09AFF2368027A2F
:10CC2000591C21601A70236815F8032C591C2160C7
:10CC30001A70236815F8022C591C21601A7015F817
:10CC4000012CAE42236803F1010121601A70E1D189
:10CC500053E7654D0846E989FCF73AFD2046A98966
:10CC6000FCF736FD012049E7604B03F170052268AF
:10CC7000073313F8071C501C20601170226813F84A
:10CC8000061C501C20601170226813F8051C501CF3
:10CC900020601170226813F8041C501C2060117071
:10CCA000226813F8031C501C20601170226813F8CE
:10CCB000021C501C2060117013F8011C9D42226858
:10CCC00002F1010020601170D1D116E70B6801223A
:10CCD0009918104621601A7010E708460021FCF7E9
:10CCE000E1FC01200AE7424D424E05F1300795F97B
:10CCF0000210414B93F9062008338A4200F08085E8
:10CD00009E42F7D10835BD42F1D1F6E63B4B03F127
:10CD10005A052268063313F8011C501C206011705C
:10CD2000226813F8061C501C20601170226813F84A
:10CD3000051C501C20601170226813F8041C501C44
:10CD400020601170226813F8031C501C20601170C1
:10CD500013F8021C9D42226802F10100206011704C
:10CD6000D7D1CAE60B680120254A1918527D2160E7
:10CD70001A70C3E6234D05F1800655F8041F2046BE
:10CD8000FCF790FCAE42F8D1B7E61F4D05F1400626
:10CD9000B5F880102046FCF79BFC236895F88220AC
:10CDA0000435591C21601A7095F87F20B54223681C
:10CDB00003F1010121601A70EAD19EE624390120B5
:10CDC000C6B2012078BA012060BC0120FF490120D1
:10CDD0000F4A01202F4A01201F4A0120C03F012095
:10CDE000F0610120C43F012084BC012098BE0120D5
:10CDF000CCCA0120E8760120B8760120182901204C
:10CE00000C77012074B4012078B40120FD49012081
:10CE1000B84D08460B682A7A591C21601A70A98BF4
:10CE2000FCF756FC298B2046FCF752FC698B204608
:10CE3000FCF74EFC2368EA7C2046591C21601A70DE
:10CE4000A98CFCF745FCE98C2046FCF741FC2368E3
:10CE5000AA7F2046591C21601A70236895F820206B
:10CE6000591C21601A70698CFCF732FC2368EA7A3D
:10CE70002046591C21601A70E968FCF713FC2368EE
:10CE800001202A7C191821601A70236895F8212046
:10CE9000191821601A7031E6974D984E05F1200758
:10CEA000DFF89482DFF894929FED958ADFF890B2D4
:10CEB000DFED948ADFF88CA20DE0FCEEE77ACDED91
:10CEC000017ABDF8041004352046FCF701FC183641
:10CED000BD423FF412AE717C0029F4D098F80030C6
:10CEE000D5ED007A012BE8D1D9F80030DB0440F110
:10CEF0004485F5EE407AF1EE10FA00F05585F4EE37
:10CF0000C87AF1EE10FA00F14F85F4EEE87AFDEE02
:10CF1000E77AF1EE10FA17EE903A00F274856FF4AA
:10CF2000F972303B02FB03F38AFB0312D917134457
:10CF3000C1EB632101F2DB5189B2C4E70B680846FB
:10CF4000714D591C2A7921601A7023686A79591C1D
:10CF500021601A702988FCF7BBFB2368AA79204658
:10CF6000591C21601A706988FCF7B2FB2368012004
:10CF7000EA79191821601A70C0E50B680125634E23
:10CF80005A190A601D700B68B278591921601A701D
:10CF90002CF080FB23685E4A5F195E492760187099
:10CFA000B1F90010B2F90000FCF72AFD23685A1904
:10CFB0002260187020463188FCF78AFB28469DE5E0
:10CFC0000A68012693190B60167018F0C3F900283F
:10CFD00040F0EE840346504D504A216841F2B417A8
:10CFE00041F27816204601F1010EC4F800E00B7002
:10CFF0002368D15D5F1C276019709159890AFCF77D
:10D0000051FBA96A20464908FCF74CFB012075E555
:10D01000FEF71EF823680028414D03F10101204668
:10D020000CBF0222032221601A702988FCF73AFB08
:10D03000A9682046FCF736FBFCF762FF0146204654
:10D04000FCF730FB012059E50B68364F591C3A7844
:10D0500021601A703B78002B3FF44FAD0025EEB2F3
:10D06000013530461DF066FD236842783046591C74
:10D0700021601A701DF05EFD01892046FCF728FB37
:10D080003B78AB42EBDC38E5274B08462749B3F940
:10D09000003081FB0321DB17C3EBA10189B2FCF750
:10D0A00017FB01202AE50A680120214B1518197881
:10D0B0002560117022685978151825601170226852
:10D0C00099781518256011702268DB781118216095
:10D0D000137013E5174D0846298AFCF7F9FA698A97
:10D0E0002046FCF7F5FA2046A98AFCF7F1FA012060
:10D0F00004E500BF0C770120983F0120F475012062
:10D100000000404200E08244102B01203C460120F8
:10D11000ACBA0120AEBA01201CB101206C9C0120E8
:10D12000201E0120354C012094BC012067666666F4
:10D13000E44901205477012078770120B47401205C
:10D14000DB9B914121053483DFF81CE30027FEB20D
:10D15000714600232268501C206016702268501C03
:10D16000206013700133226811F8010F062B02F1C1
:10D17000010525601070EDD101370EF1060E062F66
:10D18000E5D1A44900232268501C20601770226852
:10D19000501C206013700133226811F8010F0B2B13
:10D1A00002F1010525601070EDD1236807250120EB
:10D1B00000215E1C984A26601D7023681D1825609A
:10D1C0001970236892F8F020191821601A7095E4FC
:10D1D0000B680120914A1E189149157826601D7030
:10D1E000236889781D188F4A256019702368927802
:10D1F000191821601A7081E40A6808468A4B561C87
:10D200008A491D782660157022685D78561C266054
:10D21000157022689B78551C25601370C988FCF72F
:10D2200057FA01206AE4814D08462988FCF750FA34
:10D2300069882046FCF74CFA2046A988FCF748FA92
:10D2400001205BE47A4D05F16006A9882046FCF7D1
:10D250003FFAE9882046FCF73BFA29892046FCF78B
:10D2600037FA2368AA7A2046591C21601A7023686D
:10D27000EA7A591C21601A7055F80C1BFCF712FA57
:10D28000AE42E2D139E452236A492268501C206040
:10D29000137011F8013F002BF7D12EE400236648EC
:10D2A000226803EB430105680133561C6D5C0A2BB1
:10D2B00026601570026825680A4405F10106527857
:10D2C00026602A70026825680A4405F101019278F7
:10D2D00021602A70E4D110E4584D00230A682968BF
:10D2E000501C097820601170296822688978501CC8
:10D2F000206011702A6821681A440133481C527951
:10D30000032B20600A70F5D1236820462A68591C37
:10D31000127A21601A7023682A68591CD278216019
:10D320001A7023682A68591C127921601A702B68B8
:10D330005989FCF7CDF92A6823680120527A191817
:10D3400021601A702A684DE43D4B08461968FCF7C5
:10D35000A9F93C4B20461988FCF7BAF90120FFF7E0
:10D36000CDBB394B08461988FCF7B2F9374B20463C
:10D370001988FCF7ADF9364B226801201B7811188B
:10D38000034021601370FFF7B9BB324B08460A68AF
:10D390001B78511C304D03F0020321601370236889
:10D3A0002A7D591C21601A702968FCF77BF969688D
:10D3B0002046FCF777F929892046FCF789F9E989A5
:10D3C0002046FCF785F92046298AFCF781F90120DF
:10D3D000FFF794BB214D08462988FCF779F9698845
:10D3E0002046FCF775F9B5F904301D4A2046D917D7
:10D3F00082FB0323C1EBA30189B2FCF769F9012089
:10D40000FFF77CBB084610221649FCF71DF90120E6
:10D41000FFF774BB5BB5012078B40120A46C012038
:10D4200084BC012094BC01207CBC0120F42A012092
:10D43000C0C40120003B0408FC3801204C810120BD
:10D44000544F0120484F0120144901201649012062
:10D45000C8480120784F01207C4F0120584F0120FF
:10D4600067666666883F012037B50120A84B1B8B95
:10D47000B3F5006F00F29682B3F5806F00F2B782C9
:10D48000B3F5007F34BF01270227A24D05F10C063A
:10D4900055F8041B204691FBF7F189B2FCF718F907
:10D4A000AE42F5D19C4D9D4F05F10C06B5EC010A3D
:10D4B000D7ED097A80EE270A34F028F881B22046A9
:10D4C000FCF706F9AE42F1D1954D05F10C0655F881
:10D4D000041B204689B2FCF7FBF8B542F7D1FFF7F1
:10D4E0000CBB00238146DFF85C8201211D464FF60C
:10D4F000FF7ADFF854B2049306930593079305E08F
:10D5000001350B2D00F09A8118F9011F4F1C4AFAC2
:10D5100005F3F5D0DE07F3D5BBF800302B41D80773
:10D52000EED506A8FCF716FCEAE7084608227D4976
:10D53000FCF78AF80120FFF7E1BA0B6801207A4A6C
:10D540001D18917825601970FFF74CBB0B680846D1
:10D55000764A5E1C764D1178764A266019701168FD
:10D56000FCF7A0F823686F4A2046591C127A216004
:10D570001A702988FCF7ACF8A9882046FCF7A8F8AF
:10D5800029892046FCF7A4F800212046FCF7A0F8E2
:10D5900020460021FCF79CF80120FFF7AFBA0021DC
:10D5A0002046FCF795F800212046634D0E46FCF717
:10D5B0008FF820463146FCF78BF8236820465A1C2A
:10D5C00022601E7023682A68591C92F82C20216062
:10D5D0001A7023682A68591C92F8362021601A7044
:10D5E00023682A68591C92F8372021601A70236832
:10D5F0005A1C22601E7023685A1C22601E70236809
:10D600005A1C22601E702B68598FFCF761F82B683A
:10D610002046198FFCF75CF823682A682046591CBD
:10D6200092F82E2021601A7023685A1C22601E7006
:10D630002B68598EFCF74CF82B682046998EFCF726
:10D6400047F80120FFF75ABA3C4E08460B6872793A
:10D65000394D591C21601A702B68198CFCF738F869
:10D660002B682046D98BFCF733F871892046FCF7EC
:10D670002FF8B1892046FCF72BF82B682046598CEF
:10D68000FCF726F82B682046998CFCF721F8F189E5
:10D690002046FCF71DF8318A2046FCF719F82A6865
:10D6A0002368012092F82620191821601A70FFF7CC
:10D6B00025BA224EF378002B00F068810B68012216
:10D6C00008219818206019702368991821601A7031
:10D6D000236820461A4D591C2A7921601A70236844
:10D6E000AA78591C21601A702988FBF7F1FFE98993
:10D6F0002046FBF7EDFF23680120F279191821601D
:10D700001A702368EA78191821601A70FFF7F6B9C1
:10D71000FC4E0120384F0120A8740120B86C012074
:10D72000F04B01200C770120A0BC0120C03F01205C
:10D73000F061012068460120FC380120A46C012022
:10D7400054770120303B0408AAB5012013F058FE9D
:10D75000FF28064600F0348108A900250DF10D00D0
:10D7600001F8125D8DF80D5013F02AFE08A800F89C
:10D77000115D13F019FE08A800F8105D13F008FE03
:10D7800008A820F8085D13F0F7FD236820465A1C0E
:10D7900022601E7023689DF80D20591C21601A70AC
:10D7A00023689DF80E20591C21601A7023689DF88B
:10D7B0000F20591C21601A7023689DF81020591CF5
:10D7C00021601A70BDF81810FBF782FFFFF795B9BA
:10D7D0000B680120A14A1E18A149D57826601D704A
:10D7E000236849791D189F4A256019702368D278EB
:10D7F000191821601A70FFF781B90020FFF77EB970
:10D80000236820465A1C226019702988FBF760FFA4
:10D810002368EA78591C21601A7023682A79591CF8
:10D8200021601A702368AA79591C21601A70236834
:10D830006A79591C21601A70FFF764BA0025DFF875
:10D8400054A24FF008080135C5F12002A5F12003CC
:10D85000252D2AFA05F608FA02F228FA03F310D069
:10D8600016431E43002306F001021343EBD0E8B237
:10D8700027F0BEF90028E6D0294606A8FCF76AFA88
:10D88000E1E7794B1B78DA0700F1A1800025774E9C
:10D890002F4602E00135252D0DD029463046FCF7F4
:10D8A00069FA0028F6D0294606A8FCF763FA002892
:10D8B0005ED10137EEE76E4B20466E4DB3F8501047
:10D8C000FBF706FF6C4B2046198889B2FBF700FF77
:10D8D0006A4B204619684A01C1F34003C1F3800E28
:10D8E000C1F3C00602F020021343C1F3401201F05D
:10D8F000100143EA4E0343EA860343EAC203194395
:10D90000FBF7E6FE04A904222046FBF79DFE2368F0
:10D91000297820465E1C5A4A2660197011886429AD
:10D92000A8BF6421FBF7D4FEB9F1960F54D00021B3
:10D930002046FBF7CDFEB7F11903256805A920465F
:10D9400048BFA7F112036E1CA3F3C40326601A4656
:10D950002B70FBF779FE236810214A4A5D1C204694
:10D96000256019701188FBF79DFE0120FFF7C6B8EE
:10D97000394604A8FCF7EEF99BE7F4EEC87AF1EE1D
:10D9800010FA51DA4FF47A71FFF79DBA0B68B1784B
:10D99000581C3D4A2060197023681278591C216078
:10D9A0001A7095E6082770E540F2DC51FFF78BBA54
:10D9B000364D95F82430E3B93346354AFFF70DBBB1
:10D9C000236801201A1822601E70FFF797B8069B83
:10D9D00043F00103069359E723680322591C216091
:10D9E0001A7023686A78591C21601A70A3E704270B
:10D9F0004BE5274A5178022929D003290CBF04237B
:10DA00003346FFF7EABA40F2F312A3F5836302FB51
:10DA100003F38AFB0312D9171344C1EB632101F20C
:10DA2000DD5189B2FFF74FBAFDEEE77A40F2E732F7
:10DA300017EE903A303B02FB03F38BFB0312D9172E
:10DA4000C1EB622101F2E93189B2FFF73CBA042B44
:10DA500034BF02230323FFF7C0BA00BF84BC0120F8
:10DA60001CB8012094BC0120CD69012060BD0120BB
:10DA700044190120EE380120F4630120744F012085
:10DA8000462A0120D8B5012078BC01201CB1012014
:10DA90006C9C012090E33FF40228094B094928BF00
:10DAA000022000EB8002C0EBC20230B4064D441CE1
:10DAB00003EB42032870E0B20B6030BC21F034BEAF
:10DAC00020450120FC380120EE38012008B52AF05D
:10DAD000F3FDFBF787FBBDE808402AF0D5BD00BF8A
:10DAE000434B99895A89914210B501D300225A813A
:10DAF000198ADA89914201D30022DA81DA78072A79
:10DB000018BF002A3B4A3CD092F85B2001213A4CD6
:10DB100000200A2A99702170D8715FD00C2A5BD13D
:10DB2000364CDFED377AA278062A3DD92179DFED30
:10DB3000356A002940D19B782F4A07EE103A1178B8
:10DB4000B8EEC77A27EE277A07EE901AF8EEE77A52
:10DB500067EE877AF4EEE76AF1EE10FA3BDDC6EE87
:10DB6000877AFDEEE77A17EE903A102BA8BF1023C4
:10DB7000012BB8BF0123DBB28B4238BF0B461370B9
:10DB800010BD92F85B200A2A2BD00C2ADA792CD10E
:10DB9000DFED1D7A002A9FED1B7A18BFF0EE477A61
:10DBA000164CA278062AC1D8184901EB8201D1EDA2
:10DBB000176A21790029BED0013A032A0BD8B7EEA3
:10DBC000000A80EE260A33F0A1FC2388984228BF81
:10DBD0001846208010BD10BD0A2AA1D1DFED0C7AB5
:10DBE000DEE7DA79DFED0B7AD4E7DFED0B7AD1E708
:10DBF000A46C0120B86C012078BC0120547701206E
:10DC00006F12833A6F1203380AD7A339E03A040837
:10DC10000F506E3A5304E9386F12033938B50D4C82
:10DC20000D4DAC4206D2616820461434FBF766FA0B
:10DC3000AC42F8D3FCF7ACF8084C094B0022094D74
:10DC400009490A481A705A7025600860BDE83840D2
:10DC50001CF0F2B8E801000884060008FC38012036
:10DC6000EE380120204501204C810120003901209F
:10DC700008B5FFF7D3FF2AF01FFDFBF7B3FABDE8A5
:10DC800008402AF001BD00BF2DE980480A2385B075
:10DC900001308B4D02938B4FC3B28B4C8B4E039351
:10DCA0001FF05EFE4FF4FA7ADFF824924FF0100C6A
:10DCB0004FF47A70D9F80430C3F30803002B40F016
:10DCC000C180EFF31183002B40F0BC802968A2686B
:10DCD00000BF2B689942F9D1D7F800E000FB0EF3A2
:10DCE0009B1AB3FBFEF300FB01314FF0010E0191D3
:10DCF000D9F80430C3F30803002B40F08780EFF31A
:10DD00001183002B40F082802B68A16800BF2A6835
:10DD10009342F9D1D7F800B000FB0BF2521AB2FBD4
:10DD2000FBF200FB0323019A9B1AB3F57A7FDFD342
:10DD3000BAF1010ABED1039B002B40F0BD804FF425
:10DD40007A7ADFF88C914FF0100C5046D9F80430F5
:10DD5000C3F30803002B40F09280EFF31183002BF4
:10DD600040F08D802968A26800BF2B689942F9D1E4
:10DD7000D7F800E000FB0EF39B1AB3FBFEF300FBA9
:10DD800001314FF0010E0191D9F80430C3F30803BB
:10DD900003BBEFF31183EBB92B68A16800BF2A68BE
:10DDA0009342F9D1D7F800B000FB0BF2521AB2FB44
:10DDB000FBF200FB0323019A9B1AB3F57A7FE3D3AE
:10DDC000BAF1010AC2D1029B013B02937FF468AF12
:10DDD000FCF712FDEFF311888CF31288A168236819
:10DDE000DB0302D5C6F800E0A1682B685FFA88F86B
:10DDF000326888F31188D7F800801A4400FB08F3D2
:10DE00005B1AB3FBF8F300FB0233D4E7EFF311889E
:10DE10008CF31288A1682368DB0302D5C6F800E002
:10DE2000A1682B685FFA88F8326888F31188D7F800
:10DE300000801A4400FB08F35B1AB3FBF8F300FB05
:10DE4000023370E7EFF311828CF31288D4F808E004
:10DE50002368D90303D501233360D4F808E02B6885
:10DE6000D2B2316882F311883A68194400FB02F398
:10DE7000A3EB0E03B3FBF2F300FB013135E7EFF345
:10DE800011828CF31288D4F808E02368D90303D5F3
:10DE900001233360D4F808E02B68D2B2316882F3F2
:10DEA00011883A68194400FB02F3A3EB0E03B3FB9D
:10DEB000F2F300FB013164E718461FF0B7FB3EE7C1
:10DEC0002C6401203064012010E000E0286401206F
:10DED00000ED00E02DE9F047B54F2AF0EDFBB54E1F
:10DEE000BE421ED2DFF85883DFF858934446258897
:10DEF00062197DB14A450DD2052D0BD93388618851
:10DF0000C3F30B03994200F0F4801446258862198C
:10DF1000002DEFD1716830461436FBF7EFF8BE42A2
:10DF2000E4D3A54A1378A3F11701022914D9A34910
:10DF300011F83300002800F03181D8000C18646813
:10DF4000002C00F02D810144497829B19C4911F839
:10DF500033300BB9182313709A4C6378022B01D914
:10DF6000002363702378022B00F2E480964B9A78AA
:10DF7000042A00F0E68022B91A88B2F5F07F00F298
:10DF80000981924D924A2B681A40002A00F00B81B9
:10DF9000D80700F1E380590400F1E7801A0700F187
:10DFA000EB809B0400F1EF808A4D2B68998C5A8C92
:10DFB000914201D300225A84FFF792FD23F038FAF0
:10DFC000002800F0C7804FF40070FBF7CDF84FF445
:10DFD0008020FBF7C9F84FF40010FBF7C5F84FF0AD
:10DFE0000070FBF7C1F84FF08060FBF7BDF8637875
:10DFF000022B06D803EB4303774A784902EB8303ED
:10E000000B602378022B07D803EB8301744AC3EB20
:10E01000C10302EB43032B6026F062FE0021302295
:10E02000704835F08EFB286830F0C4FC6E4B2D68CC
:10E0300003F1500102E00433994279D01A78002AA2
:10E04000F9D19C78D8788442F5D268492846684B43
:10E050000A701D6013F028F9664AC82366486421D7
:10E0600015790022654C11FB0531654F654B30F881
:10E07000066C654DA46B596038602E809A60DA603A
:10E080001A615A619A61DA6183F8202083F82120AD
:10E090000CB115F055FF5D4B9FED5D5A1B885D4A35
:10E0A00006EE903A9FED5C6A1388F8EEE66A5579C1
:10E0B00007EE103A53881479C5EE265A07EE903AC7
:10E0C000564B5749574A5848B8EEC77A1D72F8EE72
:10E0D000E77A5C72106027EE067A67EE867ABDE812
:10E0E000F04783ED017AC3ED007AC1ED005A2AF0C2
:10E0F000CBBA63799B077FF408AF7168304694F818
:10E1000004A0FAF7FBFF3388BAEB133F04D01436B0
:10E11000BE42FFF4EBAE04E77388AA1FA11D70682E
:10E12000C3F30B039A42A8BF1A4633F0C1F8EEE7D7
:10E1300001228AE700232370234B9A78042A7FF474
:10E140001AAF9A8AB2F57A7FBFF41BAF4FF47A7296
:10E150009A8216E7354820F029F934E73448FBF76E
:10E1600003F82B6859047FF519AF3248FAF7FCFF22
:10E170002B681A077FF515AF2F48FAF7F5FF2B68C4
:10E180009B047FF511AF2D48FAF7EEFF4020FAF718
:10E19000EBFF09E74FF4F0721A80F2E6D800D2E6FE
:10E1A00017241470CFE643F008032B60F0E600BF9D
:10E1B00084060008E8010008C03F012068650408E3
:10E1C000586E0408EE38012054770120684601207B
:10E1D00009600002FC380120003901204C81012037
:10E1E00020450120CC240120C43F01203319012007
:10E1F00000250120102B01208ABC0120FC4E0120AB
:10E2000038BD0120B4B50120883B0120082701203A
:10E21000C0C9FB482C20012017B7D138C0280120E5
:10E220000C270120E42801203661023DCCCA0120E0
:10E23000086000020920000201600002094000029B
:10E24000024000080080000808B52AF035FAFAF705
:10E25000C9FF2AF019FAFFF73DFE0120BDE808408A
:10E2600021F062BA01302DE9F04FC3B285B08D4C78
:10E2700003930B4602918C4E002B00F099801FF007
:10E280006FFB8A4D4FF4FA7A894FDFF828924FF0EE
:10E29000100C4FF47A70D9F80430C3F30803002B44
:10E2A00040F0DE80EFF31183002B40F0D980296825
:10E2B000A26800BF2B689942F9D1D7F800E000FBB3
:10E2C0000EF39B1AB3FBFEF300FB01314FF0010E7E
:10E2D0000191D9F80430C3F30803002B40F0878084
:10E2E000EFF31183002B40F082802B68A16800BF00
:10E2F0002A689342F9D1D7F800B000FB0BF2521A0A
:10E30000B2FBFBF200FB0323019A9B1AB3F57A7F61
:10E31000DFD3BAF1010ABED1039B002B40F0BD80D0
:10E320004FF47A7ADFF88C914FF0100C5046D9F800
:10E330000430C3F30803002B75D1EFF31183002BD6
:10E3400071D12968A26800BF2B689942F9D1D7F82A
:10E3500000E000FB0EF39B1AB3FBFEF300FB013160
:10E360004FF0010E0191D9F80430C3F3080313BB39
:10E37000EFF31183FBB92B68A16800BF2A689342B1
:10E38000F9D1D7F800B000FB0BF2521AB2FBFBF246
:10E3900000FB0323019A9B1AB3F57A7FE3D3BAF10A
:10E3A000010AC4D1029B013B0293002B7FF467AFAB
:10E3B00005B0BDE8F08FEFF311888CF31288A168E7
:10E3C0002368DB0302D5C6F800E0A1682B685FFA7A
:10E3D00088F8326888F31188D7F800801A4400FB67
:10E3E00008F35B1AB3FBF8F300FB0233D2E7EFF359
:10E3F00011888CF31288A1682368DB0302D5C6F864
:10E4000000E0A1682B685FFA88F8326888F3118809
:10E41000D7F800801A4400FB08F35B1AB3FBF8F34B
:10E4200000FB023370E7EFF311828CF31288D4F80B
:10E4300008E02368D90303D501233360D4F808E04A
:10E440002B68D2B2316882F311883A68194400FB14
:10E4500002F3A3EB0E03B3FBF2F300FB01317FE702
:10E46000EFF311828CF31288D4F808E02368D90303
:10E4700003D501233360D4F808E02B68D2B23168A9
:10E4800082F311883A68194400FB02F3A3EB0E03F0
:10E49000B3FBF2F300FB013118E718461FF0C6F892
:10E4A0003EE700BF10E000E0286401202C6401205A
:10E4B0003064012000ED00E0214B5B68C3F30803EA
:10E4C00010B4C3B9EFF31183ABB91E4B1E4C1868DF
:10E4D000A16800BF1A689042F9D11C4B4FF47A72C0
:10E4E0001C6802FB04F3591AB1FBF4F15DF8044B0C
:10E4F00002FB00107047EFF31182102383F31288A0
:10E5000011498C680B6813F4803F114B02D0012035
:10E5100018608C680B49D2B20968186882F31188B8
:10E520000A4B4FF47A720844196802FB01F31B1B73
:10E530005DF8044BB3FBF1F302FB0030704700BF02
:10E5400000ED00E02C64012010E000E030640120C8
:10E55000286401202DE9F84F80461027FFF7ACFF13
:10E56000244E844624494FF47A74DFF898E0012061
:10E57000224A234DDEF80430C3F30803D3B9EFF386
:10E580001183BBB90B68D2F808A000BFD1F8009086
:10E590004B45F7D1D6F800B004FB0BF9A9EB0A09FB
:10E5A000B9FBFBF904FB0393A3EB0C034345E1D355
:10E5B000BDE8F88FEFF3118A87F31288D2F808B01C
:10E5C0001368DB0302D52860D2F808B00B685FFA45
:10E5D0008AFAD5F800908AF31188D6F800A09944F9
:10E5E00004FB0AF3A3EB0B03B3FBFAF304FB0933BD
:10E5F000DAE700BF306401202C64012010E000E065
:10E600002864012000ED00E02DE9F04FDFF830C173
:10E6100080461027464A4749474E484D18F1FF3873
:10E62000C0F08480DCF80430C3F30803002B5CD115
:10E63000EFF31183002B58D10B68946800BF086872
:10E640008342F9D1D6F800904FF47A7000FB09FEAE
:10E65000AEEB040EBEFBF9FE00FB03EEDCF804306B
:10E660004FF47A740120C3F30803FBB9EFF311836D
:10E67000E3B90B68D2F808A000BFD1F800904B4571
:10E68000F7D1D6F800B004FB0BF9A9EB0A09B9FBE6
:10E69000FBF904FB0393A3EB0E03B3F57A7FBDD222
:10E6A000DCF80430C3F30803002BDFD0EFF3118A4A
:10E6B00087F31288D2F808B01368DB0302D528600C
:10E6C000D2F808B00B685FFA8AFAD5F800908AF39E
:10E6D0001188D6F800A0994404FB0AF3A3EB0B03BE
:10E6E000B3FBFAF304FB0933D5E7EFF3118487F3A7
:10E6F0001288D2F808901368D80303D501232B6041
:10E70000D2F808900B68E4B2286884F311884FF4BB
:10E710007A74D6F800A000EB030E04FB0AF3A3EB17
:10E720000903B3FBFAF304FB0E3E97E7BDE8F08F55
:10E7300010E000E02C6401203064012028640120F6
:10E7400000ED00E030B4EFF31183102282F3128861
:10E7500008490025084CDBB20A68084801320A6003
:10E760002560026883F31188054A1368013330BCC1
:10E77000136070472C6401202864012010E000E041
:10E780007062012003685B6A03B11847704700BFDD
:10E7900003681B6A03B11847704700BF03682DE97F
:10E7A000F041DF691FB13B46BDE8F0411847002A40
:10E7B000164611DD04460D460E4400E023689B68B2
:10E7C000204698470028F9D02368204615F8011BF9
:10E7D0001B689847AE42F1D1BDE8F08103689B69A0
:10E7E000184700BF03685B69184700BF03681B69CF
:10E7F000184700BF0368DB68184700BF03689B68C1
:10E80000184700BF03685B68184700BF03681B68B0
:10E81000184700BF38B50C46097849B105460134A0
:10E820002B6828461B68984714F8011B0029F7D16C
:10E8300038BD00BF054B53F8203033B11A689B88B0
:10E8400051690B4218BF1B0493617047F8630120A4
:10E850002DE9F04FC1F3810383B0D0F800E001F05F
:10E8600003088788C1F3411B009397FAA7F6B6FA0D
:10E8700086F608F1FF3A37FA06F363D04FF0010944
:10E880004FF0030C019103E0013637FA06F358D03C
:10E8900009FA06F33B40F7D0DEF8005093FAA3F4F0
:10E8A000B4FA84F493FAA3F0B0FA80F06400BAF1F9
:10E8B000010F4FEA40000CFA04F408FA00F025EAD0
:10E8C000040440EA0400CEF800004CD9DEF80C50F5
:10E8D00093FAA3F4B4FA84F493FAA3F0B0FA80F0B4
:10E8E0006400B8F1020F4FEA40000CFA04F40BFA8E
:10E8F00000F025EA040440EA0400CEF80C00C3D17D
:10E9000093FAA3F0B0FA80F01C0A072842DCDEF884
:10E91000204093FAA3F0B0FA80F093FAA3F30F210A
:10E92000B3FA83F3800001369B0001FA00F002FA8B
:10E9300003F324EA00000343CEF8203037FA06F34D
:10E94000A6D10199BAF1010F0AD8DEF80430C1F35B
:10E95000001107FB01F123EA07070F43CEF804700B
:10E9600003B0BDE8F08FDEF8085093FAA3F4B4FAD0
:10E9700084F493FAA3F0B0FA80F0640000994000A8
:10E980000CFA04F401FA00F025EA04042043CEF85E
:10E9900008009BE7DEF8240094FAA4F3B3FA83F3AB
:10E9A00094FAA4F40F21B4FA84F49B00A40001FAB1
:10E9B00003F302FA04F420EA03032343CEF82430DD
:10E9C00062E700BF10B50409013C032C17D80D4BBA
:10E9D00000F00F0033F8142042FA00F313F00103A3
:10E9E0000DD0012303FA00F00138104031F0B0FFE0
:10E9F000054A064B125D104403EBC00010BD002019
:10EA000010BD00BF646304086C6304081C6B012024
:10EA10002DE9F04F4C484FF0010A4C494FF00209E4
:10EA20004B4B4FF004084FF0080C4FF0100E20270E
:10EA300040268025474C30F8022B12F0010F03D0FE
:10EA40001960083323F804AC12F0020F03D01960E8
:10EA5000083323F8049C12F0040F03D01960083324
:10EA600023F8048C12F0080F03D01960083323F840
:10EA700004CC12F0100F03D01960083323F804EC13
:10EA800012F0200F03D01960083323F8047C12F031
:10EA9000400F03D01960083323F8046C12F0800F84
:10EAA00003D01960083323F8045C12F4807F05D08A
:10EAB0004FF4807B1960083323F804BC12F4007F04
:10EAC00005D04FF4007B1960083323F804BC12F41E
:10EAD000806F05D04FF4806B1960083323F804BCB5
:10EAE00012F4006F05D04FF4006B1960083323F85F
:10EAF00004BC12F4805F05D04FF4805B19600833CA
:10EB000023F804BC12F4005F05D04FF4005B1960D9
:10EB1000083323F804BC12F4804F05D04FF4804B27
:10EB20001960083323F804BCD20B05D04FF400421F
:10EB30001960083323F8042C01F58061A1427FF4A9
:10EB40007AAFBDE8F08F00BF6463040800000240A4
:10EB50001C6B01200010024000B179E6704700BF35
:10EB600008B1002274E6704718B1838802681B045C
:10EB70009361704710B1036882889A61704700BF43
:10EB800038B100298388026814BF002110218B400E
:10EB900093617047104B01461B883BB90F4B104ADD
:10EBA0001B7810680BB981F00101E9E70D4B5A6938
:10EBB00082B118B91A681060587470470A48012168
:10EBC0000A4A10B40488186892FBF4F25DF8044B0A
:10EBD00002605974704700BF04640120066401207C
:10EBE000086401200C6401202464012020A1070096
:10EBF00001230A4A10B48340094C127854F82000CB
:10EC0000134029B9B3FA83F15DF8044B4909B7E71A
:10EC1000191C5DF8044B18BF0121B1E7F663012010
:10EC2000F863012008B501210220FFF7E1FF094B3D
:10EC30001B7803F00503052B08D000210120FFF706
:10EC4000D7FF00210846FFF7D3FFFEE711F09CF93C
:10EC5000F3E700BFA861012030B1036882881B6917
:10EC60001A4214BF01200020704700BF2DE9F04177
:10EC70000B4E356873691D400FD0DFF828800127DF
:10EC8000B5FA85F4C4F11F0458F8240007FA04F417
:10EC900003689847A5437461F2D1BDE8F08100BFD5
:10ECA000003C0140346401202DE9F0410B4E3568F1
:10ECB00073691D400FD0DFF828800127B5FA85F46D
:10ECC000C4F11F0458F8240007FA04F403689847B5
:10ECD000A5437461F2D1BDE8F08100BF003C014062
:10ECE000346401202DE9F0410B4E356873691D40F5
:10ECF0000FD0DFF828800127B5FA85F4C4F11F048E
:10ED000058F8240007FA04F403689847A54374618F
:10ED1000F2D1BDE8F08100BF003C01403464012025
:10ED20002DE9F0410B4E356873691D400FD0DFF8B7
:10ED300028800127B5FA85F4C4F11F0458F824008F
:10ED400007FA04F403689847A5437461F2D1BDE85B
:10ED5000F08100BF003C0140346401202DE9F04106
:10ED60000B4E356873691D400FD0DFF828800127EE
:10ED7000B5FA85F4C4F11F0458F8240007FA04F426
:10ED800003689847A5437461F2D1BDE8F08100BFE4
:10ED9000003C0140346401202DE9F0410B4E356800
:10EDA00073691D400FD0DFF828800127B5FA85F47C
:10EDB000C4F11F0458F8240007FA04F403689847C4
:10EDC000A5437461F2D1BDE8F08100BF003C014071
:10EDD000346401202DE9F0410B4E356873691D4004
:10EDE0000FD0DFF828800127B5FA85F4C4F11F049D
:10EDF00058F8240007FA04F403689847A54374619F
:10EE0000F2D1BDE8F08100BF003C01403464012034
:10EE100003685B6A184700BF2DE9F0410D460446C0
:10EE200018461646984631F099F828442768E67245
:10EE30002946A07243467D6932462046AC46BDE86D
:10EE4000F0416047036810B504461B689847236883
:10EE500020469B689847A37B0133A37310BD00BF76
:10EE6000036810B59B68044698470122FF2322736C
:10EE7000637310BD08B5FFF7A5FD38B12C22202122
:10EE800082710022C271BDE8084069E608BD00BF7A
:10EE9000427A02B97047036800F10A0110B50446CE
:10EEA000406898470023637210BD00BF437A5A1C24
:10EEB0000344D2B242729972037A93420AD84AB199
:10EEC000036800F10A0110B5044640689847002322
:10EED000637210BD704700BF302826D0312826D07D
:10EEE000322826D0332826D0342826D0352826D0DC
:10EEF000202826D0212826D0102826D0112826D038
:10EF0000122826D0132826D0142826D0152826D03B
:10EF1000162826D0172801D0002070470F22124B48
:10EF200003EB420393F8790070470022F7E70122D0
:10EF3000F5E70222F3E70322F1E70422EFE70522D7
:10EF4000EDE70622EBE70722E9E70822E7E70922D7
:10EF5000E5E70A22E3E70B22E1E70C22DFE70D22D7
:10EF6000DDE70E22DBE700BFE03A04082DE9F04FB1
:10EF70002DED028B93B0804628F0C4F98D4B1D789F
:10EF800025B113B0BDEC028BBDE8F08F8A4B1B6836
:10EF90005805F6D5894BDFF880B21B686BB1884AFB
:10EFA000DBF800101368CB1A7C2B06D9854811605A
:10EFB0000378013303701CF075F9834B1B78002B29
:10EFC0006DD0824C824AD4F81031A8EB03039342EF
:10EFD00001F2F08294F81891B9F1000F32D17D4F0F
:10EFE0003868FFF70FFCC0B201280FD9022841F0A2
:10EFF000D587794E3378002B42F01981D4F81C3133
:10F00000A8EB0303B3F57A6F82F0E282D4F82031E3
:10F01000002B44D094F81831BBB9704B0121002269
:10F020001B6884F818119B7884F82C211E3B8B42B6
:10F0300042F286823868022104301CF0E7F894F826
:10F04000243110E0D4F820314BB3D4F8283140F605
:10F05000B732A8EB0303934221D994F82431002B53
:10F0600001F09D865B4F013BDBB284F82431002B1D
:10F0700001F0CF83D4F8206194F82C2116F8011BFD
:10F0800094F82D310A4438680133C4F8206184F8BB
:10F090002C2184F82D31FFF7B9FBC4F82881504B9F
:10F0A000DBF800601B7843B14E4F386828B14E4BF7
:10F0B0001B78013B012B41F2BB834C4B1B786BB19E
:10F0C0004B4F3B6853B1DBF80030404C1A4602937B
:10F0D000D4F84431D31A632B00F2E880454F3B78D3
:10F0E000022B01F03C863C4E96F87430032B01F065
:10F0F0007B83414B1B7873B1404D2B685BB1334C24
:10F10000FFF7DAF944F61F620290D4F85031C31ABF
:10F11000934200F2AF813A4B1B78002B7ED1394BE2
:10F120001B783BB1294C384BD4F8A02213449845A6
:10F1300081F0FE81354B1B78002B3FF422AF234E2C
:10F14000334C06F2C127334D2068FFF75BFB0028E4
:10F150003FF417AF2068FFF74DFB2B7880465A1E0F
:10F1600033B120682A70FFF74DFB0028F2D108E781
:10F1700003223946781E34F0CAFA96F8C0124FF6C8
:10F18000FF7396F8C12286F8C3821FFA88F84B40B5
:10F190009B1A9BB2B8EB132FD6D1DBB296F8C222E2
:10F1A0009A42D1D1781E1BF03FFD2B78184428706D
:10F1B000CAE700BFD44B0120B4740120DC4C01200D
:10F1C000504F01204C4F012076B601203C200120F9
:10F1D0003F0D0300F44E012018000120F84E0120DD
:10F1E00078B60120E44C012080B6012088B60120C9
:10F1F000EC4E01209AB9012090B6012094B601206E
:10F2000000B7012011B70120A08601009AB60120A5
:10F21000A0B60120A4B601202C640120814C2278E4
:10F22000A2B1814B9B7A53B1FFF746F97F4B1B6824
:10F23000C31AA3F57A73B3F5FA6F07D822787C4B1B
:10F240007C491868FFF7AAFA002323707A4C7B4B9D
:10F25000D4F8982213449845FFF461AF784DC4F870
:10F2600098822B78002B41F0D786764D2B78002B97
:10F2700041F02D86744994F89C228D5CE80702F1D8
:10F280003D80A90701F1D9876A0701F19D872A0707
:10F2900001F14A8794F89C326C4A0133117893FB50
:10F2A000F1F201FB123384F89C3238E7684E4120BA
:10F2B0001BF056FFDFF8B4A1B6F90230DFF8B091C9
:10F2C0008AFB0320DB17C3EBA00080B21BF02CFFEE
:10F2D000B6F900308AFB0320DB17C3EBA00080B235
:10F2E0001BF022FFB6F904308AFB0320DB17C3EBC7
:10F2F000A00080B21BF018FF99F800103868FFF7E3
:10F3000085FA94F848A11AF0010601F07585514B71
:10F3100004931B689B0673D54F4B1B78980742F1EB
:10F320000A814E4E337D042B8CBF4FF0030A4FF001
:10F33000020A47201BF014FF30681BF0BDFE706806
:10F340001BF0BAFE464AF3893868A2FB0323C3F3D5
:10F35000471319460393FFF759FA049B99F80010D5
:10F360001A68039B12F0140F83EA010389F8003036
:10F3700041F023873389642000FB03F01BF09CFEDF
:10F38000367D38684AEA8606F6B23146FFF73EFA1D
:10F3900099F8003038685E40314689F80060FFF720
:10F3A00035FA94F848A1BAF1000F29D12D4E4F201B
:10F3B0001BF0D6FE30681BF07FFE70681BF07CFEF1
:10F3C00050461BF079FE01213868FFF71FFA224AE8
:10F3D00099F80030167883F00103386806F00106CA
:10F3E00089F800303146FFF711FA99F80030386893
:10F3F0005E40314689F80060FFF708FA94F848A1AA
:10F400000AF101030299184ADBB2C4F84411A2FBC5
:10F410000312D20802EB8202A3EB420384F84831C4
:10F420005CE600BF68B601200C77012050B90120CE
:10F4300004B7012028B601203C200120A08601004D
:10F4400008B7012009B701200CB7012010B701202F
:10F45000584F0120744F0120784F01207C4F01202C
:10F460001F85EB510C490120CDCCCCCC676666667C
:10F47000F04E012094F85631002B41F0B884D34A65
:10F480004AF60B4748F603404BF60F43126849F61D
:10F49000074602F0080100294FF0190104BF3B465E
:10F4A000064612F0040F84F8561118BF1E46910646
:10F4B00003D546F4804646F02006C6F30902C44B45
:10F4C00003925A79002A42F0D7809B79002B42F0B0
:10F4D000AC80994664204FF0FF3A03990023012243
:10F4E0000AAF0C91FE210A964FF01F0E0B96ADF855
:10F4F0003690ADF838A08DF84600ADF83430CDF830
:10F500003A30CDF83E30CDF842306371E271A170EF
:10F51000B04E84F803E00FCF0FC697E80F0007C680
:10F520001A0C26F8023BC8233146701C01F81E292C
:10F53000A37194F8662182F0F103561C227183EACC
:10F54000031384F86661DAB2130983F0E70343EA30
:10F55000022383EAC2031BB283EA0312C3F3072325
:10F56000D2B283EA121343EA022383EAC2031BB234
:10F5700083F0C802C3F3072382EA0212D2B283EAFD
:10F58000121343EA022383EAC2031BB283F001068B
:10F59000C3F3072286EA0613DBB282EA131242EAB9
:10F5A000032282EAC3021646228011F8013B73400F
:10F5B000814283EA0313DBB24FEA131282EA162276
:10F5C00042EA032282EAC3031BB29EB22680ECD138
:10F5D00083F07C03804F04F1220A83EA031307F5CA
:10F5E000C77CDBB24FEA131E8EEA162E8EEA032E7C
:10F5F0008EEAC30E0FFA8EFE1FFA8EF35FFA8EFEAE
:10F600004FEA1329238084F827E084F8289038688B
:10F61000103757F80C1C664657F8082C0CF1100CE4
:10F6200057F8043C57450FC6F1D138686B4ECCF8FB
:10F6300000003B7906F127078CF8043084F8B5E127
:10F6400084F8B69116F8011F2868FFF7DFF8B74273
:10F65000F8D194F85711002941F0BF83604B0A227A
:10F66000DBF800901B7884F85721002B01F04885C7
:10F670005C4A012B168842F2F180022BB2F802E0BC
:10F6800002F011809088032B049002F0F780042B85
:10F69000B2F806C002F0FF801089052B039002F03B
:10F6A000F680062BB2F80AA002F0E080072B9089C2
:10F6B00000D0D189002794F86621CDF828904FF02A
:10F6C000000966F30F07484E82F030032271368836
:10F6D0006EF31F4783EA0313DFF810E1C6EB06263B
:10F6E0000B97DBB201328EFB067E049F84F8662105
:10F6F00067F30F091F09B644F61787F07A076CF312
:10F700001F494FF0000CC6EB6E2647EA0327CDF8E1
:10F710003090E6468DF83D6087EAC303039F60F3AF
:10F720000F0E00201BB267F30F0C61F31F4E0AAFE0
:10F7300083EA0311C3F30723CDF838E04FF0C80E76
:10F74000C9B26AF31F4C4FF0230A84F806E083EA3B
:10F750001113CDF834C04FF0160C8DF83C0043EA7D
:10F7600001231C4E84F803C04FF0FE0983EAC10355
:10F77000607184F807A01BB284F8029083EA0E023D
:10F78000C3F3072382EA0211C9B283EA111242EAE3
:10F79000012282EAC10212B282EA0A03C2F3072EF0
:10F7A00083EA031C5FFA8CFC0FCF8EEA1C1E0FC687
:10F7B0004EEA0C2397E8030083EACC0346F8040BD7
:10F7C000B01C26F814191946238011E0744F01204B
:10F7D000604F0120442001203E200120CB21012048
:10F7E00024390120C8B20120A8B5012003082080D7
:10F7F00016F8012B4A40864282EA0212D2B24FEA40
:10F80000121383EA112343EA022383EAC20212B2EB
:10F8100091B22180ECD182F0F402DFF8D49304F2AB
:10F820008F1604F2AD1782EA0212D9F8000009F52A
:10F83000C77CD2B24FEA121E8EEA112E8EEA022E39
:10F840008EEAC20E0FFA8EFE1FFA8EF35FFA8EFE5C
:10F850004FEA132A238084F81EE084F81FA0D9F809
:10F860000410D9F80820D9F80C30ACE80F00D9F80A
:10F870001000D9F81410D9F81820ACE8070084F863
:10F88000ADA184F8ACE116F8011F2868FEF7BEFFB1
:10F89000B742F8D194F85A31002B41F0A382D04BF3
:10F8A000192204931B6884F85A219A0640F1F882C1
:10F8B000CC4B1B789B0741F1B386CB4E337D042B99
:10F8C0008CBF4FF003094FF00209FEF7F5FD338AB4
:10F8D00032894FF47A7103EB83030A900AAF01FB7C
:10F8E00002F230685B000E92BE46ADF842304FF037
:10F8F000000C0C904FF0FF31F3894FF01E0A327D5F
:10F9000070688DF844904FF018090D90ADF84030B4
:10F910008DF84520CDF82CC00F910397B34FBEE86A
:10F920000F000FC79EE80F0007C7BA1C27F81C3945
:10F9300094F86601FE21C82384F8079080F0780EC1
:10F94000A170A3718EEA0E1E2071013084F805C0EB
:10F950005FFA8EF184F803A084F866010B0983F046
:10F96000F60343EA012383EAC1031BB283EA0311CE
:10F97000C3F30723C9B283EA111343EA012383EADD
:10F98000C1031BB283F0C801C3F3072381EA01104E
:10F99000C0B283EA101141EA002181EAC00109B234
:10F9A00081EA0900C1F3072380EA0011C9B283EAA2
:10F9B000111343EA012383EAC1031846238017F891
:10F9C000011B4140974281EA0111C9B24FEA11136C
:10F9D00083EA102343EA012383EAC10109B288B212
:10F9E0002080ECD181F01801814A04F1220981EADA
:10F9F00001110592174602F5C77CC9B24FEA111AE8
:10FA00008AEA102383EA012A8AEAC1010FFA81FAFD
:10FA10001FFA8AF35FFA8AF2190A23800692079185
:10FA200084F8262084F827103868103757F80C1C03
:10FA3000E64657F8082C0CF1100C57F8043C4F45DB
:10FA4000AEE80F00F0D13868DFF8B091CCF80000D4
:10FA50009DF8183009F12607CA4684F8B4319DF89C
:10FA60001C3084F8B5311AF8011F2868FEF7CEFE65
:10FA70005745F8D1FEF720FD049B32894FF47A7187
:10FA80001B68D6F800C001FB02F113F0140F766872
:10FA900041F08F850F4694F866A14FF0000E0D914E
:10FAA0008AF06A03534A0A9083EA0313B2F90420E6
:10FAB0005148DBB20C96D61780FB02021909ADF84B
:10FAC0003CE0C6EBA202212681F0D501ADF83EE074
:10FAD000ADF842200AF1010041EA0321ADF840E00F
:10FAE00084F805E081EAC303FE21E6711BB2A17030
:10FAF0001C21CDF82CC083EA0312C3F30723E17065
:10FB0000C821D2B2DDF80CC0A17183EA12130E979E
:10FB100084F8660143EA0223344F84F804A083EAA0
:10FB2000C2031BB283EA0102C3F3072382EA021174
:10FB3000C9B283EA111242EA012282EAC10212B278
:10FB400082EA0603C2F3072683EA031E5FFA8EFEEB
:10FB500086EA1E16BCE80F0046EA0E260FC786EAA4
:10FB6000CE0307F10C0EA7F110069CE8070087E80A
:10FB700007001946238016F8012B4A40764582EA91
:10FB80000212D2B24FEA121383EA112343EA02238C
:10FB900083EAC20212B291B22180ECD182F06802F3
:10FBA0000B46134E04F1220182EA021206F5C77ECB
:10FBB0000491D2B24FEA121C8CEA132383EA022C7E
:10FBC0008CEAC2020FFA82FC1FFA8CF35FFA8CFCFB
:10FBD0004FEA132A238084F824C084F825A00FE07C
:10FBE000744F0120784F01207C4F012044200120D8
:10FBF0003E200120584F012067666666CB21012018
:10FC0000F36877463068103656F80C1C0EF1100E6B
:10FC100056F8082C0FC7049B9E42F1D133884F46FB
:10FC2000DB4EAEF8003084F8B2C184F8B3A117F807
:10FC3000011F2868FEF7EAFDBE42F8D194F866116C
:10FC40000023D44F312681F0EB020C936371FE2028
:10FC500082EA02127B6821710131D2B20B9384F8DF
:10FC60006611C8211309E6713F6883F0C503A070CF
:10FC70000A970C2743EA0223A171E77083EAC203C3
:10FC8000C54F1BB283EA0312C3F30723D2B283EA40
:10FC9000121343EA022383EAC2031BB283EA01027E
:10FCA000C3F3072382EA0212D2B283EA121343EAB1
:10FCB000022383EAC203039A1BB25E40C3F3072305
:10FCC00086EA0616F6B283EA161343EA062307CA43
:10FCD00083EAC603A7F5C4761BB286E80700267A36
:10FCE000607A5E40C3F30723A17A86EA0616E27AB9
:10FCF00094F80CE0F6B294F80DC094F80EA083EAE4
:10FD0000161343EA062383EAC603E67B1BB2584078
:10FD1000C3F3072380EA0010C0B283EA101343EA5A
:10FD2000002383EAC003207C1BB25940C3F307239E
:10FD300081EA0111C9B283EA111343EA012383EA7C
:10FD4000C103617C1BB25A40C3F3072382EA02124B
:10FD5000D2B283EA121343EA022383EAC203A27CEB
:10FD60001BB28EEA030EC3F307238EEA0E1E5FFA60
:10FD70008EFE83EA1E1343EA0E2383EACE0394F831
:10FD800013E01BB28CEA030CC3F307238CEA0C1CB0
:10FD90005FFA8CFC83EA1C1343EA0C2383EACC034E
:10FDA0001BB28AEA030AC3F307238AEA0A1A5FFA34
:10FDB0008AFA83EA1A1343EA0A2383EACA031BB2C4
:10FDC0005E40C3F3072386EA0616F6B283EA1613EB
:10FDD00043EA062383EAC6031BB25840C3F3072352
:10FDE00080EA0010C0B283EA101343EA002383EADA
:10FDF000C0031BB25940C3F3072381EA0111C9B202
:10FE000083EA111343EA012383EAC1031BB25A4078
:10FE1000C3F3072382EA0212D2B283EA121343EA3F
:10FE2000022383EAC2031BB28EEA030EC3F3072345
:10FE30008EEA0E1E5FFA8EFE83EA1E1343EA0E233D
:10FE400083EACE031BB283F02706C3F3072386EAB7
:10FE50000612D2B283EA121646EA022686EAC206E1
:10FE600036B2B3B25FFA86FA23804FEA132E059EAC
:10FE700084F814A084F815E030687168B268F368FB
:10FE8000B6F810C00FC727F803CB84F8A3E184F8B5
:10FE9000A2A119F8011F2868FEF7B8FC4F45F8D158
:10FEA00094F85E21002A41F00D803C4E052094F824
:10FEB00066C10DF1280EB6F90270B6F900108CF08B
:10FEC0006A0362711E2206EE901A794283EA0313D6
:10FED000E27107EE901AB6F90410FE22DBF800601A
:10FEE00007EE101AD9B2A2701C220B090A96E27012
:10FEF000C82283F0D503F8EEE66AA271F8EEE77A3D
:10FF000043EA0123B8EEC77A9FED256A002783EA0A
:10FF1000C10384F85E0166EE866A0E971BB267EE37
:10FF2000867A27EE067A0F9783EA0311C3F3072335
:10FF300010970CF10109C9B2CDED0B6ACDED0C7A29
:10FF400083EA11138DED0D7A164F43EA012383EAFC
:10FF5000C1031BB25A40C3F3072382EA0212D2B292
:10FF600083EA121343EA022383EAC2031BB283F03B
:10FF70001E06C3F3072386EA061A5FFA8AFA83EAA3
:10FF80001A16BEE80F0046EA0A260FC70CE000BFAB
:10FF9000EF2101200C490120CC210120584F0120E4
:10FFA00088C3E43A4420012086EACA06A7F1100378
:10FFB0009EE8070007F10C0E87E8070084F804C0EC
:10FFC000268084F8669113F8012B7240734582EA0B
:10FFD0000212D2B24FEA121181EA162141EA02213D
:10FFE00081EAC20212B296B22680ECD182F02702D8
:10FFF000DD4F04F1220A82EA021207F5C77CD2B271
:020000040801F1
:100000004FEA121E8EEA162E8EEA022E8EEAC20EDB
:100010000FFA8EFE1FFA8EF35FFA8EFE4FEA132957
:10002000238084F824E084F825903868103757F846
:100030000C1C664657F8082C0CF1100C57F8043CC1
:1000400057450FC6F1D1C94E3B8806F12407ACF8DD
:10005000003084F8B2E184F8B39116F8011F2868E3
:10006000FEF7D4FBB742F8D194F85FA1BAF1000FC4
:1000700040F02287BE4B05221B6884F85F219F0653
:1000800041F14880BB4A13F0140FDFEDBB7AD189F0
:1000900007EE101AB8EEC77A27EE277A01F01F8311
:1000A000B64BDFEDB56AD3ED007AF8EEE77A67EE8E
:1000B000A67A94F866610AABB14A4FF0640E86F0F6
:1000C00022011F46B2F9062081EA01110393B2F51D
:1000D000FA6FAC4BC9B2DFF8C4C2A8BF4FF4FA62E2
:1000E000B3F904000B092671B2F57A7F06F1010617
:1000F00083F059038DED0B7AB8BF4FF47A7284F810
:10010000666143EA0123CDED0C7AA2F57A7283EAA7
:10011000C1030EFB02F2DFF888E21BB28CFB026C1B
:10012000D2178EFB001E0021C2EBAC12964E83EA62
:10013000031CC3F30723ADF83A204A225FFA8CFC74
:100140000A91E271FE2283EA1C130D91A27014221F
:1001500043EA0C23C821E270002283EACC03A17198
:100160006271C0171BB2C0EBAE0083EA0102C3F399
:100170000723ADF8380082EA0212D2B283EA1213E2
:1001800043EA022383EAC2031BB283F04A0EC3F39D
:1001900007238EEA0E1C5FFA8CFC83EA1C1E0FCF2D
:1001A0004EEA0C2E3F688EEACC0E0FC6A4F800E093
:1001B000321D46F8107916F8013B83EA0E03964289
:1001C00083EA0313DBB24FEA131181EA1E2141EAED
:1001D000032181EAC3031BB21FFA83FEA4F800E0E7
:1001E000E9D183F01403604A04F2AB1983EA0313E4
:1001F0001146059204F28F12DBB20868164601F52B
:10020000C77C1A093746049682EA1E2E0E468EEAED
:10021000032E8EEAC30E0FFA8EFE1FFA8EF35FFADC
:100220008EFE4FEA132B238084F81CE084F81DB067
:10023000F3684968B268ACE80F0030697169338BC4
:100240003E46ACE80300ACF8003084F8ABB184F86B
:10025000AAE117F8011F2868FEF7D8FAB945F8D1C6
:100260004A4B4B4A1B781278013B049612F001016D
:10027000DBB214BF4FF0C00E4FF0400E172B03D867
:10028000444A134493F830A0434B1B889E0700F068
:1002900098874EF0100E002213F4027F18BF02223E
:1002A00013F0100F18BF062213F0200F18BF1022F2
:1002B000002941F08581032794F8660103230A92FF
:1002C000002180F046028DF8303000F101092071E4
:1002D00082EA0212C8208DF82EE04FF0090ED2B249
:1002E0008DF82CA084F803E04FF0FE0C13098DF874
:1002F0002F708DF82D1083F09203E171617143EA44
:100300000223A071204F83EAC20384F802C084F85C
:1003100066911BB283EA0312C3F30723D2B283EAC6
:10032000121343EA022383EAC2031BB283EA0002E8
:10033000C3F3072382EA0212D2B283EA121343EA1A
:10034000022383EAC203039A1BB283EA031EC3F3A8
:1003500007235FFA8EFE83EA1E1343EA0E2307CAC1
:1003600083EACE031EE000BF3E200120CB21012006
:10037000744F01207C4F01200AD7233C544F0120A9
:10038000C8B20120584F012044200120C03F012065
:10039000CD690120783B0408AAB50120D34D621035
:1003A0006766666603C71BB294F808C0607A07F5F3
:1003B000C07E8CEA030CC3F30723A17A07F5C87942
:1003C0008CEA0C1C3A70E27A5FFA8CFC94F80CA070
:1003D00094F80DB083EA1C13A67B277C43EA0C2318
:1003E00083EACC0394F80FC01BB25840C3F3072331
:1003F00080EA0010C0B283EA101343EA002383EAC4
:10040000C0031BB25940C3F3072381EA0111C9B2EB
:1004100083EA111343EA012383EAC1031BB25A4062
:10042000C3F3072382EA0212D2B283EA121343EA29
:10043000022383EAC2031BB28AEA030AC3F3072337
:100440008AEA0A1A5FFA8AFA83EA1A1343EA0A2343
:1004500083EACA031BB28BEA030BC3F307238BEABD
:100460000B1B5FFA8BFB83EA1B1343EA0B2383EA24
:10047000CB031BB286EA0302C3F3072382EA02120C
:10048000D2B283EA121343EA022383EAC2031BB205
:100490008CEA030CC3F307238CEA0C1C5FFA8CFC78
:1004A00083EA1C1343EA0C2383EACC031BB287EADA
:1004B0000302C3F3072382EA0212D2B283EA1213C1
:1004C00043EA022383EAC2031BB283F03202C3F37E
:1004D000072382EA0212D2B283EA121343EA02230A
:1004E00083EAC2031BB29AB2DBB24FEA122C22801B
:1004F000637484F812C0059E30687168B268B6F8FB
:100500000CA0049EAEE807008EF80270AEF800A0C2
:1005100084F8A0C184F89F3116F8011F2868FEF7FF
:1005200075F9B145F8D1029BC4F85031FEF7F3BD1F
:1005300094F8A432C14AC4F8A08202EB8302926C00
:100540005AB312AD04F2AB2104F2BD234FF0000EFA
:1005500045F8201DA5268021B94F0B931523284669
:10056000A7F800E084F8AA3284F8A86204F52A7695
:1005700084F8A912904728463988F9F7A9F80A9D06
:100580003146B048AD1B152DA8BF15252A4630F0C1
:100590008FFEAD4A94F8A43215700133AB4A82FB4A
:1005A0000312A2EBE37202EB42029B1A84F8A4321C
:1005B000FEF7C0BDA64A4FF47A71A64B0027D07A49
:1005C000DBF8006001FB00F1D4F814011B88301A3D
:1005D000A14A5FFA83FE88424FEA132382F81EE0A5
:1005E000D37782F814E053759770177180F079848F
:1005F0009A4B47F2305EDFF894C21B6898498CFB37
:100600000306DB170F68C3EB6613964E4FEAE779D4
:10061000896886FB07A7944803F5FA7386FB01A651
:10062000C9EBA70700689BB2C91717773F129376EB
:10063000C1EBA6018CFB00691B0A5777C6178B4FCD
:100640008644D376C6EB691982F820100B12884EC7
:10065000397830304FEA2E2E09F1780982F82130AE
:100660008907377D834B82F8249082F823E082F853
:1006700022009F7640F132847068052F3268029024
:10068000029F4FEAE2707C49039281FB02E2BE4680
:10069000DFF8FC91C0EBA25081FB0EE14FEAE77E50
:1006A000039F764ACEEBA15109FB007E029F00EB2F
:1006B00080000EEB4E0E09FB017701EB810A4FEA39
:1006C0004E0E07EB470782FB0E9100EB80004FEACE
:1006D000470704914FEAEE7982FB071204990590CF
:1006E0000AEB8A0A4FEAA242F0894FEAA141CDF80B
:1006F00018A0049200EBC0003289A1EB0906DFF8D4
:1007000094A14FEAE77902F5FA72314676B2079280
:100710004FEA8000059A0AFB11E106EB8206049A73
:10072000A2EB090E1FFA86F9554E72460AFB1E7E91
:10073000069F52B2BDF81CA083F80A9002EB870214
:10074000049286FB00264FEAE0708CFB01274FEAFB
:10075000E171C0EBA61034BF322633268CFB0E2C81
:10076000BDF810204FEAEE7E0496C1EB6711039EA0
:10077000CEEB6C1EDFF820C1F60FDA73BCF800C0B8
:10078000120A0396029EADF814C04FEA192C3D4F91
:100790004FEAD6799DF80C603F885E72C0F3072659
:1007A00083F80BC04FEA212C1A744FEA1A2283F8FF
:1007B0000E904FEA2E299A759DF810201973390A68
:1007C000DA769DF8142083F80DC083F811E083F8E1
:1007D000129083F815A0D8711E72DF7419751A77FC
:1007E000C4F81081FEF7F6BBDFF8B090D9F800002E
:1007F000FDF7F8FF00283EF47CACD9F80000012199
:10080000FDF7ECFF0222002386F874203B70FEF710
:1008100070BC94F82C1194F82D314A1C38680133BF
:1008200084F82C2184F82D31FDF7F0FFFEF735BC5C
:10083000154C4FF0000ADFF868903EE0783B040862
:10084000E4B50120983A0120AD3A0120565555559E
:10085000CC4C0120F84C0120A8B60120544F0120B7
:10086000EC4C012067666666484F0120784F0120F6
:100870007C4F0120D4B601206BCA5F6B83DE1B4323
:10088000D34D6210144901203C2001201F85EB51FB
:10089000806967FF40420F001649012028BA0120F5
:1008A000180001201B2B00F06F820D2B00F04D81F2
:1008B0004FF0010389F801303868FDF7A3FF0028E5
:1008C00039D03868FDF796FFDBF8003083B27E2B15
:1008D0002AD099F801100029EED194F82E21002A8F
:1008E000E0D07D2B00F0368294F83CE1BEF1000FA1
:1008F00004D080F0200384F83C11DBB2511C224468
:10090000C9B282F83031092984F82E1100F016821C
:100910000829D1D8B4F83A21134403EB132303F088
:10092000FF03A4F83A31C7E784F82EA184F82FA179
:1009300089F801A0C0E794F83D3133B194F8313122
:1009400084F83D01302B00F0148694F82F21CA4B17
:10095000CA499146DFF85CA3DFF85CE34A46002A07
:100960003EF4ABABDBF80020921B012A24D894F8AC
:100970003E21002A40F0268294F83FC133F81C0043
:10098000F8B94FF0010284F83F210A689706E5D5CF
:100990009AF800209007E1D5B94E4FF4F363B949B6
:1009A0004FF40360F28903FB02F381FB0321DB17A1
:1009B000C3EB61111AF00EFC002384F82F31FEF70F
:1009C0007CBB0CF1010CB0F5E06F5FFA8CFC84F895
:1009D0003FC100F099801BD8B0F5047F00F0E7809C
:1009E00035D8B0F5887F00F06981B0F5007F00F060
:1009F0002D81B0F5807FB1D10A685207AED5A24BE8
:100A000019681AF0E7FB002384F82F31FEF755BB75
:100A1000B0F5026F00F0EA806AD8B0F5E46F00F03C
:100A20008280B0F5006F00F09980B0F5E26F95D14B
:100A3000964A6423166C118B03FB06F393FBF1F1CA
:100A40001AF0C8FB002384F82F31FEF736BBB0F54F
:100A5000826F00F05281B0F5C06F00F03E81B0F5BA
:100A6000806F7FF47BAF94F840310133DBB2032B0E
:100A700000F2A28142F2107184F8403101FB03F1CF
:100A8000834B1B88002B40F095810131814B1B78F3
:100A9000DB07814B1B8848BF0431DF0748BF0A31A1
:100AA000980748BF14311A0648BF2831DF0548BFF0
:100AB0002831580748BF64311A0748BFC8319F051D
:100AC00048BF01F5C87198064FF4806048BF01F532
:100AD0007A71DA0648BF01F5FA615F0648BF01F591
:100AE0007A611AF077FB002384F82F31FEF7E5BA1C
:100AF000B0F5046F1CD0B0F5116F00F08D80B0F52B
:100B0000036F7FF42BAF40E79146604A6423D66BB6
:100B1000118B03FB06F393FBF1F11AF05BFB84F8F6
:100B20002F91FEF7CABA9146584A6423566CEFE7F4
:100B30005A4B9146B3F9041001EB810149001AF0B8
:100B400049FB84F82F91FEF7B8BA4FF0010184F801
:100B50003031A4F83A2184F82E11ADE60A689706E0
:100B60007FF5FCAE9AF8002090077FF5F7AE1CF0F9
:100B7000010F434E434900F0EB84726882EAE2734E
:100B8000002AA3EBE27303EB5303A1FB03314FEA0B
:100B9000D101ACBF41F0004141F040414FF4006051
:100BA0001AF018FB002384F82F31FEF786BA9EF85E
:100BB0000520002A3FF4D2AE394A107800283FF4CD
:100BC000CDAE384B5B7B002B00F02385364B1B886A
:100BD00093FBF0F000EB80014FF4047049001AF031
:100BE000F9FA002384F82F31FEF767BA0F68BF06C1
:100BF0007FF5B4AE9AF800C01CF0020F3FF4AEAE21
:100C00001F4E64219146338901FB03F11AF0E2FA89
:100C100084F82F91FEF751BA9EF80520002A3FF480
:100C20009DAE1F4A1278002A3FF498AE1E4B4FF437
:100C300011601B8803EB8303590091FBF2F11AF05A
:100C4000C9FA002384F82F31FEF737BA9EF8062040
:100C5000002A3FF483AE154B4FF4007014491B6813
:100C600081FB0321DB17C3EBA1011AF0B3FA0023C8
:100C700084F82F31FEF721BA783B0408744F012025
:100C80007C4F01201F85EB51544F0120FC4E012069
:100C9000D8B50120CD690120AAB50120584F012007
:100CA0002F4D0120CC4C0120F84C0120EC4C0120B0
:100CB00067666666784F0120604F01200A68520718
:100CC0007FF54CAEBE4B4FF4887019681AF082FA6B
:100CD000002384F82F31FEF7F0B99EF80620002A91
:100CE0003FF43CAEB74B4FF4C06099681AF072FA0B
:100CF000002384F82F31FEF7E0B90A68900640F12E
:100D00000081B14B40F6B832B04E4FF482601F788C
:100D1000317D07F00203002B0ABF00234FF47A73E2
:100D20004FF4FA6217F0010F18BF134619441AF076
:100D300051FA002384F82F31FEF7BFB9B4F83A21F5
:100D4000C2F1FF0293427FF4B3AD4FF0010384F888
:100D50003D31ADE54FF0010384F83C31ACE5FDF7E2
:100D6000ABFB9B4A40F6B8331268801A984200F2F7
:100D70001C81DFF8A0A29AF804303A2B00F0078318
:100D800000233B70FEF7B5B93868FDF73BFD00283E
:100D90007FF48EAD4FF0010384F82F318CE5C4F859
:100DA000203184F818311AF065FA8A4F94F824310A
:100DB000FEF759B9023169E6012342F2107184F855
:100DC00040315DE68449062019F0CEFF002384F807
:100DD0003E0184F82F31FEF770B9013984F85711BC
:100DE000FEF758BD013B84F85A31FFF759B8013B73
:100DF00084F85631FEF72DBC784B1B88D90513D4E7
:100E0000DA0600F1D483980600F16384590600F1F4
:100E10006D841A0700F17F84D80700F17F8413F0F6
:100E2000020F0CBF04260C266D4B6E4A1B78D2783D
:100E300003F001030AB143F0020353201E431AF0EA
:100E40008FF9694B1B8803EB830303EB8303980043
:100E500080B21AF069F900201AF066F9634B644A0F
:100E60001B883868C3EBC3135B0082FB0312D917DE
:100E70001344C1EB63235FFA83FA5146FDF7C6FCC6
:100E800099F80030002138688AEA030389F80030B5
:100E9000FDF7BCFC31463868FDF7B8FC99F8003026
:100EA00038687340DBB2194689F80030FDF7AEFCB4
:100EB00094F848A1FEF777BA0AF1FF3A84F85FA1E7
:100EC000FFF731BB013A84F85E21FFF7CDB84949FD
:100ED0003A2019F049FF2870FEF721B92D22DA7661
:100EE0007EE4454BDBF800101B78C4F81411013B7D
:100EF000012B3FF67DAB1021022391701371FFF798
:100F000077BB3E4A1268120600F13B833C4A127BD3
:100F1000002A3FF423AD94F84111032900F28F8495
:100F2000DFE801F032281902364B1B6859799A79AB
:100F300001F14071DB7901EB022101EB0341002358
:100F400084F841314FF482601AF044F9002384F8A8
:100F50002F31FEF7B2B82C4B1A68137A50791B0464
:100F6000927803EB002313444A1C03EB016184F8DD
:100F70004121E7E7244B1A68D37910791B04527892
:100F800003EB00231344EFE71F4B1A689379D078E3
:100F90001B04127803EB00231344E5E71AF05AF917
:100FA0001A4E01233370FEF731B8194A0021B2F806
:100FB0004A3139700133A2F84A31FEF79AB800BFBE
:100FC000484F0120EC4C0120784F01207C4F01203C
:100FD000A0B90120F44E0120CDB10208AAB501202C
:100FE000CD690120B4B50120F84C0120A8B501203D
:100FF0000308208081720308B0B50120B474012079
:10100000CC4C01204C810120FC380120180001202B
:101010003C20012088B90120A74E0024A74B0AA834
:10102000A6F13F01A64A00930891A64BA64906F8EF
:10103000404C0996F8F730FC089E2920EA21C82286
:10104000731C08933470089B5F1C089718700AA8DB
:10105000089B5F1C08971970089B591C08911A700F
:101060002EF07CFF471C0AA908983A4630F020F978
:10107000DDF820E00122FF210EEB070312A8134444
:1010800008930EF80740089B9F1808971C70089B50
:101090009F1808971C70089B9F1808971C70089B46
:1010A0009F1808971C70089B9F1808971C70089B36
:1010B0009F1808971C70089B9F1808971C70089B26
:1010C0009F1808971C70089B9F1808971C70089B16
:1010D0009F1808971C70089B9F1808971C70089B06
:1010E0009F1808971970089B991808911A7050F862
:1010F000283D9B1B337026F08FF82C70FEF70FB83D
:1011000018469A4603939C4604939E461E461946EB
:10111000FEF7D0BA13F0140F9FED6C7A7EF4C0AFD7
:10112000F0EE477AFEF7C5BF634B12AD684E002064
:101130002F46A3F13D05112103F8400C47F8205D2F
:10114000022503F83F1C384603F83E5C31680B93D8
:101150000397F8F783FA38467168F8F77FFAF3894E
:101160005C49384603EBC3039B00053381FB032135
:10117000DB17C3EBA10189B2F8F786FA338A384648
:1011800003EB8303590089B2F8F77EFA524B1B78C0
:101190009B0740F14282318901F57A7189B2039D42
:1011A0002846F8F771FA0A9B327D2846591C0A91A5
:1011B0001A7026F031F8FEF76DB8484B1868FEF744
:1011C000DDB80122FFF768B8454A00203A4B2121DB
:1011D0001268A3F140070B9303F8400CD300B970D9
:1011E00040F16B8203263F493F4B1B88580500F1B5
:1011F0006182DA0700F17082980701D503263B4926
:10120000DFF8F4903246484630F052F806EB090316
:10121000A9F102020021013312A806F809109A1A56
:1012200040F8203D7A7025F0F7FFFEF730B8C4F89B
:101230001C8186F80090FDF7E9BE1F4B002712AE17
:101240004FF00A0C4FF0080EA3F13D00284903F8B7
:10125000407C284F46F8200D304603F83FCC03F879
:101260003EEC09880B93F8F70FFA3B6830461949B2
:10127000DA1781FB0313C2EBA30399B2F8F704FA60
:10128000BF681AF0C3FD0A9B390C03F1010E3A0A3C
:10129000CDF828E019700A9B591C0A911A700A9B14
:1012A0005A1C0A921F700A9B5A1C0A9218703046E8
:1012B00025F0B2FFFDF7E8BF28B60120F338012082
:1012C00040700408387004084C70040800000000E6
:1012D0007C4F012067666666784F0120544F0120DD
:1012E00038BC012024700408AAB501203470040819
:1012F000F84C0120EC4C0120EBB50120CE4F12AE92
:101300009FEDCE8AB7F9022007EE902ACC4AF8EE7C
:10131000E77A02F8403C0B92A2F14003082267EE04
:10132000887AD91C5A701E2246F8201D3046FDEEE0
:10133000E77A9A70CDED027ABDF80810F8F7A4F9B3
:10134000B7F90030304607EE903AF8EEE77A67EEEC
:10135000887AFDEEE77ACDED027ABDF80810F8F74D
:1013600093F9B7F90430304607EE903AF8EEE77A91
:1013700067EE887AFDEEE77ACDED027ABDF80810C7
:10138000F8F782F9304625F047FFFDF77ABF9AF863
:101390000240D4B1013C00235146E4B21A46013464
:1013A000544411F8013B160A53408C4283EA03135C
:1013B000DBB24FEAC30246EA032682EA131386EA47
:1013C0000302EED1002A7FF4DBAC9E4A9E4E1288C7
:1013D0009E4BF2619E491A689E4C09689B68F262B6
:1013E000DFF88C92B4F84A21F066F364D9F8000073
:1013F000F163F265F7F7F2F9029000287DF474AE1C
:101400000221D9F80000FDF7E9F994F84C310422E3
:101410009AF80310642B049186F8742040F08181BF
:1014200094F84D31072B00F0248294F84D318A4A0C
:1014300006EB031A06930292DAF8041008460391A9
:101440002EF08CFDDAF808105FFA80FA0846059154
:101450002EF084FD069BC0B2039903F00F0E0246E6
:1014600023F00F007C4B039252449872039883F848
:101470000DE002F1080E00EBCA00524683F807E0C7
:10148000987303F10F002FF013FF744B0AF109005A
:101490000599039A18442FF00BFF6F49CB7903F19C
:1014A000010AF3B103F1FF3CC81D0023DFF8C4E1DA
:1014B0005FFA8CFC0CF1080C8C4410F8011B5940AD
:1014C00084454FEA81034FEAD10283EA410302F0E7
:1014D000180283EA01034EFA02F283EA0203DBB246
:1014E000EBD15E4A04980AF8023024F0E3FC94F849
:1014F0004D310022013384F84C2184F84D31029B98
:10150000DDF808A09B785BB11AF805100135D9F811
:101510000000FDF77BF99AF80230EDB2AB42F3D848
:1015200094F84C310322013386F874203A7084F821
:101530004C31FFF75BB94FF0010A494EFDF7F9BE98
:1015400002213868FDF74AF994F82431FDF78BBD84
:10155000326882EAE273002AA3EBE27303EB5303DF
:10156000A1FB03314FEAD101B8BF41F08041FFF741
:1015700015BB3C49881F19F09DFC84F83E01FFF71C
:10158000E4B90026102004230AA98DF828008DF85C
:1015900029308DF82A608DF82B608DF82C608DF83D
:1015A0002D6019F0F7FD84F82F61FDF786BD342614
:1015B0003AE4274B1B6803EB83035F00FEF76BBA2B
:1015C000294BDB78002B0CBF04270527FEF774BEE0
:1015D000012338683370FDF70DF906463868FDF7CA
:1015E00009F9720602D080287DF410AD8A2800F037
:1015F00080808E287DF40AAD94F81831002B7DF49C
:1016000021AD1A4A2D23C4F8202184F82431FDF796
:1016100004BD0C4B1888FFF7DDBA4FF47A71BEE5B4
:101620004FF001090E4EFEF750B9084B9146642069
:10163000B3F900A0FDF751BF584F012058A08B41CE
:1016400028B60120F84C012018000120EC4C0120A4
:10165000544F01203C20012090AE012096AE012085
:101660007C4F012074210120B4B50120A8B60120CF
:1016700028BA01200007090E89499A790B8803EBE3
:10168000830303EB83034FEA83091FFA89F9002AD6
:1016900040F0FA804FF0FF330FFA83FA1AF0B6FBEE
:1016A00040B2FDF71ABF08468A4603918C46049162
:1016B000FEF700B803267B49A2E57B4B7B4A1B68FB
:1016C0007B4903F48003834216BF11460426032698
:1016D0008AE52426FFF7A8BB0426764990E51389FE
:1016E00007EE903AF8EE677AFEF7E3BC1026FFF7B4
:1016F0009BBB714B1B689B067DF588AC94F8183139
:10170000002B7DF49FAC6D4A2D23C4F8202184F872
:101710002431FDF782BC2026FFF786BB0826FFF7A1
:1017200083BB96F875C01CF00F0F03D10CF1010CB0
:101730005FFA8CFCBCF1070F614B059528BF4FF099
:10174000010C1A46029300234FEA0C1A02F10D0E07
:10175000937206EB0A035FFA8AF2197C594B0392E3
:101760000B4493F82420039B012A0EF1010541EA62
:10177000030106EB0A038EF80010DB680CD9901EFB
:101780002A46C0B2811C714402F8013B8A424FEAEA
:101790001323F9D101300544B2440CF1010C23F0BC
:1017A000600305F1010E9AF811205FFA8CFC1343D7
:1017B000BCF1080F2B704CD003994FEA0C1A424B26
:1017C000103106EB0A02AEEB0303C9B20391117CA0
:1017D0003C4A0A4492F8242098181328C3DD059D3A
:1017E000DBB20298DFF8ECE09A1DD2B242F0400181
:1017F00002F1010AC171D2B1053302990EF1010063
:101800000022DBB20833CB18039310F8011B5140C0
:101810008A00CB0882EA410203F018034A402B49B0
:1018200041FA03F35A40039B8342D2B2EDD10498AC
:101830000AF80E2086F875C024F03CFB5FE64B1CCE
:101840000906DBB2042B84F841313FF478ABFFF793
:1018500079BB1D4B059DAEEB0303C1E708468A46E5
:1018600003918C4604918E46FDF724BF0846FDF790
:1018700021BF9DF8083084F84D31D6E508468A46E8
:1018800003918C46FDF716BF114B1B6804E7084611
:101890008A46FDF70FBF08468A460391FDF70ABF47
:1018A000F84C012028700408B47401202470040846
:1018B0001C7004082C700408744F0120D4B6012059
:1018C00090AE0120783B04089DAE01200007090E70
:1018D000EC4C012096AE01202DE9F04F95B00C465E
:1018E0001646B0F9083000AFDDB20B81442D00F090
:1018F0006F84804645D9812D00F0988300F2A48042
:10190000542D00F0D88040F2E2806E2D00F02E843D
:10191000802D40F0DF807C4B93F800A00AF1020A92
:101920001AF0FF0A00F0A380784B0A25DFF80C823A
:101930009A4403F10109764EDFF804B218E0322D23
:1019400001F08C83A5F13C00C0B2132841F2B083B2
:1019500000232268D14502F101012160157022683F
:1019600002F101012160137000F0818019F8015B20
:101970000A2DE4D1BBF80030FF2BA8BFFF23DBB258
:10198000E7E7052D00F0128421D8022D00F08B80AE
:1019900040F22983032D00F0D683042D40F09A8075
:1019A0005C4920462A46F7F74FFE5B4B20461978E4
:1019B000F7F78EFE2168012300205437CD181A4610
:1019C0002560087018466281BD46BDE8F08F242D61
:1019D00067D040F2B582282D00F07283382D79D17E
:1019E0000A6801204FF0050E0A2602EB000C0346A0
:1019F00000254A49C4F800C010700246206800EB78
:101A0000030CC4F800C080F800E0206800EB030E6F
:101A1000C4F800E006702068C618266005702068CB
:101A20000D78C6182660057020684D78C6182660A7
:101A3000057020688978C5182560017018465437EC
:101A40006281BD46BDE8F08FA02D18D040F29C8287
:101A5000B82D00F07683FE2D3CD1314D05F10806FE
:101A600035F8021B2046F7F733FEAE42F8D10123CA
:101A70001A46184654376281BD46BDE8F08F294B9F
:101A800008461968F7F70EFE274B20461968F7F746
:101A900009FE264B19682046F7F704FE01231A4673
:101AA000E7E7234BF6E7042222492046F7F7CCFD6F
:101AB00001231A46C2E7096801230020CD181A46FF
:101AC000256008702168CD1825600870B6E7522D92
:101AD0003FF470AF21462846FAF70CFF0346002872
:101AE000C5D1742D00F09582772D2BD1D8F8002028
:101AF000D8F80410914240F0788319460E4A2046E7
:101B00002BF0D2FFB3E700BF354C0120CC3B0408DB
:101B100014500120F3380120002301200B4501203F
:101B2000584C0120107AF01F147AF01F187AF01F19
:101B300068460120B87004086DCD030867666666C4
:101B40003C500120F52D01F08D83762D00F052835D
:101B5000472D01F03583292DD8F8006001F0198355
:101B6000392D01F0DC82212D01F0ED82D8F804201E
:101B70000B3D931BEF2D00F2268401A151F825F0B7
:101B80009D2A0108C7230108C7230108C7230108AC
:101B9000C7230108C7230108C7230108C723010879
:101BA000C7230108C7230108C7230108C723010869
:101BB000C7230108C7230108C7230108C723010859
:101BC000C7230108C7230108C7230108C723010849
:101BD000C7230108C7230108C7230108C723010839
:101BE000D72A0108C7230108832A0108C72301084F
:101BF000612A0108C7230108C7230108C723010878
:101C0000352A0108C7230108AD290108C7230108A7
:101C10003D290108C723010815290108C723010828
:101C200001290108C723010897280108C7230108D3
:101C3000F3270108C7230108C7230108C7230108A8
:101C4000C72301086F1A0108C7230108A92D01083D
:101C5000C7230108C72301088D2D0108C7230108E8
:101C60002D2D0108C7230108C7230108C723010838
:101C7000C7230108EF2C0108C7230108C723010867
:101C8000C7230108A32C0108C7230108512C010810
:101C9000C7230108C7230108112C0108C723010825
:101CA000C7230108C7230108C7230108C723010868
:101CB000C7230108C7230108332B0108C7230108E4
:101CC000612F0108C7230108AF2E0108C7230108AF
:101CD000FD2D0108C7230108C92D01082130010885
:101CE000C7230108C7230108C7230108C723010828
:101CF000C7230108C7230108C7230108C723010818
:101D0000C7230108C7230108C7230108C723010807
:101D1000C7230108C7230108C7230108C7230108F7
:101D2000C7230108C7230108C7230108C7230108E7
:101D3000C7230108C7230108C7230108C7230108D7
:101D4000C7230108C7230108C7230108C7230108C7
:101D5000C7230108C7230108C7230108C7230108B7
:101D6000C7230108C7230108C7230108C7230108A7
:101D7000C7230108C7230108C7230108C723010897
:101D8000C7230108C7230108C7230108C723010887
:101D9000C7230108C7230108C7230108C723010877
:101DA000C7230108C7230108C7230108C723010867
:101DB000C7230108C7230108C7230108C723010857
:101DC000C7230108C7230108C7230108C723010847
:101DD000C7230108C7230108C7230108C723010837
:101DE000C7230108C7230108C7230108C723010827
:101DF000C7230108C7230108C7230108C723010817
:101E0000C7230108C7230108C7230108C723010806
:101E1000C7230108C7230108C7230108C7230108F6
:101E2000C7230108C7230108C7230108C7230108E6
:101E3000EF2F0108C723010841300108C72301081B
:101E4000C7230108C7230108C7230108C7230108C6
:101E5000C7230108C7230108C7230108C7230108B6
:101E6000C7230108C7230108C7230108C7230108A6
:101E7000C7230108932701083D270108FB26010815
:101E8000C72301084326010829260108BD250108AA
:101E9000C7230108A32501083B25010811250108D6
:101EA000FF2401089D240108C72301086F240108AD
:101EB000C7230108C72301084D240108192401087C
:101EC00005240108D1230108A32301088123010867
:101ED0004B23010831230108C7230108C723010848
:101EE000C7230108C7230108C7230108C723010826
:101EF000C7230108C7230108C7230108C723010816
:101F0000C7230108C7230108C7230108C723010805
:101F100017230108C7230108C7230108A7220108C6
:101F2000C7230108C7230108C7230108C7230108E5
:101F3000C7230108C7230108C72301088D22010810
:101F4000202D7FF4C7AD0B680846BD4D591C6A783B
:101F500021601A7023682A78591C21601A7023683E
:101F6000AA78591C21601A702989F7F7B1FB2168FA
:101F700001236879CE181A46266008702168A8796E
:101F8000CD182560087059E5822D7FF4A3AD0B684C
:101F90000846AC4A5E1CAC4D1178A94A26601970FF
:101FA0001189F7F795FBA94B226820461B88511C25
:101FB000FF2B2160A8BFFF231370A96881F31001D4
:101FC00089B2F7F785FB2968204601F30F0189B232
:101FD000F7F77EFB21689E4A01231078CD181A4638
:101FE000256008702AE5012D7FF474AD096800268C
:101FF0002B46242001F1010E2A46C4F800E00E70A1
:1020000021684E1C26600D7021684D1C25600870EB
:1020100014E5D8F80020D8F80410914240F0E08090
:1020200019468C4A20462BF03FFD20E58A4B1E784E
:10203000033616F0FF063FF41AAD884B4FF00A093D
:10204000DFF840821E4403F1010A20E0B9F1500F8D
:1020500001F00180B9F1320F01F04080A9F13C009C
:10206000C0B2132841F24280002529462368204649
:102070005A1C226083F80090F7F72AFB2946204675
:10208000F7F726FB56453FF4F2AC1AF8019BB9F17D
:102090000A0FDBD172498B684FF6FF72096803EBB8
:1020A000830391424FEA4305A8BF1146954221EAB6
:1020B000E171A8BF154689B225EAE575ADB2D5E74D
:1020C0000B68022101254FF006085E1C0A22DFF88A
:1020D000B8912046266019702368624E5919216014
:1020E00083F800802368591921601A7023685A19EF
:1020F00022601D70B9F80010F7F7EAFAB9F802107B
:102100002046F7F7E5FA23685021002203EB050E7D
:102110002046C4F800E083F80080236803EB050E36
:10212000C4F800E019702368591921601A703188C9
:10213000F7F7CEFA71882046F7F7CAFA2B462A46F7
:102140007CE4494BA6E4096801230226002001EB48
:10215000030E1A46C4F800E00D702168CD18256002
:102160000E702168CD182560087067E4374B08466B
:102170000A681B88511C344DFF2B2160A8BFFF2328
:102180001370A96881F3100189B2F7F7A1FA374BF0
:1021900020461988F7F79CFA2968204601F30F01B9
:1021A00089B2F7F795FA01231A4647E40B22304922
:1021B0002046F7F749FA08222E492046F7F744FA55
:1021C00007222D492046F7F73FFA01231A4635E446
:1021D000002A3FF44CAC294A012332601A462DE410
:1021E000531CC8F8003011781BE7531CC8F80030A6
:1021F000117883E4D8F80020511CC8F80010127838
:10220000002A01F06A81102A01F0BD811E4619469C
:10221000256820466B1C23602A70F7F743FA314685
:102220002046F7F73FFA164B20461968F7F73AFAB7
:1022300000212046F7F74CFA00212046FFF7B8BBF3
:10224000604F01202F4D0120EC4C0120F84C012063
:10225000B0B501204DD90308354C0120DC3B040802
:10226000C84F0120FC4F01200C290120A8B50120F6
:10227000C0700408CC700408D8700408D5C80008E1
:10228000FC2601200C50012074BC0120D24B1B788D
:10229000DB0700F19880FBF719FCFBF71BFE01231D
:1022A0001A46FFF7CBBB731CC8F8003033780F2BEE
:1022B00000F28980B51CC3EBC302C849F01CC8F802
:1022C000005006F1040E75788B188D54751DC8F8F2
:1022D0000000B01DB278F11D5A7006F10802C8F86E
:1022E00000E096F803E083F802E0C8F80050357982
:1022F000DD70C8F8000070791871C8F80010B17965
:102300005971C8F80020F2799A712CF0DBF801239A
:102310001A46FFF793BBB24D4046F7F783F9E881C1
:102320004046F7F77FF90123A8811A46FFF786BBDD
:102330004046AC4DF7F776F9012300EB80001A46D2
:1023400000FA03F12980FFF779BB3046731CA649D8
:1023500006F1030EC8F80030351D10F8022B0123DA
:102360000A701A46C8F8000070784870C8F800E093
:10237000B0788870C8F80050F078C870FFF75EBB7E
:102380009A4D4046F7F74EF928824046F7F74AF94A
:1023900068824046F7F746F90123A8821A46FFF7FC
:1023A0004DBB711C3346F21CC8F8001013F8020B29
:1023B000C8F800307178C8F80020B27825F006FB24
:1023C00000287FF454AB4FF0FF331A46FFF736BBBB
:1023D0003146731C864AF01CC8F80030012311F8FE
:1023E00002EB7F4D82F800E01A46C8F8001096F81C
:1023F00001E07C4985F802E0C8F80000B0788870F8
:10240000FFF71CBB7B4B4E227B4918682EF050FF18
:1024100001231A46FFF712BB3246701C774BF11CA2
:10242000C8F80000404612F8025B1D70C8F8002092
:1024300072785A70C8F80010B2789A70F7F7F2F80C
:102440006F4A0123D0801A46FFF7F8BA6C4D404618
:10245000F7F7E8F828804046F7F7E4F86880404648
:10246000F7F7E0F80123A8801A46FFF7E7BADFF88C
:10247000B09199F80030002B3FF4F9AA614E002585
:1024800040460135F7F7CEF80DF06AFC99F80030B8
:10249000A6EC010A9D42F3DBFFF7E9BA0D2B92D1BE
:1024A000731CC8F800303578072D8CD80C26DFF85F
:1024B0007491404606FB05F6F7F7B4F809EB0605FC
:1024C000A8804046F7F7AEF8E8804046F7F7AAF84C
:1024D000D8F80030288140461A46591CC8F8001028
:1024E00012F8021BA972C8F800205B78EB72F7F7AC
:1024F00081F8012349F806001A46FFF79FBA4046C3
:10250000F7F790F8404A012310801A46FFF796BA71
:10251000731CC8F800303078060601F19E802E4BFF
:102520001B78DD073FF5A3AA032828BF0020FBF78F
:10253000B3FA01231A46FFF781BA731C4046C8F864
:10254000003096F800A0F7F755F881464046F7F7B7
:1025500051F806464046F7F74DF805464046F7F76E
:1025600061F84046F7F75EF84046F7F767F8BAF1CA
:10257000000F01F05D80BAF1100F7FF478AA234BB1
:10258000C3F800905E600DB1214B1D60214902220D
:10259000214B081F1A700EF029FE01231A46FFF77F
:1025A0004DBA0D4B1B78D8073FF561AAFBF760FBCE
:1025B000FBF790FC01231A46FFF740BA064B1B7845
:1025C000DA073FF554AA1548012301781A4641F06D
:1025D00004010170FFF732BACD69012098BE0120D5
:1025E00084BC012094BC0120E449012054770120DF
:1025F000A46C0120FC380120E05004087CBC0120C0
:10260000F42A01204C2A0120E04901200425012060
:10261000FC26012008250120CA480120784F01200E
:10262000354C0120C0C40120D24B1B78D9073FF59F
:102630001EAAD14A4FF4C871012311801A46FFF730
:10264000FDB9092B7FF7BFAE3346701CDFF85893F6
:10265000F11C321DD9F80050C8F80000701D13F8A5
:1026600002EB85F800E006F1060EC8F8003073783A
:10267000AB70C8F80010F11DB378642BA8BF6423B9
:102680006B71C8F8002006F10802F378642BA8BF2C
:102690006423AB71C8F8000040463379EB71C8F889
:1026A00000E07379642BA8BF64232B72C8F8001074
:1026B000B379EB70C8F80020F3792B71F6F7B2FF0D
:1026C000D8F80420D8F800306881D11A00290EDD2E
:1026D000581CD9F80010121AC8F800001878002AFF
:1026E000487204DD9A1CC8F800205B784B7022F019
:1026F000F7FA01231A46FFF7A1B9A04AF31C2136C5
:10270000106802469D1E591E0332C8F8005013F887
:10271000035C02F8035CC8F8001013F8021C02F80E
:10272000021CC8F80030033313F8041C9E4202F860
:10273000011CE7D12CF0B8FAFFF799B9731C904A45
:10274000C8F800303378002B00F06D87137843F021
:102750000203B11C13708B4D4046C8F8001073780B
:10276000894E2B75F6F746FF28604046F6F742FF84
:1027700068604046F6F756FF28814046F6F752FF5C
:1027800031780123E88141F002011A463170FFF7E8
:1027900055B9C3F34705122D3FF615AEC5B107F184
:1027A000500307F12A0903EB450A4E46AAF1260A0F
:1027B0004046F6F737FF26F8020FB245F8D1734BC3
:1027C00039F8022F4E4523F8022FF9D1112D0AD8DE
:1027D0006B006F480021023B00F12202034423F802
:1027E000021F9A42FBD101226A4913460A70FFF781
:1027F00025B90722B3FBF2F2C2EBC2055B1B7FF4E3
:10280000E2ADD2B202F1FF3A5FFA8AFA002A3FF44F
:102810002EA90AF1010A1D46DFF87CB13246511C8F
:102820005D4B4FF00009C8F8001092F9001005E068
:1028300009F10109B9F1060F3FF4C5AD93F9022082
:1028400008338A42F4D10BEBC90640460135B1701A
:10285000F6F7E8FED8F800302BF83900AA451946FB
:1028600003F1010203F10300C8F8002003F10402A0
:1028700011F802EB86F803E0C8F8001059783171BE
:10288000C8F800009978B171C8F80020DB7873713E
:10289000C5D1FFF7ECB8731CC8F8003031780E29A9
:1028A0003FF691ADB31CC8F80030707803283FF6AE
:1028B0008AAD0623394AF51C06F1040C03FB01F32B
:1028C00006F1050ED1184871C8F80050B51DB07852
:1028D000D054F01DC8F800C00123F2784A701A469F
:1028E000C8F800E096F804E081F802E0C8F800506B
:1028F0007579CD70C8F80000B0790871FFF79EB8FF
:10290000721C27490123C8F8002030781A46487500
:10291000FFF794B8721CC8F8002035781F2D3FF6D9
:1029200052AD052B7FF44FAD4046F6F763FE1D4BCD
:1029300043F8250017F080FAFFF799B8194D05F113
:10294000400640460435F6F76DFED8F80030A5F88D
:102950007C00591C1A46C8F8001012F8021B85F8B2
:102960007E10C8F800205B7885F87F30AE42E8D151
:10297000FFF77DB8CD6901206C810120FC38012072
:10298000784F01207C4F0120C84801205EB801200B
:1029900060B8012084B80120CCCA01201829012088
:1029A0000C77012078B401204C810120731CD34D99
:1029B0004046C8F8003033782B72F6F733FEA88310
:1029C0004046F6F72FFE28834046F6F72BFED8F850
:1029D000003068835A1CC8F800201B78EB74D8F8C4
:1029E00004309A1A032A00F3F185D8F800105A1A15
:1029F000052A11DD4B1C4046C8F800300B78EB72FD
:102A0000F6F7F8FDD8F80030E8605A1CC8F8002046
:102A10001B782B7498E80A005B1A002B7FF727A815
:102A20004A1C0123C8F800201A46097885F82110AD
:102A3000FFF704B8731CB248D21AC8F800303378D4
:102A4000002A03707FF713A8B21C0123C8F80020E6
:102A50001A467178003118BF01214170FEF7EEBFB0
:102A6000A84D4046F6F7DEFD28604046F6F7DAFD51
:102A700068604046F6F7D6FD0123A8601A46FEF7C7
:102A8000DDBFA14D002340462B60F6F7B3FD2A6859
:102A9000012310431A462860FEF7D0BF102B9B4934
:102AA0004FF0000228BF10230A604A608A60CA60A3
:102AB0000A74002B3EF4DBAFD8F800200139134430
:102AC0000132C8F800209A4212F8010C01F8010FF7
:102AD000F6D1FEF7CCBF731CC8F800303578132D43
:102AE0003FF671ACB31CC8F8003070782BF016F8C4
:102AF00000283FF468AC90F800E0F01C844B311DD6
:102B0000721D03F825E003EB8503C8F80000B578D3
:102B100080485D70C8F80010F17800689970C8F8B6
:102B200000203279DA7022F069F801231A46FEF7A4
:102B300085BF4046F6F776FD05460EF061FCFF289E
:102B40003EF495AF3F2D00F22A854FEAD5090023C8
:102B500007F1500607F12B0009F1010987F82B3026
:102B600006F8243D31460EF02BFC97F82B305FFA27
:102B700089F905F007054B4505F1010503D197F8E3
:102B80002C30AB4203D0294648460EF025FCD8F83D
:102B90000030D8F80420D21A012A7EF768AF591CF9
:102BA000002207F15000C8F800101D7800F8252D0C
:102BB0000EF0FAFB97F82B30AB420AD0564B1B684D
:102BC0003BB19A79AA4204D31B681B690BB1284612
:102BD0009847D8F8003000223046591CC8F8001039
:102BE0001D7887F82C200EF0D3FB97F82C30AB42E1
:102BF0003EF43DAF484B1B68002B3EF438AF1B68DA
:102C00005B69002B3EF433AF28469847FEF72FBF91
:102C1000424B1B78012B3EF62AAFF31C701C314649
:102C20003F4DD21AC8F8000011F8020B012AA87013
:102C3000C8F8001096F801E0C8F8003040F3268587
:102C40004046F6F7EFFC012328801A46FEF7F6BE51
:102C5000731CC8F8003096F80090B9F1110F3FF6D8
:102C6000B2ABB31C2F4D4046C8F80030737819261C
:102C700005F8193005EB4905F6F7D4FC40F6CA0310
:102C800040F2EE229842A8BF184601239042B8BFF6
:102C900010461A46A0F2EE2191FBF6F16970FEF79C
:102CA000CDBE3346721C204D4046C8F8002013F8B4
:102CB000022B2A71C8F8003073786B71F6F7B2FCFA
:102CC000D8F80030288040465A1CC8F800201B78ED
:102CD000AB71F6F7A7FCD8F8001001236880C8187C
:102CE0001A46C8F800000978E971FEF7A7BEF8F7A0
:102CF0002FFD01231A46FEF7A1BE00BF0C7701206D
:102D0000C03F0120F06101206846012060BC012025
:102D1000C43F0120FC380120D82B01203946012076
:102D20003C46012078BA0120102B0120721CDFF8EC
:102D300078930021CD4BC8F8002040463278C9F87E
:102D400000101A70F6F756FCD8F80020D9F80030B9
:102D5000561CC7490343C74D4046C9F80030C8F860
:102D6000006013780B72F6F75DFC28604046F6F7BA
:102D700059FC68604046F6F755FCA8604046F6F7F7
:102D800051FC4046F6F74EFCFEF771BEBA4B06F119
:102D900008020136C8F80060964216F8011C03F8D4
:102DA000011FF6D1FEF763BE3146721CB348012302
:102DB000C8F8002011F8025B1A468570C8F80010A8
:102DC00071784170FEF73ABE3146731CAC4AF01C74
:102DD000C8F80030012311F802EBAA4D82F803E095
:102DE0001A46C8F8001096F801E0A74985F805E0F2
:102DF000C8F80000B078C870FEF720BE4046A34D6A
:102E0000F6F710FC4046F6F70DFC4046F6F70AFCD4
:102E10004046F6F713FCD8F800302A6840461946B9
:102E200003F1010EDE1CC8F800E011F802EB82F895
:102E30002CE0C8F80010597882F83610C8F8006005
:102E40009B7882F83730F6F7F9FB4046F6F7F6FB49
:102E50004046F6F7F3FB2E684046F6F7E3FB708733
:102E600040462E68F6F7DEFB98E80A0030875A1ACB
:102E7000012A0BDD4A1C2B684046C8F800200A785E
:102E800083F82E20F6F7DAFB98E80A005B1A032B8A
:102E90000BDDD5F800904046F6F7C4FB2E68A9F884
:102EA00032004046F6F7BEFBB086286842E4731C49
:102EB000764DDFF8F8914046C8F80030D5F800A00C
:102EC000337889F80530F6F7ADFBAAF820004046C4
:102ED0002E68F6F7A7FB98E80A00F0835A1A072A2B
:102EE00015DD4046F6F79EFBA9F80A004046F6F7C6
:102EF00099FB2E68A9F80C004046F6F793FB708406
:102F00002E684046F6F78EFB98E80A00B0845A1AFD
:102F1000032A0BDD4046F6F785FBA9F80E00404674
:102F2000F6F780FB98E80A00A9F810005B1A002B5E
:102F300006DD4A1C2B68C8F800200A7883F8262092
:102F4000FAF7CEFD1DF076FE514B1B68002B00F00A
:102F50005F8328682BF044FB01231A46FEF76EBD01
:102F60003346721CDFF84491F11CC8F80020321D72
:102F700013F8025B404689F80250C8F80030454D0E
:102F800073782B70C8F80010434DB3782B71C8F8D4
:102F90000020F378092BA8BF0923AB70F6F742FB9A
:102FA00098E80A0028805A1A012A05DD4046F6F7FB
:102FB00039FB98E80A00E8818B4208D04B1CC8F81E
:102FC00000300B78003318BF012389F80730FAF777
:102FD00087FD98E80A008B423EF449AD4A1C012364
:102FE000C8F800201A460978E970FEF727BD711C61
:102FF0003346F21CC8F8001013F8025BC8F8003022
:103000007078C8F80020B178002D00F06B83012D96
:103010007EF42DAD20F00CFF2B462A46FEF70EBDA8
:103020001E4B1B7813F001017FF4CDA9731CC8F867
:103030000030307820F0AEFE01231A46FEF7FEBCC9
:103040000023174D40462B60F6F7D4FA0123286081
:103050001A46FEF7F3BC1349FFF71DB83388FF2B60
:10306000A8BFFF23DBB2FEF774BC00BFC03F012046
:103070000C770120F06101200B770120A0BC01201A
:1030800084BC01201CB8012094BC0120FC38012024
:10309000BC3F012078BC012054770120CD6901207C
:1030A0000C2901200050012068460120A46C012059
:1030B00017F040FD00283EF44BAC03780A2B2CD8C7
:1030C000B0F9023088FB0312DB17C3EBA2039BB2FB
:1030D000FF2BA8BFFF23DBB2FEF73BBCD8F80430C0
:1030E0004FF6FF72D8F80010FEF7D9BF17F022FD97
:1030F00000283EF4B9AF03780A2B3EF6B5AFB0F91D
:103100000430B0F9061003EB830321EAE17183F385
:10311000500589B2ADB2FEF7A9BF0023DBE7731CEF
:10312000C8F8003033780A2B00F0BD814046F6F72E
:1031300085FA4046F6F782FA4046F6F77FFA012311
:103140001A46FEF77BBC3346711C7E4DF21CC8F854
:103150000010404613F8021B6970C8F800307378FD
:103160002B70C8F80020B378AB70F6F75BFAD8F88C
:10317000001001232881CE1808461A46C8F80060BE
:1031800010F8026B6E71C8F800004978A971FEF75B
:1031900055BC731CC8F8003033780A2B00F0CF8080
:1031A000502B7FF4EBAD684D4046F6F73BFA288094
:1031B0004046F6F737FA012368801A46FEF73EBC10
:1031C000D8F804204046D8F800507B62551BF6F72B
:1031D00011FA7B6A052D386200F2A2808026012553
:1031E000B34620467B6294E80600521A396A103AC8
:1031F000B242B8BF1FFA82FB544A92683A61521A2F
:10320000396A9345FA6088BF1FFA82FBF6F74AFADB
:103210007B6A002B40F0A880002D00F063814B4BAF
:10322000D4F800809D683B6A5B449D4280F05181E8
:103230003B6AED1AF8F700FA2A464146386AF7F772
:1032400045FF2368B04203442360BEF610AC002162
:1032500000E0236801305A1CB04222601970F8D196
:10326000FEF705BCD8F80030D8F804209A4240F0A8
:103270005781374BFF225A704FF00008354D1FF031
:1032800035FF20224146344885F8008030F059FA55
:1032900087F82C80424697F82C30072B33D8DFF87C
:1032A000C490DFF8B48097F82C3003EB430309EBAC
:1032B000C3035B7CEBB197F82C30202103EB430375
:1032C00009EBC3035B69A3B197F82C3003EB43030D
:1032D00009EBC3035B6948F822301846FBF740FC52
:1032E0002B7858F82300FBF745FC2A780132D2B23C
:1032F0002A7097F82C300133DBB287F82C3097F81E
:103300002C30072BCFD92368591C21601A70002E4E
:103310003EF4ADAB114A012332601A46FEF78EBB74
:103320004046F6F77FF9D8F80020D8F80410834615
:103330007B6A914240F01D8106461D4651E7084DCB
:1033400032E700BF604F0120FC4F0120201E01200A
:103350000023012077BD0120A4B9012009DE030864
:1033600074BC0120F475012022680023C7F800D046
:10337000C0B0511D5371C7F808D0F961BBF1000FFF
:1033800000F009813A6A39698A4280F001817C60E3
:1033900099463D6A4FF0800A1C467B62FB681C1B05
:1033A000C04BB4F5807F9B6828BF4FF480746219CE
:1033B0009A4288BF5C1BF8F73FF9BE682846224650
:1033C0003146F7F783FEF96906EB000CB8610C781B
:1033D00066457C6132D20CF1FF3C06F1FF3E1EF8DF
:1033E000013FB14AB04802EB830210F823505688DF
:1033F0000DB300234FF4004205F1FF38164209F1E6
:1034000001044FEA520203D008784AEA000008702B
:103410005FEA5A0A06D181F801A01FFA84F9013146
:103420004FF0800ACB4503D8F44536D8984534DCB4
:1034300001339D42E2D1F445D1D1F9617B6AD9458E
:10344000BA6913449BB27B6206D27B6A3A6A1C4615
:10345000D5183B699D42A1D37C68BAF1800F03D097
:1034600009F101031FFA83F909F102012046012540
:1034700089B2F6F72DF92368796A20465A19226035
:103480001D70F6F725F922682B4602EB09012A4642
:103490002160D7F800D0FEF7D1BAFB697C681A46E4
:1034A0003B7D1370D9E7B31C8049F51C301DC8F86B
:1034B0000030012396F801E01A4681F800E0C8F8D0
:1034C0000050B5784D70C8F80000F0788870FEF7AD
:1034D000B5BAF8F7B1F85A46AFE6754B93E8420033
:1034E000FEF796BE59462046F6F7F2F823683A6A88
:1034F000591C5A4421601D706A4B26689D68AA4277
:1035000000F2B680F8F798F85A463146386AF7F76D
:10351000DDFD2268012310441A462060FEF78EBAB2
:103520005A1C19466348C8F8002011F8022B427053
:10353000042AC8F800105B78837003D9FF2A7EF450
:1035400039AA99E65C490978994205D8022A7EF49D
:1035500031AAFF2B7EF42EAA22680123D118216004
:103560001370002E3EF483AA54491A463160FEF7C8
:1035700065BA511C1D460646C8F800101378003382
:1035800018BF01232DE64E4B93E84200FEF740BEE4
:103590007B62994668E7D946C7F824B064E707F12B
:1035A0002C0630460DF0E8FEBB8DAB423FF4EFAA8F
:1035B000444B1B68002B3FF4EAAA1B689B69002B55
:1035C0003FF4E5AA28469847FFF7E1BA4046F6F7E8
:1035D00029F8A8844046F6F725F898E80A00E88418
:1035E0005A1A032A7FF703AA0B464A1C4046C8F81A
:1035F000002013F8022BAA77C8F800304B7885F822
:103600002030F6F70FF898E80A006884FFF7EFB962
:103610002D4901232D4E2E4D1A462E48316029602A
:103620000160FEF70BBA137803F0FD03FFF791B8C2
:103630001F4B1020C3F800905E601CF08DF8264AE6
:10364000137843F001031370002D3EF410AA234AAF
:10365000012315601A46FEF7F1B900F07F00032838
:1036600028BF002020F002FC01231A46FEF7E6B92D
:103670003B6AED1AF7F7E0FF3146386A2A46F7F75A
:1036800025FD236803442360FEF7F1B9144A0123A2
:10369000B07811881A4611FB0EF191FBF0F12980E8
:1036A000FEF7CCB9201E0120EC3B04080B4501209D
:1036B0000C49012000230120354C0120E1C80008FD
:1036C00004250120D82B01207582000888BF012025
:1036D000DCBF0120DCC30120784F0120FC26012043
:1036E000ACBA01202BF046F901231A46FEF7A6B921
:1036F000C44B2DE9F0471C6862072DED028B03D403
:10370000BDEC028BBDE8F087BF4D2B78002BF7D0C6
:103710006E6846F2A713861B9E42F1D9DFF84C93E0
:103720006860B9F80070DFF84883002F40F0A4818A
:1037300098F80620B7EE008AAB68013A9FEDB30A0D
:10374000DFEDB30ADFF8E892B3FBF2F307EE903A4D
:10375000F8EE677A27EE800A2EF048F838EE400A35
:10376000DFEDAC7A20EE270A2DF0D0FEB8F8083055
:10377000DFEDA96A07EE103AEB68B8EEC77AC01A17
:1037800007EE900AA7EE668AB8EEE70AD9ED0A7A44
:10379000F8EEE77A20EE080A67EEA67AA7EE270A87
:1037A0002DF0B4FE9D4B0146C9F828001860A30710
:1037B00040F1A381DFF8BCE2994CDEED007ADFED49
:1037C000995AF8EE677A226867EEA55A002A00F047
:1037D000B281954B07EE102AD3ED026AB8EEC77A94
:1037E000F8EEE66A86EE878A904AD5ED054A92EDB4
:1037F000007AB8F80C2067EE877ADFED873A06EE9C
:10380000902AB6EE004A95ED066AB7EE005AF8EE39
:10381000E66A874A67EE887A92ED0A7A66EEA36ACC
:103820007E4AF0EE643AB8EEC77A35EE665AE7EEB5
:10383000843A77EEA47A27EE057AC5ED057AF0EEA4
:10384000467AE3EEA57AA7EEA67AF0EE477ABDEEC9
:10385000C77AC5ED067A82ED007A764A1278122A86
:1038600000F0528100221A605A609A602260CEF8FD
:103870000020002F7FF444AFEA6907EE906ADFED85
:103880006E6A40F2DC548B1AF8EE677AE9610A211D
:1038900007EE103A694BB8EEC77A27EE267AC7EEE4
:1038A000276AFDEEE67A17EE900AA042A8BF2046EE
:1038B0009842B8BF1846F6F793F8B8F80A30F7EE12
:1038C000007A9FED556A07EE103A05EE900AD5EDA5
:1038D000056AB8EEC77AF8EEE55A66EE866AE7EE54
:1038E000467A67EEA57AE7EE267AB0EE670AC5ED6E
:1038F000057A2DF00BFE05210646F6F771F8504AC1
:103900005049B2F90040086084EAE473A3EBE47321
:10391000B3F5487F71DAB2F9022082EAE273A3EBD1
:10392000E273B3F5487F68DA474B1B78002B40F011
:103930000681464B0A21394A1B68126844489B1A83
:10394000B3F5FA7FA8BF4FF4FA739842B8BF184690
:10395000F6F746F83F4B1C68637A00FB03F03E4BDA
:103960000028B8BF7F30C211B2F5967FA8BF4FF4D0
:1039700096729A42B8BF1A46911BE37E374801FB04
:1039800003F3354F0668002B227F95ED087AB8BF08
:103990001F3301FB026232495B11B3F5967FA8BF6A
:1039A0004FF49673BB42B8BF3B46B2F5C81FA8BFE1
:1039B0004FF4C8128A42B8BF0A460260002AC0F219
:1039C000C380617F37EE087ADFED266A03EB62334E
:1039D00007EE901A6FF0950127EE267AF8EEE77A57
:1039E00067EE877AFDEEE77A17EE902A962AA8BF4F
:1039F00096228A42ACBF9F1A5F1A1B4A85ED088A3D
:103A000017607DE6744F01200423012008942537B8
:103A1000B1DC423ED048874A6F12833A544F0120AE
:103A2000F8280120BD378635E82801200C2B01201D
:103A300010C70120544C01200024744924FAFFFFD0
:103A4000584F0120484F012004270120FC26012067
:103A50000CFEFFFFFC380120D4FEFFFFF4260120FE
:103A60000000E7FF0000003BEC2601206A810120F6
:103A70001CB80120F4280120364998F806A00A68ED
:103A80000AF1FF3AAB68002A9FED330ADFED330AF3
:103A9000B3FBFAF39246B8BF02F1070AA2EBEA02BF
:103AA00003EB020ABAF1000F5346C1F800A0B8BFF9
:103AB0000AF10703DB1007EE903AF8EEE77A27EEFB
:103AC000800A2DF093FEF7EE007A9FED257A2B69A0
:103AD00077EEC07A9A4567EE877AFDEEE77AC5ED14
:103AE000037A35D07B1EC5F810A09FB200230021B9
:103AF000A9F800706B61AB6159E69FED1A8ADFF897
:103B00007CE0194C194BA8E695ED057AD5ED067ABF
:103B10002068BDEEC77A9A68FDEEE77A92FBF0F274
:103B200017EE109A124817EE90CA0280A0F8029081
:103B3000A0F804C096E69FED0B8A0C4B54E60D4AA4
:103B40000D4B12681C6817E702F5FF521F3238E769
:103B50000027CBE79000012008942537B1DC423ED6
:103B6000D048874A00000000F8280120E8280120FA
:103B7000584C012000270120FC380120F4280120A6
:103B80002DE9F8432F4B1B685B0701D4BDE8F88390
:103B90002D4C2E4D94F82490B9F1010F47D12B6A8A
:103BA000284698476B69284698476B6A04F12C00B1
:103BB00004F128019847276B254B07F10108A668F7
:103BC0009B79E06A984523D0636B5A1C032A24D062
:103BD0002049626394F8382041F8230022BB04EBAB
:103BE0008707002104EB88022B8AF863D26BC4F8A4
:103BF0003080B61A84F824103044A060002BC5D061
:103C0000154A0A2B1268B8BF0A231361BDE8F8836E
:103C10004FF0000884F80090D6E701210D4A0023F8
:103C200084F838109060636321F082FED7E7AB69B7
:103C300028469847EB692846984701226B8A84F802
:103C40002420DBE7744F01200423012010C701204A
:103C50001CB80120F493012030B80120F8B5554B71
:103C60001B681C0700D4F8BD534C0646534F544DF7
:103C700004F1FC007B689847B4F9FE20B4F90031E8
:103C80002846B4F9FCE0397E6A60AB60C5F800E014
:103C900010F0DAF84B4A137859073ED4D4F80401EF
:103CA000494B1B7883B1494B2968B3F90620B3F916
:103CB00008E0B3F90A70891AAB686A68DB1B2960EF
:103CC000A2EB0E02AB606A600028CCD0301A404BE9
:103CD000984242D9B4F908210021B4F91031B4F95D
:103CE00012019B18C4F80411384948BF01335A1017
:103CF000B4F90A311B18CA80B4F9140148BF013362
:103D00005A10B4F90C311B180A8148BF01335B10FB
:103D10004B81BDE8F840FAF797BA23F004032D4F22
:103D20004FF0000EB5F9001013703046B5F90420BD
:103D3000B5F90830C4F80461C7F800E0A7F804E05A
:103D4000A4F80811A4F81011A4F80A21A4F812216B
:103D5000A4F80C31A4F81431A2E70020FAF76AFDA8
:103D60002B68B4F908219342B4F91021B8BFA4F824
:103D700008319342B4F90A21C8BFA4F810316B6826
:103D80009342B4F91221B8BFA4F80A319342B4F9AE
:103D90000C21C8BFA4F81231AB689A42B4F91421BF
:103DA000C8BFA4F80C319A42BFF65DAFA4F8143135
:103DB000F8BD00BF744F01200423012044400120BE
:103DC000F04B0120784F01209C40012094BC012041
:103DD0007FC3C9019ABC012044F620631A46744B84
:103DE0002DE9F04F821895B01C7880461146069256
:103DF000704A1160002C00F02C856F4A12689042C6
:103E000040F230826D4A013C6D4917681C7007F41E
:103E10008057DFF8E4B16B4C04920391002F40F01F
:103E20002E82039B5B7D002B40F09E84049B1B68CD
:103E30001D0400F18B87644B9845A37800F27B83C7
:103E4000002B40F07B83614B0693049B1F6817F4A3
:103E5000805940F0FB83039BBBF906605B8B9E425D
:103E6000B4BF002601265A4B1B6813F0805300F0A4
:103E70001082069A127812F0010200F01182039962
:103E8000498C07EE901A5349F8EEE77A91ED037AE0
:103E9000B4EEE77AF1EE10FA81F22580002E40F0C0
:103EA00006824D4D95F8B811002940F000824B482C
:103EB0004B490568002095F82D50086048608860DF
:103EC0004849002D40F0F4810D70002A40F0F58142
:103ED000454B1978002952D1039ABBF900E0578B62
:103EE000908BBE45CCBF80220022BBF90250BBF9AB
:103EF00004C042F040038645A8BF1346BBF906E064
:103F00009B0843F08002BD42C8BF134643F0400205
:103F10008542A8BF1A46304D920895F8BA9142F0F2
:103F20008003BC45C8BF1A4642F040038445A8BF81
:103F300013469B0843F08002BE45C8BF134643F0BA
:103F400040028645ACBF18461046814501F05A81B3
:103F50000A46A5F8BC1185F8BE11244B85F8BA01B4
:103F60001F78002F01F0D1805F2801F031816F2888
:103F700001F01480069B1B78D80740F1D587049B7D
:103F80001B4A1B68059203F00403002B40F0528586
:103F90000023184D0DF1480840F6330AC8F80430E4
:103FA00005F15009192740F28336129329E000BF2A
:103FB000D8B901205CB80120D4B90120B474012023
:103FC0000C770120B4B50120404B4C00CD69012095
:103FD00038BC0120304D012004230120FC38012091
:103FE000703F012088260120DC4601203319012082
:103FF000744F0120C43F0120C8B2012004354D4553
:1040000020D0AA78EB7817FB02619A42F6D26A7840
:1040100017FB036304323BF912205245A8BF5246F6
:10402000B2F5617FB8BF4FF461728A42E6DD9A4211
:10403000E4DC29782429E1D804354046F5F78AFEE6
:104040004D45DED1B34B98E803001F78B24B83E8AF
:104050000300002F00F042840121AF48F5F78AFEEB
:10406000002840F0A081E378002B40F09C81AB4C0D
:1040700023881DB225F00105AEB2B342268000F0C0
:10408000CD86A74D02274FF014094FF0FF080E20F0
:104090002F7085F8019085F802801BF02DFA3946C3
:1040A0009D482688F5F766FE002841F05B8026F0E3
:1040B00002039BB2B34223800AD0994B1421FF2202
:1040C00002250E2059701D709A701BF015FA268873
:1040D000DFF890A2B507934B9AF80010586808BF14
:1040E00081F002010393C1F34001FAF749FD242155
:1040F0008948F5F73FFE30B9069A1378590702D57B
:1041000023F004031370059B1B6813F00A0F1DD0E6
:1041100005218148F5F72EFE002800F0B486258899
:104120006F0740F1D58706217B48F5F723FE00286D
:1041300000F096866E0640F1C38707217648F5F7B2
:1041400019FE002840F03383059B1B68980600F198
:104150003E8326880C217048F5F70CFE002800F0FD
:104160003E8146F48073B342238009D06C4B022514
:104170001421FF220E201D7059709A701BF0BCF99B
:10418000694B1B780E2B00F03681082B00F0338131
:10419000049B1B685E054BD5644B1B79002B00F01C
:1041A000E78014215C48F5F7E5FD002840F0E58044
:1041B00023F0A8F801201BF0E1F80025DFF8A89112
:1041C0004FF0CC0800E0DDB2022D08FB05F705F149
:1041D00001032DD860B359F80760002EF3D1C378DE
:1041E0004FF0030E5249324690F9020051F8233045
:1041F00001210196CDF800E01AF02AF90346CC22FD
:1042000005EB45003146049353B100EB0010013536
:1042100009EB80002FF095FA049BEDB249F80730C6
:104220002BF0DEFD022D08FB05F705F10103D1D9C6
:10423000069B1B78DD0740F1F18001233D493E4A92
:104240000B701370039B9AF80010186801F00101BD
:10425000FAF796FC059B1B685A0700F14F8115B0D1
:10426000BDE8F08F354B364A1F68049307F480573A
:104270000392DFF8F8B0334C002F3FF4D2AD0021A9
:104280002548F5F777FD00287FF4CBAD1EF06AFFD7
:10429000C7E578023FF5EDAD069A127802F001020B
:1042A000294D002185F8B811002E3FF400AE2749B2
:1042B00001200870002A3FF40BAEF9067FF508AE26
:1042C000234A1278D2063FF503AEB9F1000F7FF40E
:1042D000FFAD002B7FF4FCAD7B023FF5F9AD1D4B2C
:1042E0001B78002B01F0F5831B4B9B78002E41F0CF
:1042F00053843BB1194A1A4B12681B689B1A002B56
:10430000C1F287841020104D1BF0F6F8012385F8C8
:10431000B931DDE5D44B012038BC0120AAB501201C
:10432000182B0120F8630120C03F0120CC4C012054
:10433000E46B0408CE69012010270120B474012029
:104340000C770120B4B50120042301208826012028
:10435000784F012033190120A0BC01202C640120DA
:1043600014810120F6630120B8AE0120C8B20120FB
:10437000069B1B78D8077FF51BAF3C2021F00EFD74
:1043800000283FF455AF18F001FE3C2021F0A8FCB6
:1043900000283FF44DAF18F0F9FD3C2021F0A0FCBF
:1043A0000028F0D144E7059B1B689A077FF55FAEB4
:1043B000BC4C2688F3073FF57AAE46F001039E42D7
:1043C00023803FF474AEB84B1421FF2202250E2047
:1043D00059701D709A701BF08FF8268867E626F4D6
:1043E00080739BB2B34223807FF4C0AEAF4B1B7887
:1043F0000E2B7FF4CAAE228822F040039BB29A4271
:1044000023803FF4C5AEA84B02251421FF220E20C5
:104410001D7059709A701BF06FF8B9E6A44B93F8B1
:104420000090B9F1000F5FD1DFF8D882A14F41466B
:1044300018F8030CA8F103053E7920F0B1FB002821
:1044400000F0FB83002E40F04D8405F108016879EF
:1044500020F0A6FB002841F005829749A87A20F0B9
:104460009FFB002800F0FC83022E41F0FF8193495E
:10447000E87B20F095FB002841F0FC819049287DE5
:1044800020F08EFB002800F0FC83042E41F0F68122
:104490008C49687E20F084FB002841F0F3818A4932
:1044A000A87F20F07DFB002800F0FC83062E41F061
:1044B000B681864995F8230020F072FB002840F071
:1044C0007087834995F8280020F06AFB002800F0E7
:1044D000FC83082E40F04F877E4995F82D0020F090
:1044E0005FFB002840F0FC837B4B01221A7020F018
:1044F000DAFD059B1B685A077FF5B1AE032020F05B
:1045000077FB002800F07986238813F008047FF4F5
:10451000A6AE0820714D1BF037F9714BBBF8066051
:1045200018687049704A714B2E80086014601C60D6
:1045300015B0BDE8F08F0BB90123A3706C4B1B20A5
:1045400094F821601D46069320F052FB012E2F782F
:10455000059007F0010900F0388607F0020794F88B
:104560002030B246DFF8A081624D052B62D8DFE82B
:1045700013F0540047000600D500F9008500BAF199
:10458000010F00F09584B9F1000F00F04F81039BFB
:104590000022B8F80000B3F918101346564E61F324
:1045A0000F0261F30F0360F31F4261F31F43316891
:1045B000CBF804206269CBF800308A42C1F01D8339
:1045C000BAF1010F41F0F38294F820300327CCE7D1
:1045D00020F03AFB012801F0B280059B23B198F846
:1045E0000630002B40F09280BAF1010F22D0424EEB
:1045F000226933689A42C0F05886012384F820303B
:10460000BAF1010F3AD098F80730012B00F017816A
:104610000CF0DCF894F82030A7E7B9F1000FD7D1FF
:10462000059B4FF48060002B00F016841BF0ACF863
:1046300000232361002F3FF408AC38461AF05CFFDA
:10464000049B1F6817F480593FF405AC1D212B48CB
:10465000F5F790FB00287FF4FEAB294A039BD28834
:104660001B8BBBF90660991A8E4240F31B861344DC
:104670009E42B4BF00260126FFF7F5BB1E4E3168EF
:104680006420B8F80230002200FB03134FF480606E
:1046900084F820202361E2701BF05EF894F820304B
:1046A00063E700BFAAB50120182B0120C03F0120FD
:1046B000CE690120900001200C2A0120112A01203E
:1046C000162A01201B2A0120202A0120252A012048
:1046D0002A2A01202F2A012010270120F02601205C
:1046E000544F0120FC260120F4260120EC26012055
:1046F000CD690120D8B501202C64012038BC0120EF
:10470000F42A0120022A0120102B01200CF05EF86F
:1047100003224FF47A7384F82020E361AB4E2B8898
:1047200043F002032B801EF01DFD32680421E36973
:1047300084F820101344A361BAF1010F40F0A98559
:104740003368A2699A42BFF475AFA14B187820B9BB
:1047500020F04EFA00287FF46DAF2B8823F002037F
:104760002B808CE7994EE7E7039A013BD27D3BF91A
:1047700013301AB140F6B832D21A13B2A3F57A73D5
:104780009FED947A944AB3F57A7FA8BF4FF47A7379
:1047900023EAE37307EE903AF8EEE77A67EE877A5A
:1047A000FCEEE77A17EE903A1380FFF744BB8B4B91
:1047B0008B4AB3F904308B4982FB0302DB17C3EB4E
:1047C000A202059B1B680A8098067FF5C2AC864B47
:1047D0001B78990704D5854F3B7D042B00F26F852C
:1047E000268816F0300F3FF4B5AC10201AF0B4FF55
:1047F00020201AF0B1FF7E4B002226881A7000207C
:104800007C497D4B7D4A086010607D497D4A186077
:104810000023486088610B608B604B61CB61136043
:104820005060936053619061D36193E4674E336845
:1048300047F230520323E26184F820306FE70BF037
:10484000C5FF032240F6B833604E84F82020E361B0
:1048500065E76D4F3B78002B00F09C876B4BDFF8D2
:10486000C091DFF8C0B198464D46DFF8BCA15E4666
:104870000393049028E018F804109847032C02B220
:104880001ADC0246C0B139F824E040F6CA016B8850
:10489000A0EB0E02A3EB0E004FF47A7340F2EE2E63
:1048A00003FB02F292FBF0F21A448A42A8BF0A46C6
:1048B0007245B8BF724612B201343B782AF8022F13
:1048C00004359C4280F2DA80072C3046DBF8043055
:1048D000E1B2D0DD3046984702B2EDE7DFF84CA1F7
:1048E0004FF00108DFF848910AF15A06484D514649
:1048F0001AF8010C20F054F9F8B19AF804109AF85B
:10490000023001EB410E9AF80300013B08FA01F175
:1049100005EB8E0E03EB4303DEF8CC214B449342B0
:104920000BD095F8F8218EF8C80122EA0101CEF8E3
:10493000CC31CEF8D07185F8F8110AF1060A564547
:10494000D5D134494FF00009204A334B334D096823
:104950001B78A5F5E47AD2F80080089107936B687C
:1049600063B31E7856B3AA68A8EB0202002A0BDBD9
:1049700001219AF8F82108F5FA7001FA09F1A86006
:1049800022EA01028AF8F821079ABAB12A785978FE
:104990000432D2B2002940F0AC8203993BF91220D4
:1049A000098B01F1C800824240F345849AF8F8115E
:1049B0009A7841FA09F3D80740F1D88409F101093E
:1049C0000C35B9F1040FCAD1FFF746BB2C640120A6
:1049D00033190120AAF1823FA8B50120584F0120C8
:1049E00067666666E4260120784F01207C4F01202F
:1049F000CA4801205C2601206C270120C049012003
:104A000070490120984901202CBA01200C7701201F
:104A1000042301204C81012075B50120CC24012004
:104A200044BA0120243901201A2401201929012027
:104A3000F03F0408AC4D95F8C23153B1069B1B788A
:104A4000DE0706D5039BBBF906205B8B9A4200F379
:104A500063841121A548F5F78DF9002800F0318213
:104A600095F8C6312BB995F8C03113B93223A5F8A2
:104A7000C431012385F8C631FFF78ABADDF810800A
:104A80009B4A42F201099B49A2FB082A0A68049149
:104A90004FEA9A1A12EA090900F00F8296489749DC
:104AA00090F800E0964C0878964984F800E0087089
:104AB000BEF1000F04D0934991F800E08EF0010E92
:104AC000894D0F2185F83C11002B00F02B838E4B74
:104AD00012F4805F039C039A0C938C481B78968C8D
:104AE0004FF00002A0FB03C0B4F818C009933B7854
:104AF000674608BF374640080A9105F5A07111972F
:104B000000EB4000E78C099C08970AF59677201A7D
:104B1000CDF814E00E979E4695F83D71C0B2CDF8E1
:104B20003C800D9710954D46DFF8FCB1784FDDF8CD
:104B30003490DDF83880CDF82CC00790059B002B11
:104B400000F04182734830F9124050001FFA84FC93
:104B5000B44503D3089B9C4540F2738257F822402A
:104B6000A24580F038823BF90040002D40F04A8297
:104B700001322BF8004006317245DFDB0A984946C6
:104B8000109D73460F28644ADDF83C800CBF01215C
:104B9000002185F83D9185F83C01117000F0C98233
:104BA0005E4D01205E4CDFF8A0A12E88DAF80020CF
:104BB000A16846F00406E260521A61682E808A42BB
:104BC0004E4E504D3070287002D9002284F82120BA
:104BD000002B00F0C282049A03991768B1F824C030
:104BE00017F48057B1F818E04E4E40F0CC823946A9
:104BF0004D4835460DE06A7802EB820202EB8202F4
:104C000002F2EE2292B20131023520F8022B8B42E1
:104C10000DD016F81120002A00F01682022AEAD0E0
:104C200002880131023520F8022B8B42F1D10C9A17
:104C3000137801331370FFF7F1B808F105016879B3
:104C40001FF0AEFF00283FF408AC012E40F00A86AA
:104C500005F10D01A87A1FF0A3FF002840F0068699
:104C60003249E87B1FF09CFF00283FF407AC032E7D
:104C700040F000862E49287D1FF092FF002840F06A
:104C8000FD852C49687E1FF08BFF00283FF407ACA0
:104C9000052E40F0F7852849A87F1FF081FF0028E6
:104CA00040F0BD85254995F823001FF079FF0028C5
:104CB0003FF407AC072E40F07483214995F8280093
:104CC0001FF06EFF002840F056831E4995F82D0016
:104CD0001FF066FF00283FF407AC092E3FF404AC38
:104CE0004FF009094B4649E30423012038BC012059
:104CF000D34D6210B474012038B80120F01D01209A
:104D000075B50120F11D0120D9B90120ABAAAAAACD
:104D1000DCB901201C2401201A4C0120D8B5012047
:104D2000B4B5012078BA0120C8B20120112A0120AF
:104D3000162A01201B2A0120202A0120252A0120D1
:104D40002A2A01202F2A01202C640120CE4DD5F8DB
:104D5000A031A8EB0303002BFFF66DA8CB4ACC4B88
:104D6000527C0398069933F8122095F8A431C5F8BF
:104D7000A01192B2817D013392FBF1F203F00F0397
:104D8000C17DE81885F8A43180F8A82195F8A931EB
:104D900095F8A80195F8B721184495F8AA3103446D
:104DA00095F8AB01184495F8AC31184495F8AD313D
:104DB000034495F8AE01184495F8AF31184495F8BE
:104DC000B031034495F8B101184495F8B231184454
:104DD00095F8B331034495F8B401184495F8B5310A
:104DE000184495F8B63103441A4442F30B12642A6E
:104DF000A8BF642213B209B1C2F1640307EE903A6E
:104E00009FEDA47AA44AF8EEE77A67EE877AFCEE83
:104E1000E77A17EE903A1380FFF70DB802219F480A
:104E2000F4F7A8FF00283FF442A92580B7073FF513
:104E30004FA946F00203B34223803FF449A9984B9F
:104E400002201421FF2218700E2059709A701AF057
:104E500053FB2688FFF73CB91AF07EFCFFF7E8BB4E
:104E600025F040039BB2AB4223803FF466A98C4BF4
:104E700002251421FF220E201D7059709A701AF01D
:104E80003BFBFFF75AB9238823F00405ADB2AB42D0
:104E900025803FF448A9824B02251421FF220E20D1
:104EA0001D7059709A701AF027FB2588FFF73BB9DF
:104EB000052384F82030FFF766BB7A4991F800E0BB
:104EC000F6E595F8C031002B3FF462A8069B1B78ED
:104ED00013F001037FF45CA8012285F8C03185F846
:104EE000C121FFF755B8684D012185F8B811FFF7CA
:104EF000DEB9012900F0E88301239AF8F8210C3586
:104F000003FA09F309F101091343B9F1040F8AF80F
:104F1000F8317FF424ADFFF79FB8069B624A1B78F7
:104F20001060DF0700F1068295F8BE1100297FF4BA
:104F300026A8B5F9BC31322B7FF721A895F8BA2104
:104F40000120572A85F8BE0100F06D84049B1E687D
:104F5000770706F0040302D55A2A00F0CA855D2AB5
:104F600000F0CD845B2A00F027855E2A00F088855A
:104F7000562A00F09F85972A00F0CD85A72A40F099
:104F800085844A49049B0A781B6842F00402484819
:104F900003F0040305900A70FEF7F7BFB2F5FA7F3D
:104FA000FEF6EDAF95F8BE21002A7EF4E8AF069B31
:104FB00001211B7885F8BE11DD0700F1AB841EF0DE
:104FC00045FCFEF7DCBF002E39D057F822405000D8
:104FD000A245FFF4C8AD374B5FFA82FC1C5C03446A
:104FE000002C3CD0022C4BD15C7804EB840404EB05
:104FF000840404F2EE24A4B2032A38DD24B2002D86
:105000003FF4B6AD079B21F81340B9F1000F03D16F
:10501000099B022B7FF6ACADB1F800C04FF001093F
:105020004C88254B6444B1F804C0644424B283FB2B
:10503000043C224B1C52ACEBE47424B298E5344699
:10504000500047F8228090E5CAB2022A05D9032A07
:1050500062463FF4D8AD0288E3E57246D3E5BCF181
:10506000020F40F22C83BCF1030F09D1119C0123E4
:1050700024B203FA02FC0A9B23EA0C030A9374E5A8
:105080003BF80040B8E700BF042301207C64012006
:105090009864012014AE2341A8B5012038BC01203A
:1050A000182B012075B5012018810120784F0120AF
:1050B000744F012078BA0120565555558C24012093
:1050C00045F04003AB4223807FF4D1AEFFF735B803
:1050D00045F004039D4223800AD0BE4B02251421D3
:1050E000FF220E201D7059709A701AF005FA25885B
:1050F000B94BBA4AB3F90430B94982FB0302DB1752
:10510000C3EBA2030B80FFF70EB83946B548F4F79E
:1051100031FE00283FF401AF85F8BF711EF096FB09
:10512000FEF728BFB04A0121B048DFF8C8B20C90A2
:1051300011701B21AB480593F4F71CFE059B00285A
:105140007FF42EADAA4CDFF8CCA2E268DAF800308A
:10515000A3609B1AC82B00F23E83049B1F6807F4D0
:10516000805764E526F001039BB2B34223803FF4ED
:105170005DAE0E202F7085F8019085F802801AF040
:10518000BBF9268852E600219A4835460EE06A7837
:1051900002EB820202EB820202F2EE2292B20131B3
:1051A00020F8022B023599423FF441AD16F8112048
:1051B0001AB1022AEBD00288F1E75FFA81FC72464D
:1051C000BCF1030FEBD90288E9E70027FFF7C7B965
:1051D000B2F5FA7FFEF6D3AE95F8BE31002B7EF421
:1051E000CEAE069B01211B7885F8BE110B4000F066
:1051F000D5821DF0B7FFFEF7C2BE08201AF0ACFA48
:10520000FFF72DB87C4A47F6FF717C4B1768B5F95C
:10521000BC21FF6983FB07E3FF179B11A7EB030E7C
:1052200071448A423EF799AEDB1B1A4412B2A5F8CC
:10523000BC21FEF792BEC8398A425FDA9AF8F811AB
:105240009A7841FA09F3D9073FF5B8AB52420120E9
:1052500009921AF069FA731E099A162B00F202815C
:10526000DFE813F0CF01E301B8010802F7011A02E9
:10527000A50192017D01680153010001080240016E
:105280001A02A50192012B0117010301F000DA00B7
:10529000A3003268E3691344A361002F3EF4D5AD47
:1052A000FFF7CBB90126FEF7DEBD0BF08FFA032224
:1052B00040F6B83384F82020E361FFF730BA0A20C3
:1052C0001FF096FC26888046002800F04282F206F5
:1052D00040F12A834A4D95F80882B8F1000F7EF418
:1052E00039AF0D201AF008F90123268885F8083215
:1052F000B8F1000F7FF483AAFEF72CBF01229AF8C1
:10530000F83108F5FA7102FA09F2A96023EA0203FA
:105310008AF8F831FFF752BB00213248F4F72AFD32
:1053200000287FF496AB322385F8C201A5F8C4317A
:10533000FFF78FBB334B1B78002B3EF420AEE37896
:10534000002B7EF41CAE95F8BF310133DBB2032B8A
:1053500085F8BF317EF613AE2B4B5B7813B9002E68
:105360007EF40DAE1DF0FEFEFEF704BE002A0CBF5B
:10537000012002206CE74FF008094B4603EB830342
:1053800087F804901D44A97868780CF025F8069BEE
:1053900001211E4A1B781170D9077FF5A8A8FEF7D6
:1053A00051BF4FF007094B46E8E7DAF8FC01184F08
:1053B00090F83610BB7811446429A8BF642121EA13
:1053C000E17180F83610002B40F0098429F06CFC64
:1053D00092E500BF182B0120584F012067666666D2
:1053E000E049012038BC01201A4C0120D9B9012024
:1053F000B4B50120C8B2012030B80120D34D6210ED
:105400000423012075B50120A0BC01201027012034
:105410003C4601202C640120DAF8FC01A94F90F8E9
:105420003710BB781144FE29A8BFFE2121EAE171A3
:1054300080F83710002BC9D016201FF037FCDAF89F
:10544000FC01C3E708989F4F41781144B1F5967F5E
:10545000A8BF4FF4967121EAE1714170BB78002B2F
:1054600040F0B683DAF8FC01B0E7DAF8FC01954FBA
:1054700081781144C829A8BFC82121EAE17181704F
:10548000BB78002BA2D014201FF010FCDAF8FC012E
:105490009CE7DAF8FC018B4F41781144C829A8BF7A
:1054A000C82121EAE1714170BB78002B8ED0132016
:1054B0001FF0FCFBDAF8FC0188E7DAF8FC01814F09
:1054C00001781144C829A8BFC82121EAE1710170FF
:1054D000BB78002B3FF47AAF12201FF0E7FBDAF81D
:1054E000FC0173E7774F0898BB7841791144642930
:1054F000A8BF642121EAE1714171002BB2D00E20D6
:105500001FF0D4FBDAF8FC0160E7DAF8FC016D4F1C
:10551000017ABB781144C829A8BFC82121EAE171EA
:105520000172002B3FF452AF0B201FF0BFFBDAF8E3
:10553000FC014BE7DAF8FC01624FC179BB781144FA
:10554000C829A8BFC82121EAE171C171002B3FF42D
:105550003DAF0A201FF0AAFBDAF8FC0136E7DAF8C3
:10556000FC01584F8179BB781144C829A8BFC821D4
:1055700021EAE1718171002B3FF428AF09201FF06F
:1055800095FBDAF8FC0121E7DAF8FC014D4F41798F
:10559000BB781144C829A8BFC82121EAE171417133
:1055A000002B40F00783112E7FF462AF0EE7DAF88C
:1055B000FC01444F0179BB781144C829A8BFC82118
:1055C00021EAE1710171002B40F04683102E7FF437
:1055D00063AFFBE608993B4F0E791644642EA8BFD3
:1055E000642626EAE6760E711FF07AFBBB78002B64
:1055F0003FF438AF032031461FF058FBDAF8FC01C6
:10560000E4E608982F4F01781144FA29A8BFFA213F
:1056100021EAE1710170BB78002B3FF423AF012038
:105620001FF044FBDAF8FC01D0E60898254F81789A
:1056300011446429A8BF642121EAE1718170BB781B
:10564000002B3FF40FAF02201FF030FBDAF8FC0113
:10565000BCE608981B4FC179BB78114481F308015F
:10566000C171002B3FF4FEAE05201FF01FFBDAF8DE
:10567000FC01ABE6089B134F9979B8781144642973
:10568000A8BF642121EAE1719971002840F09A8253
:105690000D2E7FF428AFE5E6DAF8FC01094FC1785A
:1056A000BB781144C829A8BFC82121EAE171C170A3
:1056B000002B40F069820F2E7FF402AF86E60B9C30
:1056C0009AE400BF3C46012098784FF496613BF97C
:1056D0001230B3F5617F91FBF0F252DB40F63301FB
:1056E0009942A8BF19460C2EA1F5617191FBF2F108
:1056F00000F07C81182E7FF4FFABC9B2C8290B469D
:10570000A8BFC823DAF8FC21D8B2D67DB0423FF456
:10571000F3AB9B1BC34FD07548BF0733DE10BB787C
:105720000136F6B23BB9002E3FF4E6AB304619F035
:10573000FBFFFFF7E1BB18201FF0B8FAF3E7BA4E02
:105740006421B8F80230326801FB03232361FEF7BD
:1057500044BFF30600F14C810B201FF049FA0028EA
:1057600040F0F880B70600F15481B04D95F808324A
:10577000002B3FF4B6ADB8F1000F7FF440A8FEF760
:10578000E9BC0C2E00F01C81182E7FF4B5AB002173
:105790000B46B7E7A64A0392FFF772B9A549096815
:1057A00011F4003140F02E810B46A348C65C0C3347
:1057B0000F2E1ED001311529F8D1FA3A049B002191
:1057C0001B68A5F8BC219D4A03F0040385F8BE11AF
:1057D0000592FEF7DABB9A4A0121138884F821105A
:1057E000049923F004030F68138007F48057FFF730
:1057F0001EBA944E4B0037683FB197F801E05F182E
:1058000000EB87077F787745D7D20B448E4F002176
:1058100000EB83008D4B398030601960CDE74FF08D
:1058200006094B46AAE58A4A4FF47A7389491268F9
:10583000B3FBF2F3C3EB4310049A03EB800312684B
:10584000DB00A1F8B830110600F127817B4B0593EE
:105850001B685B0700F11881049B1B6803F00403BD
:10586000FEF793BB4FF001094B4687E54FF0020965
:105870004B4683E54FF003094B467FE54FF00409A3
:105880004B467BE54FF005094B4677E50021BB2AE7
:10589000129100F07681B72A00F06F81BE2A00F0E5
:1058A0006A81BD2A00F04381792A00F0CE817A2AEC
:1058B00000F0C4819E2A00F0BB819D2A00F0B181D6
:1058C000AE2A00F0F681AD2A00F0EC81EF2A00F05C
:1058D000E381FD2A00F0DA81FB2A00F0D181FE2A63
:1058E00000F0C881F72A00F0BF817B2A7EF447AB25
:1058F0004FF4FA6102201EF04DFAFEF740BB564B02
:1059000000220120554D56492A700B6019F00CFFFA
:10591000FEF735BB5349049B0A601B68474A03F0F6
:1059200004030592FEF731BB1020404D19F02CFF07
:10593000202019F011FF4C49081F0BF057FC4B4B6E
:1059400002221A7095F80832002B00F05E8126883A
:10595000FEF755BF464A474B528993ED007A07EE52
:10596000902AB0EEC77AF8EEE77AB4EEE77AF1EE75
:1059700010FA7FF5F7AE93ED017AB0EEC77AF4EE48
:10598000C77AF1EE10FA7FF7EDAEB3063FF5EDAE54
:10599000264D202019F0F8FE05F5017105F500707F
:1059A00097E80C00C5F80022C5F804320BF01EFC85
:1059B0002E4B01221A70C5E72F4B01220220A1E7CE
:1059C00000263146254B09915B78B3423FF494AAF7
:1059D000144F30461EF04AFA0999BB781BB1C9B280
:1059E0000C201FF063F90136F6B29CE6CEB2E9E76F
:1059F000102019F0B1FE1D4B268883F800804FF06F
:105A00000108A9E61D490978032900F0F980194623
:105A1000CBE62020054D19F09FFE144B00221A7092
:105A200090E700BF3C4601202C64012004230120A4
:105A30000C7701200C29012020560408744F012006
:105A4000D8B5012034260120D2260120D4260120F9
:105A5000A4740120B86C012020450120EE380120FB
:105A6000FC3801201881012010490120CA4801207A
:105A700064490120304D01206E450120B0B5012060
:105A80008F4B022203203DE7049B0A218D4A1B68AD
:105A9000118003F00403FEF778BA8B4B1B789A074A
:105AA0007FF5D4AE894B1B7D042B7FF6CFAE0BF078
:105AB00023FBCBE622F000FEF3F794FB22F0E4FD9B
:105AC000F8F708FA012019F02FFE95F8BA21FFF730
:105AD00052BA002E3EF416AC7D4D95F8B931002B2C
:105AE0003EF4F6A919F0ECFC002385F8B931FEF775
:105AF000EFB995F8C021002A77D195F8C23183F02B
:105B0000010385F8C231002B6DD10C20714B059338
:105B100019F0F2FCA0E6704A4FF4C871049B1180A2
:105B20001B686C4A03F004030592FEF72EBA4FF689
:105B3000FE736A4A674896890590D08933440144C8
:105B40009381D18122F0B8FDF3F74CFB22F09CFD4C
:105B5000F8F7C0F9012019F0E7FDB5F8BC21049B66
:105B60000021FA3A1B6885F8BE1103F00403A5F87A
:105B7000BC21FEF70ABA0223DBE70B464FF6FE71A3
:105B8000D7E70B460221D4E70F2009921FF08EF8C9
:105B9000DAF8FC01099A8EE5002B9DD050494FF4AC
:105BA0007A70504A096800FB0313136094E70327D7
:105BB000FEF743BD112009921FF078F8DAF8FC01D6
:105BC000099AF0E40D2009921FF070F8099A5FE538
:105BD00015201FF06BF8DAF8FC01FFF7F7BB172070
:105BE0001FF064F83EE40B2090E73A4A85F8C011B4
:105BF00085F8C1010592FEF7C8B90327FEF718BE64
:105C000019F05EFCB5F9BC21D7E54FF00108FFF7AC
:105C100068BB1DF0A7FA2E4D002385F8B931FEF7B9
:105C200057B90021FF202BF0F9FA95F8BA2147E681
:105C300001202BF0F3FA95F8BA213EE62A4A137AAE
:105C400043F001031372FEF79AB9274A137A23F03F
:105C500001031372FEF793B9102009921FF026F882
:105C6000DAF8FC01099AB1E4002104201EF092F850
:105C7000FEF785B9002103201EF08CF8FEF77FB9EE
:105C8000002102201EF086F8FEF779B900210120DC
:105C90001EF080F8FEF773B9002108461EF07AF86E
:105CA000FEF76DB9FF2100202BF0B8FA95F8BA2164
:105CB0000CE6012100202BF0B1FA95F8BA2102E69A
:105CC000BC4501206A810120784F01207C4F0120D2
:105CD00004230120744F01206C81012084BC012029
:105CE0002C64012014810120004C0120434B2DE93C
:105CF000F04F2DED0A8B1B7891B0012B029001F033
:105D00003880DFF804B19BF80021002A41F0408080
:105D1000072B01F047804FF00009DFF8F0A0DAF818
:105D2000043050469847002800F065810022BAF8F8
:105D3000B8508AF85920002D40F0F286BAF9424056
:105D40000AF13400DAF82C20DAF82830A21ABAF96D
:105D50004060BAF94410F61ACAF83820DAF8303040
:105D6000274ACB1A9AF85A101446CAF83460CAF86F
:105D70003C3000920EF068F82368990040F1E08012
:105D80009AED0E7ADAED0D7AB8EEC78A9AED0F7AAF
:105D9000DBF81031F8EEE77AF8EEC78A194A9BED86
:105DA000416A0133DBED426A9BED437A77EE867AF6
:105DB000126838EE268A78EE878ACBF81031934243
:105DC000CBED417A8BED428ACBED438A01F07083B3
:105DD0000A4B1D78142D02F0D1830023DBF8184103
:105DE0000193062C00F29F80DFE814F07A1246112E
:105DF000E210561312000E12661100BF544C01201F
:105E0000B4740120003C012010250120B86C012051
:105E1000D44B1A78DBF81C61D34FF0009FEDD37A96
:105E20003B1883ED007A002A73D0B0EE476AD04960
:105E3000F0EE476A00230133F1EC017A05EE903A67
:105E400067EEA77A9342F8EEE55A87FE277A76EE58
:105E5000A76AA7EEA56AEED1F5EEC06A3B1883EDFE
:105E6000007AF1EE10FA54DDC6EE265AC14AC24B52
:105E7000D2ED007A1A88B7EE007A75EEC75A65EE51
:105E8000A77AFDEEE77A17EE903A812B43F347822B
:105E90009342A8BF134607EE903AF8EEE77A8119CD
:105EA000B64B03EB810393ED007A93ED056A93ED16
:105EB000015AA7EE276AD3ED066A93ED047AE5EE60
:105EC000276AD3ED034A93ED025A27EE467ABDEED8
:105ED000C64AE6EE646AA5EE277A14EE101A812906
:105EE000C3ED056A83ED067A43F31D828A42A8BF9B
:105EF0000A4607EE902AF8EEE77AFCEEE77ACDED57
:105F0000037ABDF80C303A18938016B9132D03F0BC
:105F10008086152D42F0A3803844DBF81841984F55
:105F2000838827F816300134964A82FB0432E3173F
:105F30002244C3EBA203C3EBC303E41ACBF818411A
:105F4000914B1B78002B01F05780904C0025CDF829
:105F500004908F4F04F2DC66DFF82482DDF80090B5
:105F60008C4B1B78172B01F07F8494ED007A082B63
:105F7000DAED097AB8EEC78A28EE278A07D1B0EEA3
:105F8000480A00932BF0C2FA009B28F81500D9F8B4
:105F9000002092000BD5002D04F01381B0EE480ACA
:105FA000DAF87C3706F170009847B0EE408AB0EE20
:105FB000480ADAF89C36A6F170009847DAF80C37F0
:105FC00030469847734BB0EE408A1B78032B01F0A4
:105FD0005B840135D4F85C06B0EE480ADAF8BC30D0
:105FE0009847032D06F1240604F10404A7EC010AE6
:105FF000B6D1DDF80490674B1E78072E00F04E8670
:106000009BF828310493002B40F05486624B5B7957
:10601000002B40F0608501235E4A8BF8283112780E
:10602000072A01F07685002305935C4BF7EE007A92
:10603000DBED4C9A002593ED007A594F77EEE98A13
:10604000584B2C46584ED3F8009007F11C0368EECD
:10605000878ADFF88C810393544BDBED4BBAC8FE83
:10606000E78A0093DFF87CA1514B9FED529ADFED58
:1060700052AA9FED3EBA9FED51AA0193504B97ED66
:10608000008A2B44D3ED007AF5EE407AF1EE10FA57
:1060900017D04C4B2B44D3ED006A38EE667AB0EE45
:1060A000C76AF4EEC67AF1EE10FA08D5B5EEC07AFA
:1060B000F1EE10FACCBF37EEA68A36EEE78A83ED12
:1060C000008A414B1A8893073AD0022C38D03F48B7
:1060D00099F82E1030F91400039B07EE901A07EE82
:1060E000100A60002B44B8EEE76AB8EEC77AD3ED29
:1060F000006A4B42A6EE267A07EE903AF8EEE77A6F
:10610000B4EEE77AF1EE10FA05D407EE901AF8EE45
:10611000677AC7FEC77A2E4B2E490344085EB3F94F
:106120000C30C01A07EE100AD007B8EEC77AE7EEB7
:10613000497A40F1C785284B93ED008A27EE888A7B
:10614000019B9BF868212B44D3ED01CA38EE6CCA41
:10615000002A7ED0DBF86C21204B02991B688A1A3A
:106160009A4241E0063C0120243E0120000000004C
:1061700010250120083C0120043C01203C3E012068
:10618000584C012093244992F83B0120EC6C0120EB
:10619000A8740120544C0120A46C012030C40120BB
:1061A00044260120FC380120703F0120643F01207B
:1061B000A4740120CDCCCC3DAE47813F0000C84245
:1061C00024C4012050260120AAB501205C2601200C
:1061D00084BC0120584F01200CC4012038C4012088
:1061E0007C3F012084BF012033DD99F84830022B29
:1061F00001F0C384022C03F06D87D14B1B68990713
:1062000040F1E186CF4BD04903EB4400DFF8BCC33B
:1062100031F914E0B0F90C009CED008AA0EB0E0EF1
:10622000CA4828EE098A86ED00BA07EE90EA0068AF
:10623000F8EEE77A904227EE888A38EE6CCAC1F20F
:10624000E880F7EE007AF4EEE79AF1EE10FA01F149
:10625000B780BF4B022C2B4493ED000A009B2BEE22
:10626000800A20EE0C0AA3EC010A009303F0558784
:10627000B84ADAED006AD2ED007AB74B66EEA77A3B
:1062800096ED006A2B4467EEA87A93ED007AB34B43
:1062900067EE877AD3ED005AB0EE467AF1EE656A82
:1062A000ACEE277AF4EEC76AF1EE10FA01DCC5FE17
:1062B000C76AF7EE007A9BED4C7AB4EEE77AF1EE1E
:1062C00010FAACBF0123002343B1B0EEC66AF0EE72
:1062D000E67AF4EEC67AF1EE10FA01D5C6ED006A60
:1062E000022C58D09E4AB0EE6C0A9E4B52F8240005
:1062F0001B6898479C4A9D4B52F824001B6898479E
:1063000099F8373023B19A4B1B88002B00F04F854A
:10631000B0EE4B8A974B38EE400A9AED007A2B4448
:1063200093ED008A83ED000A30EE480A99F8483070
:10633000C0EE077A2BB3904B1B78DB0721D5B7EE65
:10634000007AF4EEC79AF1EE10FA04DB9BF868319C
:10635000002B00F0E586DBF86C31029AD31A874AED
:1063600012689A420DDD864BB0EECCCA93ED007AEE
:10637000B4EEC7CAF1EE10FA41F1678000238BF842
:106380006831804B2B4493ED007A2BEE877A67EED1
:10639000277AC8ED007A9BF8783133B9009B86EDF7
:1063A00000BA03ED01BA88ED00BA013404370436AF
:1063B00008F10408032C05F104057FF45FAE724B6D
:1063C0001B78072B01F06F82012B01F0A7830023BC
:1063D00001939BF88031002B40F020856B4B6C4A79
:1063E0001B68126813F4805792F82C2040F02C861A
:1063F00068480121408B8BF8981107EE900A664996
:106400006648B8EEE77AD1ED037A6549D0ED006AC7
:1064100091ED006A77EEC77A624976EE665ACBED67
:10642000646A91ED007ACBED626ACBED615A8BED37
:10643000656A5D49C7EE875ADFED5C4A91ED006AF7
:106440005B49D1ED007AB7EE005A5A4936EE276A19
:10645000DFED597A91ED004A584936EE046A91ED24
:10646000007A26EE246AF1EE476AC5FEC55AC5FEDB
:10647000A75AB4EEE66ACBED675AF1EE10FA01F1D5
:10648000AC8186FE476A4849D1ED017A484991EDD1
:10649000015A484977EE857A9FED445AD1ED014A79
:1064A00077EEA47A67EE857AF4EEE76AF1EE10FAF9
:1064B00001DCC7FE676A3C499FED3C5AD1ED027A88
:1064C0003B4991ED027A3E4977EE877A91ED007A69
:1064D00067EE857AF1EE473AF4EEE37AF1EE10FAE0
:1064E00001D4C7FEC73A3749497809B9F1EE633A92
:1064F000002A41F0F381B7EE004ADFF8D4A09AF801
:106500000020002A02F015822F499FED2B7A91ED91
:10651000025AD1ED014A26EE855AD1ED037AA6EE54
:10652000245AA3EEA75A24EE055AB4EEC75AC5FE64
:10653000474A8DED085AC5FE077AF1EE10FA49E098
:10654000744F012084BC0120584F012034C4012025
:10655000E0C3012098000120ECC3012054C40120B5
:106560008CBF012088BF0120E0BF0120DCBF0120DB
:10657000AAB5012080260120CD69012038C4012060
:1065800044C40120F8C30120544C0120B4740120FC
:10659000FC3801200C770120304D0120C8BA0120C1
:1065A00054BC0120FC2A0120643F01206F12833A71
:1065B000703F01207C3F01200000000058C40120F2
:1065C0005CC40120C03F01206C2A01200CC40120C2
:1065D000354C012088BFF0EE474A012A02F0CB81FA
:1065E00091ED067AD1ED052A26EE877A91ED073AEC
:1065F000A6EE227AA3EE837A24EE077AB4EEE77A47
:106600008DED097AC7FE277A87FE647AF1EE10FADB
:1066100088BFB0EE647A022A00F0AD80D1ED0A4A5C
:10662000D1ED092A66EEA44A91ED0B3AE6EE224A34
:10663000E3EE834A64EE244AF4EEE74ACDED0A4ADB
:10664000C4FEA77AC4FEC74AF1EE10FA98BFB0EEB6
:10665000647A032A00F08F80D1ED0E4AD1ED0D2A25
:1066600066EEA44A91ED0F3AE6EE224AE3EE834A43
:1066700064EE244AF4EEE74ACDED0B4AC4FEA77A55
:10668000C4FEC74AF1EE10FA98BFB0EE647A042A4D
:1066900071D0D1ED124AD1ED112A66EEA44A91EDE6
:1066A000133AE6EE224AE3EE834A64EE244AF4EE1D
:1066B000E74ACDED0C4AC4FEA77AC4FEC74AF1EE04
:1066C00010FA98BFB0EE647A052A54D0D1ED164A7C
:1066D000D1ED152A66EEA44A91ED173AE6EE224A6C
:1066E000E3EE834A64EE244AF4EEE74ACDED0D4A28
:1066F000C4FEA77AC4FEC74AF1EE10FA98BFB0EE06
:10670000647A062A37D0D1ED1A4AD1ED192A66EEFD
:10671000A44A91ED1B3AE6EE224AE3EE834A64EE88
:10672000244AF4EEE74ACDED0E4AC4FEA77AC4FE31
:10673000C74AF1EE10FA98BFB0EE647A072A1AD071
:10674000D1ED1E4A91ED1D3A66EEA46AD1ED1F4AC5
:10675000E6EE036AE4EEA36A66EE846AF4EEE76AA4
:10676000CDED0F6AC6FEA77AC6FEC76AF1EE10FA33
:1067700098BFB0EE667A77EEC77AF7EE006ACBED97
:106780004C7AF4EEE67AF1EE10FA43F3DE8186EE0F
:10679000A77ADDED097A022A25EE075A67EE877A95
:1067A0008DED085ACDED097A2DD0DDED0A7A032A58
:1067B00067EE877ACDED0A7A25D0DDED0B7A042AD3
:1067C00067EE877ACDED0B7A1DD0DDED0C7A052AC8
:1067D00067EE877ACDED0C7A15D0DDED0D7A062ABD
:1067E00067EE877ACDED0D7A0DD0DDED0E7A072AB2
:1067F00067EE877ACDED0E7A05D0DDED0F7A27EEC4
:10680000877A8DED0F7AB749096811F0805801F049
:106810004580F6EE005ACBED675A002A02F0A580BB
:106820009BED657A03F01001DBED647A03F48009D7
:10683000BDEEC77A9BF99841AB4DAC4806EE904A45
:10684000AB4B17EE10EABDEEE77AAA4E1B78F8EED6
:10685000E66AA94C95ED005A03F0010CA74D17EE1E
:10686000103AC0783678B5F90650648B9BED616AB2
:106870009BED627A002841F05880A148002940F041
:10688000A186D0ED007A9DED085A65EEA77A9D4964
:10689000E5EE267AB0EE475AA7EE865AFDEEC57AA7
:1068A00017EE905A17EE904A7545A8BF7446AB4252
:1068B000C8BF1C46012A07EE904AF8EEE77AC1ED00
:1068C000007A00F0DC80D0ED047A9DED095A65EE87
:1068D000A77AE5EE267AB0EE475AA7EE865AFDEE85
:1068E000C57A17EE905A17EE904A7545A8BF7446C0
:1068F000AB42C8BF1C46022A07EE904AF8EEE77A80
:10690000C1ED017A00F0BB80D0ED087A9DED0A5A06
:1069100065EEA77AE5EE267AB0EE475AA7EE865ADC
:10692000FDEEC57A17EE905A17EE904A7545A8BF4E
:106930007446AB42C8BF1C46032A07EE904AF8EEE5
:10694000E77AC1ED027A00F09A80D0ED0C7A9DEDE5
:106950000B5A65EEA77AE5EE267AB0EE475AA7EE17
:10696000865AFDEEC57A17EE905A17EE904A754595
:10697000A8BF7446AB42C8BF1C46042A07EE904A23
:10698000F8EEE77AC1ED037A79D0D0ED107A9DED7B
:106990000C5A65EEA77AE5EE267AB0EE475AA7EED6
:1069A000865AFDEEC57A17EE905A17EE904A754555
:1069B000A8BF7446AB42C8BF1C46052A07EE904AE2
:1069C000F8EEE77AC1ED047A59D0D0ED147A9DED56
:1069D0000D5A65EEA77AE5EE267AB0EE475AA7EE95
:1069E000865AFDEEC57A17EE905A17EE904A754515
:1069F000A8BF7446AB42C8BF1C46062A07EE904AA1
:106A0000F8EEE77AC1ED057A39D0D0ED187A9DED30
:106A10000E5A65EEA77AE5EE267AB0EE475AA7EE53
:106A2000865AFDEEC57A17EE905A17EE904A7545D4
:106A3000A8BF7446AB42C8BF1C4607EE904A072A5F
:106A4000F8EEE77AC1ED067A19D0D0ED1C7A9DED0B
:106A50000F5A65EEA75AE6EE855AA6EE257AFDEEA8
:106A6000C77A17EE900A8645A8BF86468342D8BFEC
:106A7000734607EE903AF8EEE77AC1ED077ABCF17B
:106A8000000F00F0A586204B1B68002B40F0B1835F
:106A90001E4B1B7893B19AF8000060B1194D002489
:106AA0001B4EE0B23368B5EC010A013498479AF8FE
:106AB00000008442F5DB174B1B689847164B1B7888
:106AC000072B00F0038701238BF8003111B0BDECD8
:106AD0000A8BBDE8F08F114B1B78013BDBB2FFF74F
:106AE0009BBA00BF38BC0120482A0120B4B5012060
:106AF000CD690120787701200C770120C8B20120F0
:106B00006C2A0120983F01207CBF0120807F01205A
:106B10006C77012074770120544C012078BC01204F
:106B2000AE4B4FF47A74AE4901931B68AD4F91F8A8
:106B30000180AD49B7F906000E78B4FBF3F3C3EB5F
:106B4000431403EB8403DC00A4B2A54201F0608689
:106B5000DAF88C10BAF940E0DAF870304A1C07EE27
:106B600090EA7344012AF8EEE77ACAF88C20CAF852
:106B7000703001F05A869AED1F5A07EE102ADAEDAE
:106B8000216A012D77EEC55AB8EEC76A85EE867A7E
:106B900037EE057A77EEC77A8AED207A8AED1F7A8A
:106BA000E7EEA56AF0EE667ACAED226ACAED216ABE
:106BB00001F0FA87DAF8A010BAF942E0DAF8743096
:106BC0004A1C07EE90EA7344012AB8EEE77ACAF845
:106BD000A020CAF8743001F043869AED245A07EEDB
:106BE000902ADAED266A012D77EE455AB8EEE76A6B
:106BF000C5EE867A77EE857A37EE677ACAED257A22
:106C0000CAED247AF0EE667AE7EE257ACAED277AA5
:106C1000CAED267A01F0F187DAF8B410BAF944E047
:106C2000DAF878304A1C07EE90EA7344012AB8EE8D
:106C3000E77ACAF8B420CAF8783001F02C869AEDC9
:106C4000295A07EE902ADAED2B6A012D77EE455A84
:106C5000B8EEE76AC5EE867A77EE857A37EE677A20
:106C6000CAED2A7ACAED297AF0EE667AE5EE877ADD
:106C7000CAED2C7ACAED2B7A01F0F887F880BAF8C1
:106C8000B830594A013B1678AAF8B8300023019968
:106C9000072E4B608B60CB607FF4B2A9F7F70CFC3A
:106CA000504FA0EB09009BF8283138800493002B4B
:106CB0003FF4ACA9013B8BF8283111B0BDEC0A8B35
:106CC000BDE8F08FB1F90020B1F9021082EAE27359
:106CD0009BED577ADBED586AA3EBE27381EAE17230
:106CE00086FE876AA2EBE17240499342B8BF134621
:106CF0000A7807EE103AB8EEC77A27EE097A002A2A
:106D000040F0E5813A4BD3ED005AF4EEEA5AF1EE49
:106D100010FA40F1F986B7EE005ADFED366ADFED82
:106D2000364A36EEC77A354B35EE655AD3ED006AF2
:106D300025EE245AE5EE075A65EEA65AF5EEC05A3E
:106D4000F1EE10FA40F2A685CAEE256AB7EE007A97
:106D5000F0EE475AE6EE665AC5FEC76AC6FE8B6A73
:106D6000274B93ED007A67EE877AA7EEA68AFFF7A6
:106D7000E7B9244A244B1268DFF89CB0D169194F57
:106D80001A889BF8003139807A80002B3EF4C3AF1B
:106D900003F0BCFA144B00221B788BF80021072B60
:106DA0007EF4B9AFF7F788FB8146FEF7B6BF174B05
:106DB000F7EE006A164A2B44D2ED007A93ED007A82
:106DC000144B67EE277A93ED007AC7FEE67A67EEFA
:106DD000877A27EE888AFFF79DBA00BFA474012046
:106DE000A46C0120584C0120544C012018C40120EF
:106DF00020C4012000003443610BB63B14C40120C1
:106E000010C4012030B80120462A01206C26012040
:106E100008C4012004C4012010250120D64BDFF84E
:106E2000B0A31B78DE0740F1D5819AF80030002B23
:106E30003FF429AEDBED583AF3EE046A9BED574A76
:106E4000DBED627AF4EEC43ACC4A77EEA64A9BEDCB
:106E5000617A92ED005AF1EE10FADBED555A9BED96
:106E6000546AC748C74900F1EB8690ED026AB0EE5C
:106E7000674A26EE656AA6EE074AB4EEE44A34EEA7
:106E8000666AF1EE10FA48BFB0EE456A012B81ED5B
:106E9000006A3FF4F8AD90ED066AB0EE674A26EE60
:106EA000656AA6EE074AB4EEE44A34EE666AF1EE8D
:106EB00010FA48BFB0EE456A022B81ED016A3FF43B
:106EC000E2AD90ED0A6AB0EE674A26EE656AA6EE7C
:106ED000074AB4EEE44A34EE666AF1EE10FA48BFAF
:106EE000B0EE456A032B81ED026A3FF4CCAD90ED24
:106EF0000E6AB0EE674A26EE656AA6EE074AB4EE61
:106F0000E44A34EE666AF1EE10FA48BFB0EE456A24
:106F1000042B81ED036A3FF4B6AD90ED126AB0EE3A
:106F2000674A26EE656AA6EE074AB4EEE44A34EEF6
:106F3000666AF1EE10FA48BFB0EE456A052B81EDA6
:106F4000046A3FF4A0AD90ED166AB0EE674A26EEF3
:106F5000656AA6EE074AB4EEE44A74EE666AF1EE9C
:106F600010FA48BFF0EE456A062BC1ED056A3FF402
:106F70008AADD0ED1A6AB0EE674AB3EE046A66EEE7
:106F8000E56AA6EE874AB4EEE44A74EE466AF1EE8C
:106F900010FA48BFF0EE456A072BC1ED066A3FF4D0
:106FA00072ADD0ED1E6A66EEE55AE5EE877AF4EE34
:106FB000E74A77EEC67AF1EE10FAC8BFF0EE457AEE
:106FC000C1ED077A5FE5704B86ED00BA1B6893420E
:106FD000BFF637A96D4A002312888BF86831002A62
:106FE00041F0E4836A4A6B4B1178186881F0010123
:106FF000F7F7C6FDFFF72DB9674D684F05F24C74E2
:1070000005F5F766F5EC017A20469AED090AF8EEE7
:10701000E77ADAF87C3727EE800A9847A4F1E00097
:10702000DAF89C369847A4F17000DAF80C3724346B
:107030009847D5F85806DAF8BC309847A642A7EC2E
:10704000010ADFD1FEF7D7BF4B490978CD0703D43A
:107050005349098BABF88C1152495348098890ED7C
:10706000037A07EE901AF8EEE77AB4EEE77AF1EEDB
:1070700010FA40F293854D48008807EE900AF8EE2A
:10708000E77AB4EEE77AF1EE10FAC0F2578577EEC0
:10709000677A4749BCEEC77A4648D1ED006A17EED9
:1070A000101A90ED007A0120CBED646A37EE666A23
:1070B000ABF88C114049CBED626A8BED657A8BEDB4
:1070C000616A8BF8980191ED007AFFF7B2B93B4BFA
:1070D000D3ED005AF5EEC05AF1EE10FA40F3DA8320
:1070E000374B93ED005AB5EEC05AF1EE10FA40F36B
:1070F000D18326EE4A6A35EE477AF7EE004AC6EEAD
:10710000256A87EE056A76EEA46A86FE646A86FEC4
:107110000B6A66EE266AC6FEE46AC6FE8B6A1FE646
:10712000284AB0EEE77AD2ED006AB4EEE67AF1EEE4
:1071300010FA7FF710A9244AB0EECC7AD2ED006A9B
:10714000B4EEE67AF1EE10FA7FF705A997ED007A32
:107150001E4AB0EEC77AD2ED006AB4EEE67AF1EEDE
:1071600010FA7FF5F8A8012202998BF86821CBF874
:107170006C11FFF7F4B800BFCD690120482A012047
:107180006C2A0120983F012034C4012004640120AE
:107190000664012008640120EC6C0120A874012021
:1071A0000C770120002B0120304D0120022B012003
:1071B000EC2A012054BC0120082B012014C401201A
:1071C0001CC4012048C4012044C401204CC4012037
:1071D000354C01209AF80020002A3FF454AC92006C
:1071E000A149A2482AF064F8A14B1B68002B3FF488
:1071F0004FACA04B1B78192B07D801219E4A01FAEE
:1072000003F31A40002A41F03D859C4B9C4D9D4E56
:1072100000931B689C061BD5F37AFF2B04D09A4A77
:1072200012789A4201F2A081B6F90870F37D2F809E
:10723000FF2B04D0944A12789A4201F29A81B6F94F
:10724000144008206C801DF0D3FC002840F08F868D
:10725000B5F90000B6F90620B6F912E0B5F90280DA
:107260008242B6F904101346A8BF0346C645B5F9D5
:107270000470A8BFC6468842ACBF1A460A46B6F993
:107280001E10B5F906C0B6F92A30B9422A80A8BF47
:1072900039466345B6F91020A8BF63460846424503
:1072A000D8BF7246B5F908E01C46B6F93630B6F9D3
:1072B0001C1073456A80A8BF73468F42A8BF014661
:1072C000B6F94200B5F90A701A46A980B842B6F973
:1072D0002810A8BF38466145CCBF0B462346B5F9F8
:1072E0000C40B6F94E10EB80A142B6F93430B6F935
:1072F0004CC0A8BF21467345D8BF1346B5F90EE070
:10730000B6F95A202B817245B6F94030A8BF7246B3
:10731000BB42D8BF0346B6F95800A445D8BF8C4637
:107320005A4E8645B8BF02466B81A5F80CC0EA816B
:10733000B38923B3564FDFF8749107F11004DFF8D7
:107340004481B7F90230484608F10C0809F12409D4
:1073500000EE103AB8EEC00AF0F734FF2AF0D6F883
:1073600038F9083C00B238F9062C984203DB824217
:107370001346A8BF034627F8023FA742E1D13D4B81
:107380001B78013B182B01F2CC82DFE813F02609B1
:10739000CA0ACA0A2A02CA0ACA0ACA0A0909CA0AB7
:1073A000CA0ACA0ACA0ACA0A5A09CA0ACA0ACA0AAE
:1073B000CA0ACA0A2A021709CA0ACA0A5A0926099F
:1073C000019A344BD2ED017A93ED007AF0EEE77A30
:1073D000F4EEC77AF1EE10FA7EF53BAFD2ED027A09
:1073E000F0EEE77AB4EEE77AF1EE10FA7EF731AF1D
:1073F000D2ED037AF0EEE77AB4EEE77AF1EE10FA26
:107400007EF727AF244B1B689A077FF5E3AD23492E
:10741000234BB3F90C20B1F900E02248AEEB020E89
:1074200000688EEAEE72A2EBEE728242BEF611AFF7
:10743000B3F90E30B1F90220D21A82EAE273A3EB5B
:10744000E27398427EF705AFC4E597ED007A164BDC
:10745000B0EEC77AD3ED006AB4EEE67AF1EE10FA38
:107460007EF78FAFFEF78ABF4C2A0120983F01209C
